:100000005446495300010000E41C02009A0BE8FE2C
:1000100009390113181218174A50504F09390202B2
:10002000181218174A50504F0939010318121312A9
:100030004A50504F03000000000000000000000084
:1000400054464353002000006804020000000000F2
:100050000000021001210000252100004D350100A3
:10006000292100002B2100002D2100003D2100004E
:100070003D2100003D2100003D2100002F21000016
:10008000312100003D21000033210000A157000074
:1000900087580000372100003D21000099B9001069
:1000A000372100005D3C0000633C00003D21000062
:1000B0003D210000D7530000214B0000693C0000A7
:1000C00049510000372100003D2100003D21000082
:1000D0000000000000000000000000000000000020
:1000E0000000000000000000000000000000000010
:1000F0000000000000000000000000000000000000
:1001000000000000000000000000000000000000EF
:1001100000000000000000000000000000000000DF
:1001200000000000000000000000000000000000CF
:1001300000000000000000000000000000000000BF
:1001400000000000000000000000000000000000AF
:1001500000F003F800F020F8FEE70D480168890878
:100160008900002001C101C101C101C17047000027
:1001700084E20010FEE7FEE7FEE7FEE7FEE7FEE7AB
:10018000FEE7FEE7FEE703480047FEE7FEE7000064
:10019000202100003D21000000F002F800F068F886
:1001A0000AA090E8000C82448344AAF10107DA45D2
:1001B00001D100F05DF8AFF2090EBAE80F0013F0BC
:1001C000010F18BFFB1A43F001031847F01E01008E
:1001D000401F01000A444FF0000C10F8013B13F0DF
:1001E000070408BF10F8014B1D1108BF10F8015B90
:1001F000641E05D010F8016B641E01F8016BF9D183
:1002000013F0080F1EBF10F8014BAD1C0C1B09D1D9
:100210006D1E58BF01F801CBFAD505E014F8016B4B
:1002200001F8016B6D1EF9D59142D6D370470000DD
:10023000103A24BF78C878C1FAD8520724BF30C812
:1002400030C144BF04680C607047000000230024E4
:1002500000250026103A28BF78C1FBD8520728BFD6
:1002600030C148BF0B6070471FB51FBD10B510BD32
:10027000DFF80CD0FFF7F8FF04F055FD11F080F91E
:100280000000021003B4FFF7F1FF03BC11F080F986
:1002900008B5002103200B460A46009110F026F80D
:1002A00008BD38B5F84D0024AC80EC802C810FF0EF
:1002B000F6FF6861FF20A870F448234622460460D8
:1002C000446004720120E87003202146009410F07D
:1002D0000DF8012038BD38B5EB4D0228AC78224628
:1002E0000DD0052810D0A24208BF38BD002003461B
:1002F0000246214600900FF0F9FFAC7038BD02298C
:1003000014BF01240224EEE7022914BF64246524EB
:10031000E9E738B513460A464FF0010C00240146C0
:10032000604600940FF0E2FF38BDD7490120087005
:100330007047D54800787047D3490020087070474F
:100340002DE9F04104460127002503F00700CE4EB9
:100350008846012804BF0020308146D0022844D1BD
:10036000308904280BD2002818BF306902D110F060
:10037000E5F8306110F8011B217030612EE006288D
:1003800008D210F0DDF83189C1F10501C900C8407B
:10039000207023E0082808D210F0D6F83189C1F186
:1003A0000701C900C840207018E00C2808D20FF0DF
:1003B00076FF3189C1F10B01C900C84020700DE002
:1003C0000E2808D20FF06DFF3189C1F10D01C9006F
:1003D000C840207002E0FF20207000273089401CB8
:1003E00080B230810E2828BF012588F80050384699
:1003F000BDE8F08130B403F007000024DFF888C2C4
:1004000001280BD06046BCF808308088022B0CD243
:10041000120242EA1020ACF8040010E0ACF80440EC
:10042000ACF80640ACF808400CE01844851EB5F561
:10043000806F04DADCF81450284400F8022C581CB1
:10044000ACF808000C7030BC00207047F0B40746D0
:10045000002003F007048C4D0646012C04BF2E81BA
:10046000EE6025D0DFF820C2022CBCF806C003D015
:1004700013F0070F0DD01BE02A890CEB0203B3F534
:10048000806F15D26869C05C3870501C28810120CB
:100490000EE0120242EA1C22EA80EB68012B05D131
:1004A000B2F5806F24BF40F2FF32EA805A1CEA6046
:1004B0000E70F0BC704738B503F0070000240D46FD
:1004C00001280AD1704821460B4604818480C480EB
:1004D00002200A4600940FF009FF2C70002038BD5E
:1004E00030B50C006AA183B009684FF00002029198
:1004F00008BF03250AD0217802AB5D5C002D18BF30
:10050000022D41D0012D7ED0032D0DD10F21017080
:100510000321417042808280C280028142818281B7
:10052000817B21F001018173002D1EBF012D03B0DD
:1005300030BD04F00DFC05281CBF03B030BD09F030
:1005400036FE042804BF03B030BD002D0CBFC02010
:10055000C1208DF8000060788DF8010060880123CB
:10056000000A8DF80200A0788DF80300A08806220A
:10057000000A8DF8040020798DF8050069460720EF
:100580000CF060FC03B030BD617800EB011202F8A2
:10059000101C617800EB011101F80F5C6278618832
:1005A00000EB021222F80E1C6278A18800EB021206
:1005B00022F80C1C6278A17900EB021222F80A1CC6
:1005C0006278217A00EB021222F8081C6278617AC4
:1005D00000EB021222F8061C6278217B00EB02126B
:1005E00022F8041CE1790529617800EB011010F86C
:1005F000021C0EBF41F0010121F0010100F8021CB4
:1006000092D132E0FFE7617800EB011303F8101C90
:100610006378012100EB031303F80F1C63786188F2
:1006200000EB031323F80E1C6378A18800EB03137F
:1006300023F80C1C617800EB011121F80A2C617879
:1006400000EB011121F8082C617800EB011121F871
:10065000062C617800EB011121F8042C617800EB85
:10066000011010F8021C21F0010100F8021C5BE7E8
:100670000549002048707047034840787047024998
:100680000120487070470000000401108807011025
:1006900003000201154A1154704700B583B0017878
:1006A0008DF8001041788DF8011081788DF80210D6
:1006B000C1788DF8031001798DF8041041798DF817
:1006C000051080798DF8060000208DF80700684637
:1006D00010F074FF03B000BD70470549002818BF33
:1006E0000120C87070470248C07870478807011021
:1006F000000401107047FE48D0F8C00000F001006F
:10070000704770B5FA4C05000AD001F04DFA38B9BF
:10071000D4F8C00010F0010F1CBF0020A06005D16C
:100720000120A060002D08BF002000D00120206221
:10073000002D18BF70BDD4F8D410D4F8D00011F03B
:10074000010F18BF11F0600F24D0D4F8B02222F4AA
:100750008032C4F8B02241F0610242F0FF22C4F8B6
:10076000D42040F0610242F0FF22C4F8D02021F0F2
:100770006102C4F8D42020F06102C4F8D020D4F87B
:10078000B02242F48032C4F8B022C4F8D410C4F8C5
:10079000D00070BD10F0010F18BF10F0600FD4D161
:1007A00070BDD348006A002818BF01207047C00000
:1007B00000F1804000F5A04041637047C00000F1A7
:1007C000804000F5A040006B00F48070704710215D
:1007D000C00000F1804000F5A04041637047C4496B
:1007E000D1F8402160F30D22C1F840217047C04884
:1007F000D0F84001C0F3052070470207520DC0F346
:10080000031002EB401000F1804000F5A0400029E9
:10081000D0F8401114BF41F0010121F00101C0F8EE
:10082000401170470107490DC0F3031001EB401060
:1008300000F1804000F5A040D0F8400100F0010038
:100840007047AB4900230B6202680A6042684A6045
:1008500082688A60C268CA60426A0A64826A4A64BC
:1008600002698A614269CA61426B0A66826B0A67E1
:10087000C26B4A67026C8A67426CC1F88020826C46
:10088000C1F88420C26CC1F88820026DC1F88C20A8
:10089000026EC1F89C20426EC1F8A020826EC1F8A1
:1008A000A420C26EC1F8A820C26FC1F8C020D0F841
:1008B0008020C1F8C420D0F88420C1F8C820D0F826
:1008C0008820C1F8CC20D0F88C20C1F8D020D0F8F6
:1008D0009C20C1F8E020D0F8A420C1F8F020D0F886
:1008E000A820C1F8F420D0F8AC20C1F8F820D0F846
:1008F000B020C1F8FC2021224A63CA63C2694A625F
:10090000C26A8A64026BCA64026FC1F8AC20D0F874
:100910009020C1F8D420D0F89420C1F8D820D0F885
:10092000A020C1F8E420426FC1F8B020826FC1F866
:10093000B420D0F8F821C1F88022D0F8FC21C1F809
:100940008422D0F80022C1F88822D0F80422C1F80D
:100950008C22D0F80822C1F89022D0F80C22C1F8DD
:100960009422D0F81022C1F89822D0F81422C1F8AD
:100970009C22D0F8182222F48032C1F8B022D0F89C
:10098000B420C1F80021D0F8B820C1F80421D0F873
:10099000BC20C1F80821D0F8C020C1F80C21D0F843
:1009A000C420C1F81021D0F8C820C1F81421D0F813
:1009B000CC20C1F81821D0F8D020C1F81C21D0F8E3
:1009C000D420C1F82021D0F8D820C1F82421D0F8B3
:1009D000DC20C1F83021D0F8E020C1F84021D0F867
:1009E000E420C1F84421D0F8E820C1F84821D0F82B
:1009F000F020C1F85021D0F8F420C1F85421D0F8EB
:100A0000F820C1F85821D0F8FC20C1F85C21D0F8BA
:100A1000EC20C1F84C21D0F82021C1F88021D0F879
:100A20002421C1F88421D0F82821C1F88821D0F8E8
:100A30002C21C1F88C21D0F83021C1F89021D0F8B8
:100A40003421C1F89421D0F83821C1F89821D0F888
:100A50003C21C1F89C21D0F84021C1F8A021D0F858
:100A60004421C1F8A421D0F84821C1F8B021D0F820
:100A70004C21C1F8C021D0F85021C1F8C421D0F8D0
:100A80005421C1F8C821D0F85C21C1F8D021D0F898
:100A90006021C1F8D421D0F86421C1F8D821D0F860
:100AA0006821C1F8DC21D0F86C21C1F8E021D0F830
:100AB0007021C1F8E421D0F87421C1F8E821D0F800
:100AC0007C21C1F8F021D0F88021C1F8F421D0F8C0
:100AD0008421C1F8F821D0F88821C1F8FC21D0F890
:100AE0005821C1F8CC21D0F87821C1F8EC2101E0DF
:100AF00000500040D0F88C21C1F80022D0F890219D
:100B0000C1F80422D0F89421C1F80822D0F8982125
:100B1000C1F80C22D0F89C21C1F81022D0F8A021F5
:100B2000C1F81422D0F8A421C1F81822D0F8A821C5
:100B3000C1F81C22D0F8AC21C1F82022D0F8B02195
:100B4000C1F82422D0F8B421C1F83022D0F8B8215D
:100B5000C1F84022D0F8BC21C1F84422D0F8C0210D
:100B6000C1F84822D0F8C821C1F85022D0F8CC21D1
:100B7000C1F85422D0F8D021C1F85822D0F8D4219D
:100B8000C1F85C22D0F8D821C1F86022D0F8DC216D
:100B9000C1F86422D0F8E021C1F86822D0F8E82139
:100BA000C1F87022D0F8EC21C1F87422D0F8F021FD
:100BB000C1F87822D0F8F421C1F87C22D0F8C42101
:100BC000C1F84C22D0F8E421C1F86C22FB4A12682B
:100BD00032F0FF0C05D1D1F890C062F3030CC1F8DC
:100BE00090C0F74A5370C36F13F0010F1CBF01236D
:100BF0005370D1F8C03023F00103C1F8C030D0F8F1
:100C00008C3013F0010F03D0537843F0020353707C
:100C1000D1F8D03023F00103C1F8D030D0F89000E3
:100C200010F0010F03D0507840F004005070D1F85C
:100C3000D40020F00100C1F8D4007047E0480078EB
:100C40007047DF4880787047DD49C8707047DC48DE
:100C5000C0787047DB490028D1F8C00014BF40F0CD
:100C6000010020F00100C1F8C0007047D54951F8DB
:100C7000C42F60F309020A607047D248D0F8C4005C
:100C8000C0F309007047CE4948607047CD48C0683E
:100C900070472DE9F047DFF82893054615F4003F2B
:100CA00099F8010099F8031000EA010418BF24F034
:100CB000010415F4802F18BF24F0020415F4002F4E
:100CC00018BF24F0040415F4801F18BF24F0080492
:100CD000DFF8F082D8F8B00220F48030C8F8B00213
:100CE00014F00F0F59D0D9F80460D8F8B8020027D3
:100CF00040F00100C8F8B802D8F8B80220F00100AE
:100D0000C8F8B802D8F8B00240F48030C8F8B00291
:100D10004FF0630A0DE002F0D4FD5046D8F8B81247
:100D200011F0010F01D0012703E0011EA0F1010025
:100D3000F4DC301EA6F1010601DD002FEBD067B315
:100D4000D8F8C00014F0010F0CBF20F0010040F0F3
:100D50000100C8F8C000D8F8D00014F0020F14BF8A
:100D600040F0010020F00100C8F8D000D8F8D4000D
:100D700014F0040F14BF40F0010020F00100C8F887
:100D8000D40089F80240012089F80000D8F8B002A8
:100D900040F48030C8F8B00233E0D8F8C00020F04A
:100DA0000100C8F8C000D8F8D00020F00100C8F851
:100DB000D000D8F8D40020F00100C8F8D4000020FA
:100DC00089F80200ACB1022089F80000D8F8B0021E
:100DD00040F48030C8F8B002D8F8B80240F0010002
:100DE000C8F8B802D8F8B80220F00100C8F8B80274
:100DF00007E0D8F8B01221F48031C8F8B01289F8B1
:100E00000000D8F8400115F0020F20F00D0018BFC7
:100E100040F0010015F0080F18BF40F0040015F075
:100E2000040F18BF40F00800C8F8400115F0010F8A
:100E300021D001F0A9F8044601F0A9F80146D8F83C
:100E40000C0000280EBF2046084621460028D8F88E
:100E5000C00114BF40F0010020F00100C8F8C0013B
:100E6000D8F8E001002914BF40F0010020F0010093
:100E7000C8F8E0010BE0D8F8C00120F00100C8F884
:100E8000C001D8F8E00120F00100C8F8E00115F039
:100E9000200F18BF002417D0204601F07FF800284B
:100EA0004FEA441000F1804000F5A040D0F8401215
:100EB00014BF41F0010121F00101C0F84012641C8F
:100EC000022CE9D3BDE8F087D8F8400220F00100F9
:100ED000C8F84002D8F8600220F00100C8F86002AB
:100EE000BDE8F0872DE9F0030246002011074C0D04
:100EF000C2F3031104EB411101F1804101F5A0415E
:100F0000D1F8401111F0010F11D142F01001C1F3DD
:100F1000031104EB411101F1804101F5A041D1F829
:100F2000401111F0010F04BFBDE8F0037047D60176
:100F300006F1804101F5A041D1F81C31C3F3080945
:100F4000204BDB69D1F8001103F008071FFA81F884
:100F5000002142EA0113C3F3031304EB431303F12B
:100F6000804303F5A043D3F8403113F0010F18D0AC
:100F700006EB411303F1804303F5A043D3F844C1CA
:100F8000CCF3080517F1000C1CBFD3F844C1CCF317
:100F9000023CD3F8403105FA0CFCC3F3054360442E
:100FA0001844491C0229D4D300FB08F0C9EB0911ED
:100FB000BDE8F00300EB410070470000E0FE0300D5
:100FC000180401100050004010B50120FFF78AFFFF
:100FD00004460220FFF786FF044400F0E0FB2044B3
:100FE0004FF47A71484347F23051B0FBF1F010BD35
:100FF0002DE9F041FE4E0546306810F01F0408BF91
:1010000001240120FFF76EFF07460220FFF76AFF69
:10101000074400F0C4FB3918F64F002D18BF002913
:101020004DD0D6F8C000002210F0010F34D0782047
:10103000B0EB151F08D9D6F8CC0020F00F0040F017
:101040000100C6F8CC002CE0D6F8C400EA4BC0F38F
:1010500009006043A0EB001003EB4003E748A0FB4E
:1010600005C04FEA502CB3FBF1F0102828BF0F2029
:10107000844598BF6046002808BF012005D001289C
:1010800084BF00FB1132B2FBF0F2D6F8CC3060F333
:101090000303C6F8CC3004E0B7FBF5F0884288BF04
:1010A000421AC4EB04104000B2FBF0F0B0F5005F50
:1010B00028BF41F6FF70726860F30C0272607068BE
:1010C000C0F30C006043C0EB001001EB4000B7FB25
:1010D000F0F0BDE8F081C648D0F8C01011F0010F63
:1010E00007D0D0F8CC0000F00F00C0EB001080015A
:1010F000704770B50168406801F01F05C0F30C0629
:101100000120FFF7EFFE04460220FFF7EBFE044448
:1011100000F045FB06FB05F1C1EB011104EB4101B9
:101120000844B449B1FBF0F070BDB148D0F8CC0030
:1011300000F00F007047AE494A684B68C2F30C02DA
:1011400060F30C034B6010467047A9484068C0F339
:101150000C007047C00100F1804000F5A040D0F8BD
:1011600000014EF6602180B2B1FBF0F0401C400857
:10117000704730B44EF6602331B1B3FBF1F1491C36
:101180004A08B2F5804F01D343F6FF72B3FBF2F188
:10119000491C4D08C101530801F1804101F5A041EE
:1011A000002807BF981FA3F10C0CD1F8040180B2EE
:1011B00018BFA2F1060C2CF0010CD1F8004162F32B
:1011C0000F04C1F80041D1F8002163F31F42C1F8B8
:1011D0000021D1F8042160F30F02C1F80421D1F8F5
:1011E00010016CF30F00C1F81001284630BC7047A5
:1011F000C00100F1804000F5A040D0F80001000CD3
:101200007047C20102F1804202F5A042D2F80031DB
:1012100061F31F43C2F80031002818BF70478A1FCE
:10122000901F20F001017248D0F8043162F30F03DF
:10123000C0F80431D0F8102161F30F02C0F810217A
:1012400070470107490DC0F3031001EB401000F196
:10125000804000F5A040D0F84401C0F3080070477A
:101260000207520DC0F30310654B02EB401000F172
:10127000804000F5A0409B58D0F84421CB1A61F380
:101280000802C0F84421D0F844119B1E63F31841B2
:10129000C0F8441170475649C9695A4A11F0100FF5
:1012A0004FEA00714FEA5151C0F3031001EB4010B7
:1012B00000F1804000F5A0405258D0F84401D2B26D
:1012C000C0F3080008BF0022801A0004000C08BF09
:1012D000012070470309DB0103EB810101F140515B
:1012E00001F5C0410007C00E0B6802FA00F0184378
:1012F000086070470209D20102EB810101F14051FF
:1013000001F5C04100070968C00E21FA00F000F0A5
:10131000030070470207520DC0F3031002EB4010A8
:1013200000F1804000F5A040C0F84C117047010763
:10133000490DC0F3031001EB401000F1804000F5AF
:10134000A040D0F84C017047294A0021D26912F020
:10135000080F0DD00107490DC0F3031001EB401039
:1013600000F1804000F5A040D0F84401C0F3023104
:10137000084670471E4AD36943F00803D361020749
:10138000520DC0F3031002EB401000F1804000F555
:10139000A040D0F8442161F30E32C0F844217047D8
:1013A000134A0021D26912F0080F0DD00107490D30
:1013B000C0F3031001EB401000F1804000F5A040A5
:1013C000D0F84801C0F30241084670470207520DA9
:1013D000C0F3031002EB401000F1804000F5A04084
:1013E000D0F8482161F31242C0F84821704700004C
:1013F0000050004000389C1C1B81070089888888A9
:101400001451004020510040042988BF704710B497
:101410000023FD4CE26912F0080F4FEA00724FEA18
:101420005252C0F3031002EB401000EB04021CBF49
:10143000D2F84401C0F302330020D4F81CC01CF0E1
:10144000080F1CBFD2F84801C0F30240C91A084473
:10145000042803DD081A011D042003E00028BCBF96
:10146000014400201944E36943F00803E361D2F822
:10147000443161F30E33C2F84431D2F8481160F3BD
:101480001241C2F8481110BC7047DF490028886932
:1014900014BF40F0080020F0080088617047DA4867
:1014A0008069C0F3C00070470207520DC0F30310FB
:1014B00002EB401000F1804000F5A040D0F8482138
:1014C00061F30F02C0F8482170470107490DC0F3CE
:1014D000031001EB401000F1804000F5A040D0F86F
:1014E000480180B27047C84AD2F8CC10022903D113
:1014F00010F0010F18BF7047D2F8400110F0010F33
:1015000008BF7047D2F84801D2F844110304C1F370
:1015100002311B0C14BF002970474FF6FF71484081
:10152000C2F848017047B84A0021D26912F0080F8A
:101530000DD00107490DC0F3031001EB401000F17D
:10154000804000F5A040D0F84801C0F300510846A3
:1015500070470120704710B4022ADDF804C026BF8E
:10156000921E52080022022B26BF9B1E5B080023FE
:10157000A64CA4FB0C4C4FEA1C144FEA007C4FEA2B
:101580005C5CC0F303100CEB401000F1804000F5F0
:10159000A040D0F854C161F31B6C62F3134C63F3A9
:1015A0000B2C64F3070CC0F854C110BC704770B426
:1015B0000407640DC0F3031004EB401000F18040F9
:1015C00000F5A040DDF80CC0D0F854010029C0F3AC
:1015D0000366C0F30345C0F30324C0B218BF0E6016
:1015E00012B16900891C116013B16100891C196076
:1015F000BCF1000F04BF70BC704700EB800080009E
:10160000CCF8000070BC704770B491B000224FF469
:1016100080456C10EC4601E0082A05D2531C03EB10
:101620008303B5FBF3F304E0D31F03EB8303B4FBA5
:10163000F3F35B1A48BF5B424CF82230521C102A6D
:10164000EAD30026009B01215CF821209A42BCBF0E
:1016500013460E46491C1029F6D30107490DC0F365
:10166000031001EB401000F1804101F5A041D1F8D9
:101670005801D1F8582100F00F0066F30302C1F8B9
:101680005821082807D2401C00EB8000B5FBF0F081
:1016900011B070BC7047C01F00EB8000B4FBF0F0CD
:1016A00011B070BC70470107490DC0F3031001EB86
:1016B000401000F1804000F5A040D0F8580100F043
:1016C0000F00082834BF401CC01F00EB800034BF4F
:1016D0004FF480414FF40051B1FBF0F0704710F02F
:1016E0000F0F08BF70470007400D00F1804000F564
:1016F000A0400029D0F824110CBF21F4803141F41E
:101700008031C0F824117047002110F00F0F0BD06A
:101710000007400D00F1804000F5A040D0F8240102
:1017200010F4803F18BF012108467047364AD2F8AE
:10173000AC0011F0010FD2F8AC10C0F3C00014BF20
:1017400041F0080121F00801C2F8AC1070472E4AA0
:101750005067916770472C490028D1F8AC0014BF3E
:1017600040F0020020F00200C1F8AC0070472649AA
:101770000028D1F8AC0014BF40F0010020F00100B7
:10178000C1F8AC0070472048D0F8DC0070471E4913
:10179000C1F8E00070471C48D0F89800704770B45A
:1017A000194E0020D6F8401111F0010F04BF70BC93
:1017B000704711F0040FD6F81C3101F00805D6F877
:1017C00000C1C3F308031FFA8CF4D6F844C1CCF36C
:1017D000080C18BFC1F30740F269C1F3052112F0EC
:1017E00008021CBFD6F84421C2F30232002D18BFF4
:1017F000491C0CFA02F201FB0200604370BCC3EB0F
:10180000031100EB4100704700500040CDCCCCCC20
:10181000FEF7C7BF10B5FEF7C4FF012818BF10BD03
:101820000020FEF76EFF21210020FEF7C0FF2121DE
:10183000BDE810400120FEF7BABF10B5FEF75AFF11
:10184000FEF7AFFF01280AD10020FEF75AFF212141
:101850000020FEF7ACFF21210120FEF7A8FF0121A7
:10186000052001F06CFB0121052001F068FBFC491B
:101870000020087110BD10B54FF4066001F0B5FBF3
:10188000BDE810404FF4066001F0A0BBF44A0146E9
:10189000107B002818BF0120002918BF01211173F7
:1018A0007047EF4A516A506208467047EC49002081
:1018B000C872887048707047E9490020C872887003
:1018C000487070470007C00EE64A801E02EBC01049
:1018D0004FF480720FF077BE70B50646FEF787FFB3
:1018E000E14D0446C6B1A201314628460FF06BFE19
:1018F00005EB84100021016041608160C1600161DD
:1019000041618161C161016241628162C1620163C1
:1019100041638163C16370BD800100F140012846CD
:10192000BDE870400FF054BE10B5CD4CE061FFF73C
:10193000B0F9FFF783F9A1696FF30F01A161A26903
:10194000C1B242EA0121A161022818BF10BDA069FD
:1019500040F00100A06110BDC4488168C44A114331
:1019600081600168521C1143016000F0D4BD2DE973
:10197000F047BE4A0D4606469368BD48184390603E
:101980001068BC490843106000F0C5FD0024002D1C
:101990006FD00020FEF7B5FE286820B1FEF751FF9A
:1019A0000020FEF7AEFE3046FFF7BEFF0020FEF738
:1019B00039FF002852D0D5F80480FEF718FFDFF871
:1019C000A89201260746B8F1000F1ED0BA01414681
:1019D00048460FF0F8FD09EB87100460446084600E
:1019E000C460046144618461C461046244628462CD
:1019F000C462046344638463C4639F48E96859B163
:101A00004FF480720FF0DFFD21E0800100F1400112
:101A100048460FF0DDFDF0E7984F4FF480710FF06E
:101A2000D7FD0020395600290EDB0A09D20102EB4E
:101A3000800202F1405202F5C0420907C90E136844
:101A400006FA01F119431160401C2028EAD38C48A2
:101A5000696949B14FF480720FF0B5FD0120FEF7BE
:101A6000E1FE804E50B905E04FF480710FF0B0FDFB
:101A7000F4E719E01120FEF7D5FE30B1A96821B1D5
:101A800030464FF480720FF09EFD0220FEF7CAFE32
:101A900018B91220FEF7C6FE30B1296921B1794884
:101AA0004FF480720FF08FFD6D48C47284704470E3
:101AB0004462017B002101734FF4066001F095FA46
:101AC000BDE8F0474FF4066001F080BA10B5002081
:101AD000FEF717FE00F00CFD6148C078002808BF33
:101AE00010BD6248016821F0030141F00D7141F021
:101AF00080510160816821F0020141F00D7141F0D7
:101B00008051816010BD4FF4066001F064BA10B5D9
:101B10004FF4066001F05FFAFEF743FE01280AD198
:101B20000020FEF7EEFD21210020FEF740FE2121DE
:101B30000120FEF73CFE5448D0F8B01221F4803169
:101B4000C0F8B0120020FEF7DCFD00F0D1FC4448E4
:101B5000C078002808BF10BD4448016821F0030187
:101B600041F00D7141F080510160816821F0020166
:101B700041F00D7141F08051816010BD10B501F050
:101B80002FFA10F0600018BF012010BD3448C06962
:101B9000704733488069704772B631498A6922EAD2
:101BA0000000886162B670472D480078002818BF91
:101BB0000120704770B5FEF7F4FD002818BF70BD16
:101BC0000024274DEC72AC706C7021212046FEF78A
:101BD000EEFD21210120FEF7EAFD2C70BDE87040EA
:101BE0000120FEF78EBD70B50446FEF7DAFD002831
:101BF00018BF70BD00211A4DE972A97069702121CA
:101C00000020FEF7D4FD21210120FEF7D0FD022C9B
:101C10003CBF0120FEF7DBFD012028702C62BDE8EF
:101C20007040FEF76EBD10B5FEF7BBFD002818BF73
:101C300010BD00200A4CE072A07060702121FEF7F8
:101C4000B6FD21210120FEF7B2FD0120FEF7BFFD08
:101C5000012020702062BDE81040FEF752BD000058
:101C60002004011040480030004000300080004057
:101C7000020034120300341200600030910701109A
:101C80000080003040490030005000400020FEF746
:101C900038BDFF490020887048700120FEF731BD33
:101CA000FB4988627047FA48806A7047002000F05C
:101CB00068BB012000F065BB10B5FFF764FD04466A
:101CC000FFF765FDF348044208BF10BDF048816985
:101CD00041F0040181610E2101EAD43104F00102D6
:101CE0000A43816962F31F418161EB48016841F059
:101CF0002001016010BD002818BF0120E449C87010
:101D00007047E6487047E6487047E148C06A704748
:101D1000DF484179C279914214BF006B406B704734
:101D2000DB48406B70472DE9F00FDC4E4FF0000CA4
:101D300088B006F14007E1464FF0FF3806F80C8006
:101D400007F80C900CF1010CBCF1200FF6DB4FF002
:101D5000000C002807DD12F80C4006F80C400CF1CE
:101D6000010C6045F7DC002422464FF0010A0028F0
:101D70000EDD16F902C0BCF1000F06DBBCF1200F2E
:101D80003CBF0AFA0CFC4CEA0404521C8242F0DB11
:101D9000002294466D460AFA02FB1BEA040F1ABFA2
:101DA00005F802C00CF1010C05F80280521C202A33
:101DB000F1DB0022002810DD16F902C0BCF1000F93
:101DC00008DBBCF1200F3ABF15F80CC007F802C0C1
:101DD00007F80280521C8242EEDBAD4C0022002844
:101DE000C4F82C9008DD17F902C0944501D0E762D1
:101DF00002E0521C8242F6DBAA4F0020A7F1600CE1
:101E0000A7F120060CF8008006F8009007F8009073
:101E1000401C2028F6DB0020002905DD1A5C0CF8A8
:101E20000020401C8142F9DC0022104600290BDD15
:101E30001CF90030002B04DB202B3CBF0AFA03F313
:101E40001A43401C8842F3DB002003460AFA00FBD9
:101E50001BEA020F1ABF2B545B1C05F80080401CC4
:101E60002028F3DB002000290ADD1CF90030002BBC
:101E700003DB202B3CBFEB5C3B54401C8842F4DB73
:101E80000020C4F83490002907DD3B56834201D07E
:101E9000676302E0401C8842F7DB11F0010F18BFB6
:101EA0001F2009D00AFA00F3134203D10AFA00F006
:101EB000024301E0401EF5D5002003460AFA00F770
:101EC00017421ABF2B545B1C05F80080401C2028C9
:101ED000F4DB002000290ADD1CF90020002A03DBC6
:101EE000202A3CBFAA5C3254401C8842F4DB00200C
:101EF000C4F830900029DEBF08B0BDE8F00F70478D
:101F00003256824204D0266308B0BDE8F00F704715
:101F1000401C8842F4DB08B0BDE8F00F704762490E
:101F200000EB401001EB8010704700EBC0005F49F0
:101F300000EB400001EB80007047DFF854C1012B3B
:101F40008CF805008CF8061003D9401C20F0010025
:101F500011468CF807008CF8081000FB01F24FF6D0
:101F6000FF7101EA4202ACF8122001EA4000ACF82D
:101F7000140070474648007A70474548C07970475A
:101F8000434A5072917270474148807A7047404886
:101F9000407A7047464A1070517070474449085C57
:101FA00070472DE9F047DFF8E890044699F80C00F7
:101FB000002804BF99F801000FF00FFB99F80B00FF
:101FC000002808BFBDE8F0874FF00008D9F81C00D2
:101FD00047464646454610F0020F1CBFDFF8C88052
:101FE00010F0040F05D0B9F812102F4A21F00101AA
:101FF0008F1810F0010F18BF2C4E10F0200F18BFD3
:102000002C4DD9F828002060FEF71BFE10F0010FC0
:1020100006D0FFF78AF8022828BF99F8020000D2FC
:102020000020E760C4E90108C4E904650120BDE8B7
:10203000F08717490020C872704710B50446FEF7B4
:10204000D6FB82012046BDE810401B490FF0BBBA09
:102050002DE9F041FEF7CBFB04460020FFF767F9BE
:102060000022002C84BF012541F6F07635D90021ED
:102070004FEA821C05FA01F3034228D04B080CEB0F
:10208000830303F1405303F58043CF071B6815E03A
:1020900020040110010007005C04011091070110E9
:1020A000B10701101108011064980110A4A00110DB
:1020B0002D0401107CA1011000400030FF0EFB40F8
:1020C000C3F30C03B34202D90020BDE8F081491CE0
:1020D0002029CFD3521CA242C9D30120BDE8F081F0
:1020E0000B460007C00EC549801E01EBC0114FF41E
:1020F000807218460FF067BA2DE9F05F00F00F0606
:1021000070000025A0F1020B012741F6F07846EAA5
:1021100005194846FEF786FB002835D04846FFF7EC
:1021200013F907FA00F4022C88BF02244846FFF78F
:10213000FEF80022002C84BF0BEB05014FEAC11A08
:1021400022D900210AEB821907FA01F3034215D0C4
:102150004B0809EB830303F1405303F580434FEA37
:10216000C17CD3F840384FEADC6C23FA0CF3C3F39C
:102170000C03434502D90020BDE8F09F491C2029EB
:10218000E2D3521CA242DCD36D1C022DBFD301202E
:10219000BDE8F09F2DE9F05F0026994C4FF6FF75E2
:1021A00000280F4644D000F00F01C0F303100129AE
:1021B0000EBF00210229BDE8F09F022828BFBDE81C
:1021C000F09F01EB0009FEF7ECFA5FEA00081CBF84
:1021D0000020FEF796FA00204FEAC919002209EB09
:1021E0008011530801EB830303F1405CD307DB0E3E
:1021F0000CF5804C05FA03FBDCF840A807FA03F362
:102200002AEA0B0A4AEA0303521CCCF84038202A77
:10221000E7D3401C0228E1D3B8F1000F08BFBDE8A6
:10222000F09FA6706670BDE8F05F0120FEF769BA06
:10223000FEF7B7FA5FEA00081CBF0020FEF761FA5C
:10224000002000228101530801EB83034FEAC27C86
:1022500003F140534FEADC6C03F5804305FA0CFAB6
:10226000D3F8009007FA0CFC29EA0A0949EA0C0C99
:10227000521CC3F800C0202AE5D3401C2128E0D31B
:10228000B8F1000FCDD1BDE8F09F10B5FFF703F80E
:102290005B49088210BD5A4AC1B200F4F853128A51
:1022A000914288BF11464FF0640C01FB0CF1B1FB69
:1022B000F2F11A0A02FB0C1110F4005F12BF08B20F
:1022C000484200B2704710B54FF480714D4C4E48F3
:1022D0000FF07EF9002001232156002910DB0A09A6
:1022E000D20102EB800202F1405202F5C04209071E
:1022F000C90ED2F800C003FA01F14CEA01011160E5
:10230000401C2028E8D310BD10B53E4C4FF480711E
:102310003D480FF05DF9002001232156002910DB14
:102320000A09D20102EB800202F1405202F5C042DA
:102330000907C90ED2F800C003FA01F14CEA010105
:102340001160401C2028E8D3BDE810404FF4246100
:102350002E480FF03DB92A4810B5808B00F48170EB
:10236000FFF7E2FA4FF4807127480FF031F94FF48C
:10237000046126480FF02CF9BDE810400020FEF75C
:10238000DABE70B51E4C0546A06A401CA0622078DB
:1023900050B1206A10B1206A401E2062206A0028D5
:1023A00004BF0020FEF7ADF920212846FEF7FFF913
:1023B000616A00291CBF28468847FEF73FFC0228B7
:1023C00015D11348D0F8B81211F0010F0FD0D0F882
:1023D000B81241F00101C0F8B812D0F8B81221F0DB
:1023E0000101C0F8B812A06940F00200A0610948DC
:1023F000016841F02001016070BD000040480030DC
:1024000020040110910701100060003000400030EE
:10241000005000405C0401102DE9F0410027634D9D
:102420000126002808BF2E701FD001282F7018BF6A
:102430006F701AD0DFF87881D8F800005D49084342
:10244000C8F8000029785C4C002914BF4BF608300E
:102450005A48E06014BF5A484FF0BB70A06059481A
:10246000006830F0FF0206D101E06E70E2E7E2683A
:1024700060F30302E26051B1A06840F01800A06070
:10248000012000F071F8A06840F48050A0600120A5
:1024900000F06AF8687818B1E06840F03000E06059
:1024A000D4F8B00040F00100C4F8B000012000F002
:1024B0005BF8E6674FF4E0602061C4F88870287824
:1024C000002818BFC4F89460E06820F03000E06095
:1024D000A06820F48050A060D8F8000020F004002C
:1024E00040F00D7040F08050C8F80000BDE8F08169
:1024F0003148C16821F03001C160816821F4805108
:1025000081602B48016821F0040141F00D7141F018
:1025100080510160704726480268264911430160D6
:10252000224925480A783AB1826842F0180282604E
:10253000826842F480528260497819B1C16841F0E2
:102540003001C160D0F8B01041F00101C0F8B01006
:1025500070471D49C0B241EA00201749086470471E
:1025600015491A480864704782B040F24C42009006
:1025700013E000BF00BF00BF00BF00BF00BF00BF2F
:1025800000BF00BF00BF00BF00BF00BF00BF00BF53
:1025900000BF0198411E0191EBD20098411E0091AD
:1025A00028BF0192F5D202B0704700005804011014
:1025B00000800040040034120060004005F4010077
:1025C0002000BB00D0FE030013005FA000005FA04E
:1025D000414840498161891CC161491E41630268CB
:1025E00022F0030242F00D7242F080520260426912
:1025F00022F0010242F00D7242F080524261026903
:1026000011430161354981603549C1603549002078
:102610000860704710B501F04CF932480468002C8E
:1026200008BF30BFFAD00021016001F046F9204612
:1026300010BD10B501F03DF926482A4B2649421C31
:102640001C682CB10020186001F037F9204610BD3D
:1026500072B648638A6120BF88614A6362B6BFF37D
:102660006F8FBFF34F8FEBE71B48016821F0030129
:1026700041F00D7141F0805101601B498160016999
:102680001A4A1143016130BF704772B611491248AE
:102690004163C91CC161891E816162B670470E48E1
:1026A0000168134A1143016070470B48016821F02B
:1026B000030141F00D7141F080510160704772B625
:1026C000044905488161891CC161491E416362B6A4
:1026D0007047000000003412008000403C003412BB
:1026E000280034125C040110080034120100341276
:1026F000030034127047002818BF01204FF4E02176
:10270000486070470022B2EBD10F26D20368B3F1C4
:10271000FF3F04BF4368B3F1FF3F17D18368B3F1B4
:10272000FF3F04BFC368B3F1FF3F0FD10369B3F1AB
:10273000FF3F04BF4369B3F1FF3F07D18369B3F1A2
:10274000FF3F04BFC369B3F1FF3F01D000207047D2
:102750002030521CB2EBD10FD8D30120704710B4F7
:102760000023B3EBD20F30D2D0F800C00C68A445E0
:1027700022D1D0F804C04C68A4451DD1D0F808C0BF
:102780008C68A44518D1D0F80CC0CC68A44513D1EE
:10279000D0F810C00C69A4450ED1D0F814C04C6913
:1027A000A44509D1D0F818C08C69A44504D1D0F84B
:1027B0001CC0CC69A44502D010BC0020704720305A
:1027C00020315B1CB3EBD20FCED310BC012070477D
:1027D0002DE9F041054601F074F8002021264FF460
:1027E000825784464FF4E0221660C5F800C0116895
:1027F00041F004011160116811F0040FFBD1176062
:1028000040232C460021D4F80080B8F1FF3F04BFDC
:10281000D4F80480B8F1FF3F1DD1D4F80880B8F196
:10282000FF3F04BFD4F80C80B8F1FF3F13D1D4F8B8
:102830001080B8F1FF3F04BFD4F81480B8F1FF3F17
:1028400009D1D4F81880B8F1FF3F04BFD4F81C8038
:10285000B8F1FF3F08D0C2F800C0401CC0B2082841
:10286000C2D30220BDE8F081491C2034B1EBD30F64
:10287000C9D3C2F800C00120BDE8F0812DE9F041C4
:10288000054601F01EF80020092684464FF4E02397
:102890001E60C5F800C0196841F00401196019688C
:1028A00011F0040FFBD12C464FF480620021276801
:1028B000B7F1FF3F04BF6768B7F1FF3F17D1A768C3
:1028C000B7F1FF3F04BFE768B7F1FF3F0FD12769BA
:1028D000B7F1FF3F04BF6769B7F1FF3F07D1A769B1
:1028E000B7F1FF3F04BFE769B7F1FF3F08D0C3F876
:1028F00000C0401CC0B20328CAD30220BDE8F0814A
:10290000491C2034B1EBD20FD1D3C3F800C0012051
:10291000BDE8F0812DE9F05F0F46804604264FF0B8
:10292000020A4FF0000B4FF4E02900F0CAFF4446C2
:102930003846C9F800A00F21B0E82C10A4E82C10EC
:10294000491EF9D2D9F8000040F00400C9F800008F
:10295000D9F8000010F0040F06D000BF00BFD9F86E
:10296000000010F0040FF8D1C9F800B04546384611
:102970000F21D5E90023D5E902C4D0F800E096453F
:1029800004BF42689A4205D18268624504BFC268AA
:10299000A24208D0761E03D34046FFF719FFC4E7D2
:1029A0000220BDE8F09F10301035491EE1D2012011
:1029B000BDE8F09F70B50D46044600F082FF4FF46D
:1029C0008072214628460EF0FEFD012070BD2DE9E3
:1029D000F041C0B014460E46054610F0FF0F23D05C
:1029E00025F0FF086F4600F06CFF4FF480724146FF
:1029F00038460EF0E8FDE8B2C0F58077A74288BF00
:102A0000274668443A4631460EF0ECFD4046FFF753
:102A1000DFFE022843D069464046FFF77BFF0228CD
:102A200041D03D443E44E41BB4F5807F19D34FF4BC
:102A30008072314668460EF0D5FD2846FFF7C8FE85
:102A400002282CD069462846FFF764FF02282AD0C6
:102A5000A4F5807405F5807506F58076B4F5807F61
:102A6000E5D2C4B16F4600F02CFF4FF480722946C6
:102A700038460EF0A8FD2246314668460EF0B2FDFB
:102A80002846FFF7A5FE022809D069462846FFF729
:102A900041FF022807D040B00120BDE8F08140B0DE
:102AA0000A20BDE8F08140B00B20BDE8F0810000B5
:102AB0002E490860086100F010B82C490860486190
:102AC00000F00BB829494867704728498867704764
:102AD000264801210166016570474FF04022116BC5
:102AE00010F0010F18BF21F4404110F0020F1CBF7D
:102AF00021F4405141F4805110F0040F18BF21F42B
:102B0000406110F0080F18BF41F4407110F0100F31
:102B100018BF41F0C00110F0200F18BF41F0300184
:102B200010F0400F18BF41F00C0110F0800F18BFDB
:102B300041F0030141F4BE0141F020411163D2F89C
:102B4000901010F4807F1CBF21F0030141F00201BE
:102B500010F4007F1CBF21F00C0040F0080141F48C
:102B6000BE0040F02040C2F89000704700100040C6
:102B70007047D0488268D0490A438260C2681143D6
:102B8000C1604169CD4A114341617047C9484169FB
:102B900021F0010141F00D7141F080514161C168A6
:102BA00021F0400141F00D7141F08051C160816818
:102BB00021F0400141F00D7141F08051816070477A
:102BC00010B5BC4CA168BC480143A160E168084352
:102BD000E0606069B94908436061B94843F63F71F4
:102BE000C160002181638164C0F8B01003210A2014
:102BF00000F0A5F90A2000F0C5F9606920F0010095
:102C000040F00D7040F080506061E06820F04000BE
:102C100040F00D7040F08050E060A06820F040006F
:102C200040F00D7040F08050A06010BDA44A1060CC
:102C30005160484390607047A14A1060516048431A
:102C400010F0010F18BF401C906070479C49C1F8FC
:102C5000B00070479A49002818BF01208864704767
:102C600097498863C86840F00200C8607047DFF881
:102C700050C2CCF82000CCF82410CCF82820CCF896
:102C80002C300120CCF83000DCF8340010F0010FBB
:102C900005D020BFDCF8340010F0010FF9D110F09E
:102CA000020018BF4FF0FF3070478548C16821F01F
:102CB0000201C16070478248C16841F00101C160F2
:102CC00070477F4B186259629A6201201864586CF1
:102CD00010F0010F04D020BF586C10F0010FFAD192
:102CE00010F0060018BF4FF0FF3070477448C168FD
:102CF00021F00101C16070477148C16841F00401D1
:102D0000C1607047027C017B02F03F0241EA024150
:102D10006B4A916501685162416891628168D16234
:102D200001211165516D11F0010F04D020BF516DCB
:102D300011F0010FFAD1D36D8382D36D1B0CC382C6
:102D4000136E0383136E1B0C4383536E8383526E87
:102D5000C2F30E42C28311F0020018BF4FF0FF30E1
:102D600070475748C16821F00401C160704754485A
:102D7000C16841F00801C1607047DFF844C1CCF878
:102D80007820CCF82000CCF82430CCF82810012092
:102D9000CCF87000DCF8740010F0010F05D020BFF3
:102DA000DCF8740010F0010FF9D110F0060018BF24
:102DB0004FF0FF3070474248C16821F00801C16000
:102DC000704701684FEA31423D49C1F89C20406894
:102DD000C1F8A000C86840F02000C86070470168D2
:102DE0004FEA31423649C1F89C208088C1F8A000E2
:102DF000C86840F02000C8607047314B18625A62C2
:102E000099620120C3F89400D3F8980010F0010FE4
:102E100005D020BFD3F8980010F0010FF9D110F0C1
:102E2000060018BF4FF0FF307047254A106251620C
:102E30000120C2F89000D2F8980010F0010F05D0E0
:102E400020BFD2F8980010F0010FF9D110F0060061
:102E500018BF4FF0FF3070471948C16821F02001BA
:102E6000C16070471648C16841F01001C1607047E9
:102E7000A3F1050C124BC3F888C018625A6299621C
:102E80000120C3F88000D3F8840010F0010F05D0B2
:102E900020BFD3F8840010F0010FF9D110F0060024
:102EA00018BF4FF0FF3070470548C16821F010018E
:102EB000C1607047008000404000341201003412AD
:102EC000009000401B4810B5022140F8501F01211E
:102ED00001611021416241F20601416100218161DD
:102EE0000421816390214163416B41F00101416301
:102EF0004FF4817101610161032000F043F800216A
:102F0000032000F01CF8002010BD10B5032000F0D5
:102F100045F808484FF480710166002101661021D0
:102F2000816702214165002010BD0349002008701F
:102F3000704700000030004060040110704700F04E
:102F40000303DA004FF0FF0C0CFA02F24FF0050C0D
:102F50000CEBC30301FA03F300F00C0101F1E021D3
:102F6000002807DAD1F8140D90431A401043C1F835
:102F7000140D7047D1F8000490431A401043C1F873
:102F80000004704700F01F01012202FA01F140091C
:102F9000800000F1E020C0F80011704700F01F0130
:102FA000012202FA01F14009800000F1E020C0F89E
:102FB0008011704700F01F01012202FA01F140095F
:102FC000800000F1E020C0F8801270474FF0E0214F
:102FD000C1F8000170474FF0E021C1F8800170474F
:102FE0004FF0E020D0F8000170474FF0E021C1F829
:102FF00080027047084800687047074A11681060EF
:1030000008467047044A126800F1100352F8230082
:1030100042F823107047000008ED00E002210C2068
:10302000FFF78DBFB8488268B8490A438260C2681A
:103030001143C1607047B448816821F4805141F068
:103040000D7141F080518160C16821F4805141F0DF
:103050000D7141F08051C1607047AD4881B0016F82
:1030600011F4007FFBD1816E11F0010F1CBFD0F86D
:103070008410009104D0D0F88410009A9142FAD0C4
:10308000016F11F4007F04BF4CF27101016642F23E
:103090004131816601B070479D4981B04FF40D52B6
:1030A0008A660A6FCA66012898BF012005D9401EAA
:1030B000B0F5803F28BF4FF6FF7082B24FF05C50F2
:1030C00040EA022048664FF01140C1F88000086FC6
:1030D00010F4007FFBD1886E10F0010F1CBFD1F8F7
:1030E0008400009004D0D1F88400009A9042FAD075
:1030F000086F10F4007F04BF4CF27100086642F2C2
:103100004130886601B07047814881B0016F11F489
:10311000007FFBD1816E11F0010F1CBFD0F884102D
:10312000009104D0D0F88410009A9142FAD04FF464
:103130000D51816601B070477348806810F480506B
:1031400008BF70477248806E00F0010070477048F9
:10315000406EC0F30F2070476D48D0F88400704770
:1031600010B50C20FFF726FF0C20FFF70BFF684976
:103170000220486710BD664910B5032088670C20FF
:10318000FFF70CFFBDE810400C20FFF713BF614AAA
:1031900011681060084670475D4810B5016FC16640
:1031A0005C480068002818BF80475B48016841F40C
:1031B0008051016010BD574840687047524810B5B3
:1031C000826852490A438260C2681143C160504913
:1031D000032088670C20FFF7E1FE0C20FFF7EAFED2
:1031E00000F066F94D4B0420C3F888004FF6FF70DD
:1031F000C3F88C0072B66033FFF74EFF4FF40070D7
:10320000186062B610BDF8B572B64148016F11F48E
:10321000007FFBD1816E11F0010F1CBFD0F884102C
:10322000009104D0D0F88410009A9142FAD04FF463
:103230000D51816639494FF400320A6662B6D1F801
:103240000412314D002946D0324C4FF6FF73591A03
:10325000A160AA69D5F81CC002F00F020CF00F0C97
:103260006244121D01FA02F2A2F5EA41DFF8B0C091
:10327000313961452FD2D0F88400191AE160B1F5D7
:10328000803F28D2274B4FF0000CA1FB03070CFB1B
:10329000037301FB0C3163460EF0A9F9401C400892
:1032A0002061B0F57A7F38BF4FF47A701E4B996871
:1032B000002908BF98605A681A609968C3E901102C
:1032C0008A421BD9824205D9814201D9616002E05C
:1032D000606000E0626000F0F7F8A86820F48050B9
:1032E00040F00D7040F08050A860E86820F48050F5
:1032F00040F00D7040F08050E860F8BD8242E9D89F
:103300008142E5D8E2E7000000800040001034125E
:1033100000C00040640401105C04011000A00040E3
:103320002F6E160000879303340801100F48816840
:103330000F4A114381600F48016841F40471016034
:10334000001F016841F004010160016841F01001B3
:1033500001607047084908607047BFF34F8F084904
:1033600006480860BFF34F8FFEE700000080004072
:103370000400341214ED00E008ED00E00400FA054A
:103380000CED00E018488168184A11438160100371
:10339000416941F001014161016A21F00F021449C4
:1033A0000A430262134B8A1EC3F8C42001657047AA
:1033B0004FF04020006900F0700070474FF040204F
:1033C0000D4940F8301F0D4941600D4901660D4916
:1033D000416670474FF0402148680B4A904202BF57
:1033E000496C0029094870470080004004003412ED
:1033F00003005FA000600040C0845FA050995FA000
:103400000A005FA000005FA061A5650561B66505C3
:10341000022824BF00207047DE4B53F8202043F8D9
:1034200020101046704770B5DB4C206FD94D10F05E
:10343000010F05D00120E0662868002818BF8047EA
:10344000206F10F0020F08BF70BD0220E0666868B0
:10345000002808BF70BDBDE870400047CF4810B5D8
:103460008268CF490A438260C2681143C160CA4979
:1034700002220A6501230B660323CB664A65816835
:1034800021F0800141F00D7141F080518160C168EF
:1034900021F0800141F00D7141F08051C16009209F
:1034A000FFF770FD0221BDE810400920FFF747BD7E
:1034B000BA488268BA490A438260C2681143C1604F
:1034C000B549022008657047B34902204865B348F2
:1034D000816821F0800141F00D7141F080518160DF
:1034E000C16821F0800141F00D7141F08051C1604F
:1034F0007047AA488068C0F3C0107047A648016FA3
:1035000011F4007F14BF4FF440714FF480710166D5
:10351000704710B5A04CE06F10F0020F4FF00100A3
:1035200018BF0320606700F068F99C498A69C9697F
:1035300002F00F02D04001F00F01C8400521B0FB9E
:10354000F1F04FF405710009C4F880109549A1FB12
:1035500000104009C4F88400206F10F4007F14BFED
:103560004FF440704FF48070206610BD8A48016FA0
:1035700011F4807F14BF4FF440714FF40071016665
:103580007047854B30B4DA6F12F0010F14BF03227D
:1035900002225A6700EB4005C5EBC0104FF4967449
:1035A000C1EBC0004C4300EB80007F4904EB4010AE
:1035B000A1FB0010794900224FF0020C8C69C00871
:1035C000C96904F00F0401F00F012144C84005212E
:1035D000B0FBF1F0B0F5803F05D3511C4008CAB2F2
:1035E000B0F5803FF9D242EA0C2141F01001C3F856
:1035F0008810C3F88C00186F10F4807F14BF4FF44C
:1036000040704FF40070186630BC70476248016F1C
:1036100011F4003F14BF4FF440314FF48031016684
:1036200070475D48016F11F4803F14BF4FF4403183
:103630004FF40031016670475748006FC0F3002017
:1036400070475548006FC0F3402070475349896860
:10365000C1F3C011002904BF002070474E49002863
:103660000CBFD1F80002D1F8040270474B4B9A68A6
:10367000C2F3C012002A04BF00207047464A002847
:103680000CBFD2F88000D2F88800C0F30A200CBF2B
:10369000D2F88020D2F8882002F00F02D3F818C0A8
:1036A000DB690CF00F0C03F00F0363441A449140E4
:1036B000012202EB400048433C49A1FB00100009F5
:1036C00070473B4901200870704770B4334BC1EB21
:1036D000011149009A69D3F81CC002F00F020CF0E6
:1036E0000F0C6244121DD14008BF012104D0B1F576
:1036F000803F28BF4FF6FF719A68C2F3C012002ABC
:103700001CBF70BC7047D3F808C0254A4CEA020CB5
:10371000C3F808C0D3F80CC04CEA0202DA601E4AB3
:103720004FF0020CC2F850C04FF400341466042568
:10373000C2F88850C2F88C101E4DD566C2F874C00D
:103740001D4902283CBF134E46F82010002118489E
:1037500001704FF400711166017819B920BF01782A
:103760000029FBD014669567D566C2F854C09868E6
:1037700020F0800040F00D7040F080509860D868D4
:1037800020F0800040F00D7040F08050D86070BC98
:10379000704700007C04011000A000400080004041
:1037A000800034121F85EB51CDCCCCCC8988888821
:1037B0007804011002000202735600004FF0E0216D
:1037C0000020886108611F494860704710B54FF0BC
:1037D000E02460610020A0610221401EFFF7AFFBE2
:1037E0000720206110BD4FF0E021002008617047E4
:1037F00014480188491C018070471248806870474E
:103800002DE9F0410F4C002705462780A0684FF4B2
:103810007A71B0FBF1F04FF0E026401E7061B761A5
:103820000221C81EFFF78BFB072030612188A942C7
:10383000FCD33761BDE8F081034948430149886002
:10384000704700008404011040420F00704770B5BB
:1038500005464FF40D500406A0660320E066264896
:1038600060664CF2710020662448C4F8800042F281
:103870004630A06602210020FFF761FB0020FFF721
:1038800081FB002D08BF70BDA06E42F2413108439C
:10389000A06670BD012110B5880781674FF40D51F6
:1038A00081660020FFF77AFBBDE810400020FFF79B
:1038B00081BB012081074867704701208107886725
:1038C00070474CF271008107086670470C4A116816
:1038D0001060084670470A4808B5006818B180476C
:1038E000002818BF08BD4CF2710188070166016FFE
:1038F000C166006F009008BD07383937009C1C91E5
:103900009004011070B5FF4D00244FF4A0612C709D
:103910006C70EC70FC480DF05BFE4FF4A061FB484E
:103920000DF056FEFA48AC602C71C0F80043C0F8A8
:103930000443C0F80843C0F80C43C0F81043C0F873
:103940001443C0F81843C0F81C43C0F82043C0F823
:103950002443C0F82843C0F82C43C0F83043C0F8D3
:103960003443C0F83843C0F83C43C0F84043C0F883
:103970004443C0F84843C0F84C43C0F85043C0F833
:103980005443C0F85843C0F85C43C0F86043C0F8E3
:103990006443C0F86843C0F86C43C0F87043C0F893
:1039A0007443C0F87843C0F87C436C716821D948EF
:1039B0000DF00EFE6821D8480DF00AFEEC6070BDD7
:1039C000D049002048707047CE4840787047CD48B5
:1039D0000079002818BF01207047CA4840790028A4
:1039E00018BF01207047C748C078002818BF0120C1
:1039F0007047C448407800EB800101EBC000C54926
:103A000001EBC00070472DE9F041BE4D0446C149AD
:103A10006A78C24F02EB820000EBC200C04E01EB9D
:103A2000C0033A78307821461044420018460DF021
:103A3000D9FD6A78B84902EB820000EBC20001EBC5
:103A4000C0033A78307821461044420018460DF001
:103A5000C9FD01206871BDE8F081AA48C0687047BF
:103A6000A848A949407800EB800001EB002070478E
:103A70002DE9F041A34E07463078002814BFA9482D
:103A8000A948047814BFA948A948057804FB05F89B
:103A9000FFF76FF829462046FFF7C8F870789B4C6F
:103AA00000EB8000984904EB002201EB00203B462C
:103AB0000146FFF7DCF8FFF769F870784FEA480233
:103AC00000EB800004EB002039460DF08BFD012057
:103AD000F070BDE8F0812DE9F0478A4D04468A492F
:103AE0006878DFF8408200EB800001EB002C28783A
:103AF000DFF834928D4E8E4F2146002815BF98F87E
:103B0000002099F8002033783B7802FB03F04FEA5D
:103B1000400260460DF066FD68787C4900EB80004D
:103B200001EB002C28782146002815BF98F80020CA
:103B300099F8002033783B7802FB03F04FEA40020B
:103B400060460DF04FFD0120E870BDE8F0876D483C
:103B50008068704770B5774C0546014622787648F4
:103B600052000DF03FFD22782946520073480DF0B7
:103B700039FD64490120087170BD2DE9F04FADF2A7
:103B8000445DDFF880910120CDF8240599F8030009
:103B9000CDF8200599F80400CDF81C0599F805002A
:103BA000CDF81805FDF734FECDF83C05FDF7FCFF18
:103BB000CDF83805FDF7C9FACDF83405FDF741F821
:103BC0000446FDF727FEFCF796FDCDF830050020F2
:103BD000FDF740F8D9F8140024F001040428BCBF14
:103BE0000420C9F8140099F80200B9F81410000272
:103BF00040EA014040F0010200239121072009F032
:103C0000F1F814F0010F05D0FDF7D4FF0020CDF836
:103C1000240504E00020FDF78EFAFEF704F80026E4
:103C20003746B3464FF0010A05F097F901281DD039
:103C30000DF5A060FEF7B5F9002800F000820DF543
:103C4000A06005F0DFFF002089F80100D9F814001A
:103C5000C01E8642CABF874201250025DDF80C053B
:103C6000002836D0DDF81C0520B132E04FF0010B02
:103C700000F0CBB96846DDF80C150DF0BDFC8046B0
:103C80007DB12C4C4146207842002B480DF0AAFC17
:103C900020784146420029480DF0A4FC89F804A090
:103CA00017E0FEF766FF234C01212078FEF7BEFFE8
:103CB000224A4346A2F140010846FEF7D8FFFEF72C
:103CC00065FF2078414642001C480DF08BFC89F8C6
:103CD00004A0DDF80805002800F0EB80DDF82005E1
:103CE000002840F0E68099F80000DDF8084500283B
:103CF00062D1D9F80880B8F1000F44D009480078A3
:103D00001EE0000094040110C0A101104008011041
:103D100040140110C0A60110C0170110CC040110FE
:103D2000CD040110CA040110C7040110CB04011016
:103D3000C8040110CE0401104017011080170110B3
:103D4000CDF82C05FC480078CDF82805FEF711FFCA
:103D5000DDF82815DDF82C05FEF76EFF21464246FA
:103D60000846FEF7AEFFFEF711FFF4480078022880
:103D700004BF404605F019FDF0480078092804BF4B
:103D8000204605F012FDEE480078012814D9DFF82E
:103D9000AC8398F80000042804BF204605F005FD18
:103DA000214668460DF02DFC044698F800000528D1
:103DB00004BF204605F0F9FCADB399F8010099F86D
:103DC000002000EB8001DF48002A00EB01202146A3
:103DD0000CBFDD4ADD4A137814BFD74ADC4A12789B
:103DE00003FB02F24FEA42020DF0FCFB99F80100DE
:103DF00000EB8001D74800EB012399F80000214631
:103E0000002814BFD148D048007814BFCA4AD04A0D
:103E1000127800FB02F04FEA400218460DF0E2FB78
:103E200089F803A038E0FFE7CDF8284599F80000AD
:103E3000002814BFC548C44890F8008014BFBE488D
:103E4000C348047808FB04F0CDF82C05FEF791FE7A
:103E500021464046FEF7EAFE99F80100BD4C00EB12
:103E60008000B84904EB002201EB00200146DDF898
:103E70002835FEF7FCFEFEF789FEDDF82C05DDF89F
:103E80002815420099F8010000EB800004EB0020A7
:103E90000DF0A8FB89F803A0A8480078032808D1F2
:103EA00099F8010000EB8001A64800EB012005F025
:103EB0007CFCDDF8100500287DD0DDF81805002811
:103EC00079D199F80000DDF8104548BBD9F80C808D
:103ED000B8F1000F24D0A0480178A0480078084429
:103EE000401C4008019002200090FEF742FEDDE9F0
:103EF0000010FEF7A1FE214642460846FEF7E1FE0D
:103F0000FEF744FE96480078022804BF404605F0BC
:103F10005EFD93480078092804BF204605F057FD50
:103F200045B399F801008C4D00EB800101EBC00115
:103F30008C48DFF8288200EBC1032A7898F800004B
:103F400021461044420018460DF04CFB99F8010040
:103F50002A7800EB800101EBC001834898F800301B
:103F600000EBC1001A44214652000DF03BFB89F8DA
:103F700005A02EE07848A0460178784800780C1813
:103F8000FEF7F7FD601C40080221FEF74FFE99F88E
:103F90000100754D00EB800101EBC000714905EB9C
:103FA000C00201EBC00108464346FEF760FEFEF783
:103FB000EDFD620000E01BE099F8010000EB8001DC
:103FC00001EBC00005EBC00041460DF00BFB89F88A
:103FD00005A06348007803280AD199F8010000EB96
:103FE000800101EBC0015F4800EBC10005F0EFFC70
:103FF000FEF71FF8D9F81400761C7F1C8642A8BF74
:10400000874215DBD9F8100090B1FDF703FCDDF80D
:104010003405FDF790F8DDF83005FCF71BFEDDF800
:104020003C0588B1DDF8380560B1FDF7FCFD0BE01B
:10403000DDF82405002818BFFDF7F5FDF4E500F0D4
:10404000D4FEF1E5FDF7B6FDBBF1000F04BF04207F
:10405000C9F814000BD0DDF8200589F80300DDF85D
:104060001C0589F80400DDF8180589F80500B9F881
:1040700014104FEA0B2040EA01420023912107204F
:1040800008F0B0FE0DF2445D5846BDE8F08F10B563
:104090000024FDF77BFD354910F0020F0AD0CA78E5
:1040A000002A08BF012410F0040F03D00A79002A67
:1040B00008BF012410F0010F03D04879002808BF81
:1040C00001240020002C08BF10BD00200870BDE8AE
:1040D000104052E508B50F2100F095FF012804D1EA
:1040E000FFF7D5FF009001F0DBF82048C1780029E8
:1040F0001CBF4179002904D0007900281CBF012091
:1041000008BD002008BD08B50F2100F07CFF012884
:1041100004D1FFF7BCFF009001F0C2F81348C1784A
:1041200000291CBF4179002904D0007900281CBF58
:10413000012008BD002008BDCB0401104905011075
:10414000C9040110C0A10110C7040110CA04011064
:10415000C804011040080110CC040110CD04011066
:104160004E050110C0A60110C017011094040110E3
:104170007047FB490020C8700871487109F062BAA5
:1041800010B54FF4A061F7480DF022FABDE81040D9
:104190004FF4A061F4480DF01BBAF4487047F4489E
:1041A0000178F448007848434100F0480DF010BA17
:1041B00070B50646EE480478EE480578FEF7D9FC5F
:1041C00029462046FEF738FDE548E649407800EBF1
:1041D000800001EB00223146E448FEF772FDFEF755
:1041E000D5FCE5480078152818BF70BDDF48BDE84C
:1041F000704005F0DABA002818BF0120D849C8700D
:10420000704710B5D64C002804BFA06010BDDFF881
:104210006CC3DB490B78DB490A7801465A435200EC
:1042200060460DF0DFF9D548A06010BDD6490020EA
:10423000C1F80003C1F80403C1F80803C1F80C0376
:10424000C1F81003C1F81403C1F81803C1F81C0326
:10425000C1F82003C1F82403C1F82803C1F82C03D6
:10426000C1F83003C1F83403C1F83803C1F83C0386
:10427000C1F84003C1F84403C1F84803C1F84C0336
:10428000C1F85003C1F85403C1F85803C1F85C03E6
:10429000C1F86003C1F86403C1F86803C1F86C0396
:1042A000C1F87003C1F87403C1F87803C1F87C0346
:1042B0007047B6487047002818BF0120A849087108
:1042C000704710B56821B2480DF082F9BDE8104082
:1042D0006821B0480DF07CB9002818BF0120A04922
:1042E0004871704710B59E4C002804BFE06010BDB7
:1042F00068220146A8480DF075F9A748E06010BD96
:1043000070B5974C00210546E1702171617109F08B
:1043100099F9002D14BF012000202070BDE87040E5
:104320002BE42DE9F04F8BB04FF4A06193480DF0D2
:104330004FF9682198480DF04BF9FDF727FC04462A
:10434000FDF766FA0990FDF72FFC0890FCF7FDFEDB
:104350000790FDF75FFAFCF7CEF906900020FCF716
:1043600079FC0020FCF7E7FEFDF75DFC00252E46FA
:1043700004F0F3FD012853D06846FDF712FE002833
:104380005ED0684605F03EFC14F0020F1CD07C485D
:10439000DFF8E8B1DDF8089090F800807948DA4657
:1043A0000778FEF7E6FB0120FEF754FC394640464D
:1043B000FEF742FC524649465846FEF782FC002072
:1043C000FEF748FCFEF7E2FB14F0010F20D0734823
:1043D000DFF8C4B14FF0020801787148DA46DDF821
:1043E000109000780844401C4708FEF7C2FB0120EB
:1043F000FEF730FC41463846FEF71EFC5246494661
:104400005846FEF75EFC0020FEF724FCFEF7BEFBDC
:10441000FDF70FFE6D1C102D03D2FDF704FCA7E77E
:104420000126FDF7F7F90798FCF785FE0698FCF7DB
:1044300011FC099848B1089828B1FDF7F4FB04E095
:1044400000F0D3FC94E7FDF7B5FBCEBB444F14F06E
:10445000020F18D04A48494B01784A489C460078D8
:1044600001FB00F210200021002A0AD93CF911803A
:1044700008EB5008B8FBF0F523F81150491C8A42AC
:10448000F4D83E48B86014F0010F19D04348DFF863
:1044900008C101784248634600780A184FF01001BD
:1044A0004FF000000AD033F9105005EB5105B5FB71
:1044B000F1F42CF81040401C8242F4D83648F860E1
:1044C0000BB03046BDE8F08F01207047354870478B
:1044D00034480068704733490A68B2F1FF3F15D08D
:1044E000052804BFC87A704728DC012804BF087972
:1044F0007047022804BF087A7047032804BF487A2F
:104500007047042804BF887A704727E0052813D035
:1045100007DC012822D002281CBF032804280BD066
:104520001CE0142812BF15282D207047162804BF40
:1045300028207047172811D100207047142804BF85
:10454000087B7047152804BF487B7047162804BFB6
:10455000887B7047172804BFC87B7047FF207047CF
:1045600094040110C0A1011040080110400D011079
:10457000C7040110C80401104905011040120110C0
:10458000CA040110CB04011040140110401701109F
:10459000C0A60110C017011028180110CC0401108A
:1045A000CD04011000AE020030B5C1B000244FF4BC
:1045B000807168460DF00CF8FF22CD4D511C684605
:1045C0000DF024F8FF21224661F307022D23214636
:1045D00063F3070163F30F2128234BF6BB3063F32A
:1045E000174164F31F61CDE90002CDE90241049453
:1045F0002846FEF7EDF869462846FEF78BF941B0EC
:1046000030BD2DE9FF4FDFF8E882C1B08346D8F80E
:1046100000004E9F91468A464446B0F1FF3F08BFD6
:10462000FFF7C2FFD4E901106BF307018B466AF371
:104630000700449969F30F2061F317402568D4E916
:10464000036467F31F600746FF22511C68460CF0A5
:10465000DDFF0297CDE90364CDE9005B4046FEF73C
:10466000B7F869464046FEF755F9012818BF002003
:1046700045B0BDE8F08F2DE9F74FDFF8749283461F
:104680000020D9F80060C0B08A464C46B6F1FF3F22
:1046900004BF43B0BDE8F08FD4E902856768FF220C
:1046A000511C6846D9F810400CF0B0FF6BF30705B9
:1046B00042986AF30F2560F31745012060F31F65E8
:1046C000CDF80880CDE903544846CDE90067FEF7F0
:1046D0007FF869464846FEF71DF943B0BDE8F08F04
:1046E0002DE9F04F8248834E00250368C1B0744223
:1046F0002F461720FFF7EFFE84461420FFF7EBFE4E
:1047000040B2B3F1FF3F04D0BCF1000F03D12D281C
:1047100001D0FFF749FF1420FFF7DDFE40B2029001
:104720001520FFF7D8FE4FFA80F91620FFF7D3FEC9
:1047300040B201901620FFF7CEFE404240B20090FA
:10474000FDF724FADFF8B0A1834600208AF80300C1
:104750008AF804008AF8050008F074FF00208AF83F
:104760000000FFF70AFA1BF0010F04D00CF053FF12
:10477000012808BF01251BF0020F7DD05F489AF881
:104780000110604A90F800C05D4801EB810102EB26
:10479000012200784FF000080028C8BFACF1010AE0
:1047A0001EDD0021BAF1000F16DD01F1010B01FB46
:1047B00000830BFB008B32F8133032F81BB0A3EBF5
:1047C0000B031BB2002BB8BF5B421BB2BB42C8BF7E
:1047D0001F46491C5145E8DB08F101088045E0DB34
:1047E000B945B8BF45F002054FF00008C146BCF11D
:1047F000000FC8BFA0F1010A1BDD0021BAF1000FB4
:1048000013DD09FB001332F813B002EB43035B889E
:10481000ABEB03031BB2002BB8BF5B421BB243459B
:10482000C8BF9846491C5145EBDB09F10109E14538
:10483000E3DB02994145B8BF45F004054FF000099C
:10484000BCF1000F13DD002300280CDD09FB003153
:1048500032F91110B142C8BF0E46A142B8BF0C4692
:104860005B1C8342F2DB09F10109E145EBDB0198B6
:10487000B04204DB009800E003E0A04201DD45F017
:10488000080560421A4C08F0FF0B00F0FF08206892
:1048900007F0FF0A06F0FF09B0F1FF3F08BFFFF77E
:1048A00083FED4E901106BF307006AF30F2026683A
:1048B00069F31740D4E9037465F3070168F31F60D7
:1048C0000D468046FF22511C68460CF09FFECDF835
:1048D0000880CDE90374064CCDE900652046FDF75C
:1048E00077FF69462046FEF715F841B0BDE8F08F26
:1048F00000AE0200F1D8FFFF94040110C8040110BB
:10490000C7040110C0A10110F848C0787047F748EB
:1049100040797047F54920F07E4008617047F348C0
:1049200000697047F14880897047F048C089704736
:104930007047084318BF7047EC48006910F0807F4B
:104940001CBF0020107070472DE9FF5F8346E848C8
:104950000027DDF838A005780398109EB9463C463C
:1049600050452CD006FB050E0F983BF91EC006FBE8
:1049700005093BF91900BCEB000348BFA0EB0C0391
:1049800006FB05A83BF91840B4EB000C48BFA0EBB0
:10499000040C03EB0C0004B231F91EC031F919000C
:1049A000BCEB000348BFA0EB0C0331F918C0BCEB13
:1049B000000148BFA0EB0C0158180FFA80F9012A3A
:1049C0002DD04FF001080CF02BFECA49002C0A78BC
:1049D0002EDD0F9906FB05113BF911101431282922
:1049E00026D9039902EB0A0C11448C4520D9119B5E
:1049F000129D13442A448B421CBF8D1A15F1020FDD
:104A000030F9115000EB4106B6F90260A5EB06053E
:104A100008D01E353C2D08D94FF0000808E0A1450C
:104A20000CDD0AE00A35142DF6D8491C8C45E2D875
:104A3000A14503DDB8F1000F00D0012704B03846CE
:104A4000BDE8F09FAC4A0280428000218280C18094
:104A50000181534243818181C181018241828182EE
:104A6000C18202837047A1480078002818BF012046
:104A7000704710B54FF4A061A0480CF0A9FD4FF4A9
:104A8000A0619F480CF0A4FD98490020087010BD5B
:104A90002DE9FF4F85B09846DDE913A691460446FF
:104AA000DDF848B008F0DFFD0025904F002840F009
:104AB000CF8000F04DF9052800F0CA800698CDE9B6
:104AC00002060A2004908F481E260078009089482C
:104AD00000780190B88910B9787801281FD108F0C2
:104AE000FDFDE0B9BAF1010F19D0BBF1010F02D100
:104AF000F889C82813D8F889002804BFB889002885
:104B00000DD008F09CFD01280BD0DDE9002100202C
:104B1000521812D0029931F91010B14209DDFD711D
:104B20001BE0052004900398012814BF3C2646266C
:104B3000EBE7401C80B28242ECD8386910F4803F29
:104B40000BD0F879401CC0B2F8710499884204D99E
:104B5000012078714FF0FF34FD7108F070FD0128DD
:104B600076D1BBF1000F2BDCBAF1010F28D03869E8
:104B700010F4003F0AD0B879401CC0B2B8710A28BE
:104B800004D9012078714FF0FF34BD710A200190E3
:104B90005C48002690F800B0564890F800A01E200F
:104BA00000900CF042FD01460020AAF1010CBCF17E
:104BB000000F17DD31F91020C82A03DD3D7247E0F0
:104BC000BD71E3E701EB4003B3F90230002BB8BF3E
:104BD000002A03DAD21AB242C8BF16B2401C80B211
:104BE0006045E7DB31F91000C828E7DC0AEB0B0071
:104BF000431E534515DD31F91A00C828DEDC01EBF0
:104C00004A02B2F90220002AB8BF002803DA801A4B
:104C1000B042C8BF06B20AF101001FFA80FA53453C
:104C2000E9DC31F91A00C828C8DC386910F4002F13
:104C30000ED000988642C1DD387A401CC0B238726E
:104C40000199884204D9012078714FF0FF343D72F8
:104C5000B4F1FF3F28D0002C07BFF878012809B035
:104C6000BDE8F08FFD704FF4A06124480CF0B0FC5B
:104C70004FF4A06122480CF0ABFC3D7000F06EF8E0
:104C8000042841D0B9F1000F1CBF4846FEF723FFAE
:104C9000B8F1000F04BF09B0BDE8F08F404609B07D
:104CA000BDE8F04FFEF7AFBE787901281CBF09B010
:104CB000BDE8F08F4846FFF77BFA7D714FF4A061A5
:104CC0000E480CF085FC4FF4A0610D480CF080FC00
:104CD0003D70B9F1000F1CBF4846FEF7FCFEB8F16D
:104CE000000FDBD109B0BDE8F08F0000AC0401106B
:104CF000C7040110CD040110F1D8FFFF901D011071
:104D000090180110CC040110B9F1000F1CBF4846E7
:104D1000FEF7AEFEB8F1000FE4D009B04046BDE8A2
:104D2000F04F0CF087BC10B506F052F906F0FBF915
:104D3000002010BDFD4988707047FC48807870479E
:104D400004283CBFF949C8707047F848C0787047DC
:104D5000F64800787047F54840787047F348007887
:104D6000022805D005281CBF0020704705F01FBA97
:104D700008F048BCED490870704770B5EB4E04462A
:104D80000D463078A04212D002281AD0052814BF50
:104D9000002005F00CFA44EA05213278002341EAAC
:104DA000024141EA00626121072008F01BF875709A
:104DB000072C28BF70BDDFE804F016070B13160F91
:104DC000160008F01FFCE6E7284600F077FA0AE034
:104DD000284608F0B8FC06E0284605F0DDF902E0B8
:104DE000284608F0B7F8347070BDD1490020096832
:104DF000B1F8641011F4807F08BF7047FDF70ABC5A
:104E0000CB4900200968B1F8641011F4807F08BF15
:104E10007047FDF70EBCC64900200968B1F8641060
:104E200011F4007F08BF70470CF009BCC049002096
:104E30000968B1F8641011F4806F08BF70470CF076
:104E400003BCBA49087900281CBF401E087170478E
:104E500070B5B849D1F8CC00B44C10F0030F0AD0AB
:104E600040F4BE0040F02040C1F8C800207900287E
:104E700004BF01202071B0488068AD4D10F0020FD2
:104E8000296807D14FF04020406910F0010F01D090
:104E9000207940B1B1F86410002011F4807F18BF70
:104EA000FDF7C7FB07E0B1F86410002011F4806F34
:104EB00018BF0CF0C9FBA149084208BF70BD2968A2
:104EC000496E090C217170BD10B572B6FEF7E2FC97
:104ED000BDE81040FEF741BA10B5012802D0022803
:104EE00005D008E04FF42F30FDF772FC03E04FF0DF
:104EF00040219348086772B6FEF7CCFCBDE810402D
:104F0000FEF72BBA894900284A7918BF0120487159
:104F1000C0B2824208BF70470022002818BF012299
:104F200000230121022007F05DBF8048407900285E
:104F300018BF012070477D48807970472DE9F04106
:104F40007A4E00281CBF0020B07104D1B07900282F
:104F500018BFBDE8F0814FF040273D6B0120FDF701
:104F6000ACFD0420FDF7A9FD764C0520E066FEF7B8
:104F7000A8FC40F2CF70216F11F0010F04D0B0797E
:104F800040F00E00B07103E0011EA0F10100F2DC60
:104F9000B07978B1FEF795FC6B48216F11F0040FE2
:104FA00004D0B07940F00100B07103E0011EA0F11F
:104FB0000100F2DC45F4BE0040F020403863BDE85B
:104FC000F0815A488069704758484069704757488F
:104FD0004069002818BFC07A70475449C8617047BB
:104FE0005248C06970475149086270474F48006A8B
:104FF00070474F48026802F5C073118A508A02F563
:10500000A072FCF790BE2DE9F04FDFF8209197B029
:105010000E46C9F8180005F0FCFEC9F81400002877
:105020007ED090F800C089F807C0417889F8081050
:10503000837804460CF1010089F8093000F0FE0085
:1050400089F80A00E27889F80B20207989F80C00A9
:10505000607989F80D0009F10F004FF0000B80F81E
:1050600000B080F801B0207889F80E006046FCF7A7
:1050700064FF99F80D1099F80C00FCF781FF694660
:10508000204605F0EFFE608AD9F81C5000281CBFAE
:105090006843050B678BD9F82080002F08BF4FF4B9
:1050A00080574FF4805A002016F0040F18BF4FF4B9
:1050B000857016F0080F18BF40F0040016F0020FBC
:1050C0001CBF40F20121084316F0010F18BF40F445
:1050D0008460616A6FF30F0608406FF30F010843A5
:1050E0000643009810900498119008981290019827
:1050F000139007981590CDF850B010A93046FCF7E2
:1051000036FC16F0020F73D005F009FA5FEA000BC7
:1051100045D005F01BFA6843050B5946002000E016
:1051200030E0FCF726F8218A00290FE0C0040110C6
:10513000F8050110006000400080004008000300F6
:10514000AD2007B0001000403F0D03001CBF002041
:10515000FCF786F805F01AFA08FB00F0000B803027
:10516000010A0820012202FA00F30B4201D1401E7D
:10517000F9D5A0F10408A07B002818BFA0F1010B0D
:1051800017D112E04B480068B0F8640010F4807F3B
:1051900018BFFDF74EFA002017B0BDE8F08FB4F845
:1051A0000CB0BBF1000FB8D1BDE70020FCF7CCF884
:1051B0008346E07B002814BF401EFCF7F1F80BEBA0
:1051C0000801042905DDA8EB010101F1040804210F
:1051D00004E00029BCBFA8EB010800218044B8F11D
:1051E000040F06DDA8F10400C5404FF0040808E0F4
:1051F0000EE0B8F1000F04DAC8F1000085404FF06E
:1052000000080020FCF7B6F841460020FCF7DEF865
:1052100016F0010F23D0A18A00291CBF0120FBF743
:10522000A8FF268B3EB131460120FCF719F8314624
:105230001120FCF715F8A67D3EB1711E0120FCF788
:1052400099F8711E1120FCF795F8E67D3EB1711EAC
:105250000120FCF7BBF8711E1120FCF7B7F8E07ACB
:1052600000281CBF0001FBF7C3FE029805F033F9CC
:10527000039830B12B4699F8082099F807100CF0E4
:10528000E8F95246394628460CF0E8F90598FEF749
:10529000B8FF0998FFF726F817B00120BDE8F08F96
:1052A00010B5FCF734FC05F01EF9034900204861F5
:1052B000012010BDF8050110C0040110FB49087061
:1052C0007047FA4800787047F94810B4F94A016805
:1052D000914218D14168B1F5907F14D80022D0F8DE
:1052E00008C003461146B2EB9C0F24BF10BC7047A8
:1052F00053F82140491C2244B1EB9C0FF8D3002AFB
:1053000004BF10BC7047002010BC7047E848FDF790
:105310005FBAE64901200870704770B50E46054631
:105320001024FFF751FE15F0020F18BF052403D11A
:1053300015F0010F18BF09243246102C28BF70BD8C
:10534000002A08BF70BD204490F928102046BDE80F
:10535000704005F0BABDF0B5ADF6040D0446FFF798
:1053600033FE054614F0020F0AD06F460426384675
:10537000FCF763FE95F92C103A46304605F0A5FD82
:1053800014F0010F04BF0DF6040DF0BD08246E46A5
:1053900031460120FCF7A4FE95F930103246204634
:1053A00005F093FD0DF6040DF0BD2DE9F34F8BB024
:1053B00000200790086808900879029048790190C9
:1053C0008879B1F90890B1F90AA08A6904928A89AA
:1053D000D1E90784C0F5807602EA00070B980969D5
:1053E00010F0010F09914FF0000016D000900198C5
:1053F000002840F2FF800098012101FA00F209988C
:10540000104018BF01200390009A0499002001EB7E
:1054100082118346059100F0E3B8FCF79AF88346C1
:10542000DDE901014843032101EB400020F00302C4
:10543000414620460CF0D6F85846FCF78AF8019809
:105440004FF0000B002840F2D5800122099802FAA3
:105450000BF1084018BF01200021039004988C46EE
:1054600000EB8B1005904DE0012000FA01F2089846
:10547000024244D038F9020B039AA0EB0A000CF167
:10548000010C002A0CBF09EB0004A9EB000448083A
:10549000059A069052F82000CA07D50E0090E84001
:1054A00082B2C2F30420D3B212F4005F02D0002C07
:1054B00002DB03E0002C01DD9C1B00E09C19BC42D8
:1054C00005DD1F283ABF0024401C3C4606E0002CA6
:1054D00004DA0028C6BF3C46401E002402F40052F5
:1054E00042EA00204FF6FF73009AAB4020439A43F4
:1054F000A84042EA0003DDE9050240F82230491CD9
:10550000202902D202988445AED301980BF1010BF9
:1055100083459AD36EE0012101FA00F208990A420C
:105520005BD034F9021B039AA1EB0A010BF1010BCA
:10553000002A0CBF4944A9EB010138F9022BA2EB68
:105540000A0214BFA9EB02024A440029B4BF4B422D
:105550000B46002AB8BF52429A423ED9059B4208E8
:10556000069253F82220C3074FEAD36E0A9222FA1A
:105570000EF293B2C3F3042203F0FF0C13F4005FA6
:1055800002D0002902DB04E0002902DD0CEB060555
:1055900001E0ACEB0605BD4205DD1F2A3ABF002540
:1055A000521C3D4606E0002D04DA002AC6BF3D46E7
:1055B000521E002503F4005141EA022129434FF60F
:1055C000FF730A9A03FA0EF39A4301FA0EF142EAC4
:1055D0000103DDE9051241F82230401C202802D2E7
:1055E00002998B4597D300980199401C00908842FE
:1055F000FFF401AF0B98032826BF012007900798FE
:105600000DB0BDE8F08F2DE9F04F8BB00022059270
:105610000D794E7991F806C00C68CDF808C0B1F943
:105620000830B1F90A2006928A690392D1F810C0B5
:10563000CA69CDF81CC08989DDF808C001EA0C07E9
:10564000C0F108010091F0B1081EC0F2DF804FF0F8
:10565000000A002E7DD9012101FA00F00490009883
:10566000401E01FA00F00A904FF00108079808FA6E
:105670000AF1084018BF01200021019003988C46D0
:1056800000EB8A1BB4E04FF0000A002E61D94FF006
:105690000108079808FA0AF1084018BF0120002104
:1056A000019003988C4600EB8A1B4FE0E404011044
:1056B00000AF02005443524601208840204242D0AD
:1056C00032F9028B06980CF1010CA8EB0000DDF812
:1056D0000480B8F1000F0CBF03EB0008A3EB000837
:1056E000480808905BF820004FEAC1794FEAD96971
:1056F000049020FA09F080B210F4005F0AD0B8F1EB
:10570000000F0FDA10F4F85018BFA0F5807040F4C5
:10571000005007E0B8F1000F04DD10F4F85018BF96
:10572000A0F5807040F080004FF6FF7EDDF810801D
:105730000EFA09FE28EA0E0800FA09F048EA000805
:1057400008984BF82080491C202901D2AC45B3D3DE
:1057500000E054E00AF1010AB24598D34FE001207D
:105760008840204241D032F9028B06980CF1010C9E
:10577000A8EB0000DDF80480B8F1000F0CBF03EBCC
:105780000008A3EB0008480809905BF820004FEAE6
:10579000C1794FEAD969089020FA09F080B210F473
:1057A000005F03D0B8F1000F07DA02E0B8F1000F94
:1057B00003DDDDF8108020EA0800DDF80080B8F194
:1057C000000FC4BFDDF8288048EA00004FF6FF7ED6
:1057D000DDF820800EFA09FE28EA0E0800FA09F02A
:1057E00048EA000809984BF82080491C202901D27A
:1057F000AC45B4D30AF1010AB245FFF435AF0098C5
:105800000028C2BF05980BB0BDE8F08F4FF0000B29
:10581000002E45D90298C0F580700090029840F49F
:1058200080700190039A0020014602EB8B1A31E050
:1058300001224FEA184C82404FEA0C4C224226D0FB
:105840004FEA5009C2075AF82980D20E28FA02F30B
:105850009BB2DDF800E003F0FF0C0CEB5E0EDDF810
:1058600004C0491C0EEA0C0CBC4588BFBC4623F0A2
:10587000FF0343EA0C034FF6FF7C0CFA02FC28EA14
:105880000C0C03FA02F24CEA02024AF82920401CEE
:10589000202801D2A942CBD30BF1010BB345C1D3D0
:1058A000012005900BB0BDE8F08F2DE9F04F89B0D5
:1058B000002202920A790F6804924A790092B1F9A3
:1058C0000830B1F90A608A690592CA6909690391C9
:1058D000FE494969A0EB010CCCF1050881424AD888
:1058E0004AD100984FF0000A002844D901210398BA
:1058F00001FA0AFC1CEA000018BF0120019005997A
:105900000020844601EB8A1B2DE0012181403942B1
:1059100026D032F9021B019C891B4FEA19454FEA38
:1059200005450CF1010C002C0CBF5D185D1A4FEA07
:10593000500EC1075BF82E90CC0E29FA04F189B203
:10594000002DC8BF41F4005141F480514FF6FF755E
:10595000A54029EA0505A14045EA01044BF82E407F
:10596000401C202802D204998C45CED300980AF11D
:10597000010A8245BAD35BE0B8F1000F5DDB009805
:105980004FF00009002853D908F10800012101FA5D
:1059900000FB401E01FA00F008900124039804FA6D
:1059A00009F1084018BF01200021019005988C469C
:1059B00000EB891A34E00120884038422DD032F9BA
:1059C000020B019C801B0CF1010C002C0CBF1C185D
:1059D0001C1A480807905AF82000CD07ED0E0690D3
:1059E000E84080B210F4005F02D0002C04DA01E03D
:1059F000002C01DD20EA0B00B8F1000FC4BF089CA9
:105A000020434FF6FF7E0EFA05FE069CA84024EACE
:105A10000E04044307984AF82040491C202902D26A
:105A200004988445C7D3009809F101098145B4D38E
:105A3000B8F1000F04BF01200290029809B0BDE840
:105A4000F08F2DE9F04FD5B083460020884649906D
:105A5000489072B6FCF79AF80646FDF74AFD48B141
:105A6000FDF7EAFD4990FDF7D1FDFDF7EAFD48900D
:105A7000FDF7D7FDFBF770FFFBF7CAFE4E90FCF772
:105A800093F84D90FBF7C6FE0120FBF71EFD5290E8
:105A90001120FBF71AFD5190FDF74EFB4C90FDF7DE
:105AA00033FB4FF49350FDF7A0FA62B6FBF7F7FC17
:105AB0004B900120FBF7E9FC0120FBF74AFD5390D6
:105AC0000020FBF7EEFE50900020FBF7DFFE4F902A
:105AD0000020FBF730FB5490FAF70DFE4A900020AF
:105AE000FBF7B8F80020044636AF47F82040401CCA
:105AF0000628FAD3DFF8D89116F0020F4FF001050F
:105B000005D04FF40461484636950BF061FD16F060
:105B1000010F10D04FF480716E480BF059FD012039
:105B2000FAF780FE002818BF38951120FAF77AFEA0
:105B3000002818BF3995DFF8A0A1644E369850B3FD
:105B40000020FBF7F4FB00909AF800008DF80400A9
:105B500062480078012894BF6148624800788DF857
:105B600005000020FBF7DFFC002818BF4FF0FF30D6
:105B700004908DF806807088ADF80800ADF80A40F2
:105B80000020FBF788FBADF80C004FF04050CDE94A
:105B900006905548089037984FF0FF0838B300201A
:105BA000FBF7C5FB09909AF800008DF828008DF8E6
:105BB00029500D948DF82A807088ADF82C00ADF82E
:105BC0002E400020FBF767FBADF830009DF8050084
:105BD00009EB80110F919DF8041048434FF040519C
:105BE00001EB40011091404901EB40001190DFF8BA
:105BF000FC90DFF8FCA0389858B30120FBF797FB26
:105C00001290FBF743F800280CBF9AF8000099F8AF
:105C100000008DF84C000120FBF796FB05FA00F020
:105C20008DF84D000120FBF750FCC04316908DF815
:105C30004E80B088ADF85000ADF852400120FBF71F
:105C40002AFBADF85400234818902A4819902A4896
:105C50001A90399858B31120FBF769FB1B90FBF79A
:105C600015F800280CBF99F800009AF800008DF88C
:105C700070001120FBF768FB05FA00F08DF8710049
:105C80001120FBF722FCC0431F908DF87280B08872
:105C9000ADF87400ADF876401120FBF7FCFAADF8D2
:105CA00078001648219016482290164823909DF8B7
:105CB0004D000221022829D9042805D99DF84C203D
:105CC000199800EB820019901EE00000E404011016
:105CD0000040003040480030CA040110C9040110DF
:105CE000C8040110CB04011000200030CC040110C6
:105CF000CD0401104008003040280030C04800307A
:105D0000C00A0030C02A00308DF84D109DF8710097
:105D1000022809D9042805D99DF87020229800EBA3
:105D2000820022908DF871100120FBF7CEFB4FF01E
:105D3000553420B161000120FBF7B6FB1694112009
:105D4000FBF7C3FB28B14FF0AA311120FBF7ACFBE6
:105D50001F94BDF8520000F58060ADF85200BDF808
:105D6000760000F58060ADF87600FBF75CFF00265A
:105D7000B246B1463446B04642AF03F0EEF80128D1
:105D80007BD0BAF1800F78D83CA8FCF70AF900283C
:105D90007BD03CA803F036FF19F1010971D04FF018
:105DA000000948460AF1010A012147F82010401C69
:105DB0000628F9D3002C08BF00250CD0012C08BF01
:105DC00000251AD0022C08BF002528D0032C08BFBC
:105DD000012635D05EE036A850F8250048B105EB25
:105DE000C501684600EB81014046FFF75EFD47F8BC
:105DF00025006D1C062DEED322E036A850F82500B4
:105E000048B105EBC501684600EB81014046FFF74C
:105E1000FAFB47F825006D1C062DEED310E036A8DE
:105E200050F8250048B105EBC501684600EB81013B
:105E30004046FFF7BAFA47F825006D1C062DEED351
:105E40000121002057F82020CAB1401C0628F9D3B0
:105E5000A9B11F2C0ED20120641C00FA04F111EA32
:105E60000B0F07D1641C032C9CBF00FA04F111EA4C
:105E70000B0FF7D04FF0000803E00BE005E008F14E
:105E800001083EB9FBF7CFFE77E7FEF7B9FF002E1A
:105E90003FF473AFFBF7BEFC01205299FBF704FB04
:105EA00011205199FBF700FB4B98FBF7EEFA539842
:105EB000FBF74FFB5098FBF7F4FC4F98FBF7E6FC21
:105EC0005498FBF738F94A98FAF7C4FE4E9830B167
:105ED0004D9810B1FBF7A7FE01E0FBF76BFEFDF755
:105EE00008FB48B14998002818BFFDF707FB489800
:105EF000002818BFFDF73AFB4C98002818BFFDF7A3
:105F0000ACF8002E0CBF0120002055B0BDE8F08F8A
:105F10002DE9F04FFF48ADF63C0D01270678FEF75E
:105F200017FF012840F07181FB480068B0F9361076
:105F3000B0F934000BF097FB16F0020F00F05C8113
:105F40000DF50065FFF7C0F90024A0B1B0E80E1010
:105F500085E80E10B0E80E10103585E80E10B0E898
:105F60000E10103585E80E10D0E90010CDF830186D
:105F7000CDF8340827E0FF22382128460BF046FBF5
:105F8000E648CDF800084FF49070CDF804083820AA
:105F9000CDF808085020CDF810084FF0FF30CDF8AC
:105FA0000C48CDF81448CDF81848CDF81C48CDF869
:105FB0003448CDF82C08CDF82808CDF82408CDF8C1
:105FC0003048CDF82008D648FCF702FCDDF814086C
:105FD00040F27778401C0025CDF83848CDF81408F9
:105FE00080E0284604F015FF00287AD0008900EAF6
:105FF000080424F0CC0030F47C4072D00F212846F5
:10600000FFF701F800286CD0FBF7C0FDDDF8381869
:10601000002964D1FBF788FCFF210F20FFF711FD59
:10602000CDF83808FBF7F6FBDDF83808002856D124
:106030003FB314F0010F0ED0FEF7C6FF8146EA46CB
:106040004FF0040B5046FBF7F8FF99F92C1052461D
:10605000584604F03AFF14F0100F0FD0FEF7B4FFCB
:106060008346E9464FF0080A49460120FCF738F814
:106070009BF930104A46504604F027FFDDF83808F7
:1060800068BB14F0660F08D0FEF74BF9CDF838085E
:10609000FBF7C0FBDDF8380808BB07B314F0020FAC
:1060A0000DD0FDF754FD8146FEF78EFF05235FEA14
:1060B000090204D090F92D10184604F006FF14F0E0
:1060C000200F0CD0FDF7C9FC0446FEF77DFF092325
:1060D000220004D090F93110184604F0F6FEFFF7C4
:1060E000DFF86D1C04F091FEA842DDF8380803D9F2
:1060F00000283FF476AF03E0002808BF012000D05D
:10610000002018B1FEF7E0F9012827D0DDF81C08BF
:106110000023401CCDF81C085020CDF810081A466A
:106120002121072006F05EFE0020034602460146BC
:106130000090FE20FEF765FA0DF5006404F049FEBC
:10614000C8B18169CDF82018C169CDF8241841691A
:10615000CDF82818C068CDF82C0816E016F0080F06
:1061600014BFA220A120CDF81008DDF81808401CAB
:10617000CDF81808E0E74FF0FF30CDF82C08CDF847
:106180002808CDF82408CDF820086448CDF8000888
:106190004FF49070CDF804083820CDF8080800209E
:1061A000CDF80C08A3682246014652F820C0401CD6
:1061B0006144B0EB930FF8D34D42FF22511C684667
:1061C000E5600BF023FAA268F4E804018DE82700EB
:1061D0000FCC04AD85E80F000FCC08AD85E80F00AB
:1061E000D4E900014E4CCDE90C012046FCF7F0FA51
:1061F00069462046FCF78EFB0020FDF7BAFF00231E
:1062000032464021072006F0EDFD0DF63C0DBDE8BD
:10621000F04F02F05FBE3F4A002804BF5180704734
:10622000012808BF9180704701004FF00000394AF3
:1062300004BFB2F902007047012908BFB2F9040097
:10624000704770B50126FFF73FF820B10069A1281B
:1062500018BFA22801D0002070BD002404F0D5FD95
:10626000002833D9204604F0D4FD00281EBF05893C
:1062700025F0CC0030F47C4023D00F212046FEF7DF
:10628000C2FEF0B115F0010F0AD0FBF7E1FE38B9FC
:1062900044F4807200232021072006F0A3FD00268D
:1062A00015F0100F0BD00120FBF726FF38B944F48E
:1062B000805200232021072006F094FD0026FEF7DF
:1062C000EFFF641C04F0A1FDA042CBD8304670BDA6
:1062D0000020704700207047002818BF01200D499A
:1062E000487070470B484078002818BF012070475D
:1062F00070B582B00D460446FEF71FFD002877D129
:10630000044E306900287FD07078682300283FD081
:10631000002007E0E4040110F80501105443524640
:1063200000AF02007070B5F9000042F6E061014470
:1063300045F6D91291422BD3B5F90210081A41F251
:10634000883108444900884222D9288869888DF814
:106350000030030A8DF801308DF80200080A8DF82C
:10636000041003228DF803008DF805200023062277
:106370006946072006F066FD10210120FEF7FDFCAE
:106380000320B060F068401CF06002B0012070BDD6
:10639000B4F9000042F6F82188422ADDB4F902007F
:1063A00088422DDDB0680022401CB06003282BD34A
:1063B000208861888DF80030030A8DF801308DF84F
:1063C0000200080A8DF804108DF803008DF80520EE
:1063D000002306226946072006F034FD1021012023
:1063E000FEF7CBFCF068401CF06002B0012070BDED
:1063F0000AE007498842BCBFB4F902008842D1DBF9
:106400000020B06002B070BD02B0002070BD00007E
:1064100020D1FFFF70470020704710B503F0070040
:10642000042808BFFEF750FD002010BD70B503F032
:1064300007020025F84CF94B012A02D0022A14D099
:1064400011E0052018709D60FCF7C4FF22685321FD
:1064500011702268452151702268010A91702168EB
:10646000C87020680571002070BD1A78052A13D104
:106470009A68052A28BF104607D2D4F800C01CF835
:1064800002C080F800C0501C9860052804D101208B
:106490009D60087003201870012070BD2DE9F04147
:1064A00003F0070201260025DB4CDC4B012A02D059
:1064B000022A3BD037E0052018709D60FCF78AFF68
:1064C0002168AC270F702268010A5170216888701A
:1064D00004F052FCDFF8488380B1D8F8000004F0E3
:1064E00039FD58B1D8F8000090F8200010F0020FE4
:1064F00004D0206847702168432088702068C670E7
:106500002068057104F038FC50B1D8F8000004F0A0
:1065100021FD28B1D8F800002168007E487102E012
:106520002168FF2048710020BDE8F0811A78052A13
:1065300012D19A68062A28BF104607D2D4F800C0A4
:106540001CF802C080F800C0501C9860062803D1D7
:106550009D600E70032018700120BDE8F08103F0EB
:106560000702022A1CBF002070472022027001206F
:10657000087070472DE9F041A84F0D46064613F00C
:10658000070F04D003F00700022808D004E012F03F
:10659000040F1CBF0020B8700020BDE8F08102F09D
:1065A00093FC002814BF0124002402F090FC002872
:1065B00014BF0222002242EA0403B878002814BF64
:1065C0000422002242EA0300307001202870BDE856
:1065D000F08170B503F0070C0026904C8E4DBCF195
:1065E000010F0AD0204613F0070F00780DD0BCF140
:1065F000040F08BF062818D029E0A6602868067096
:10660000286846700520207021E005281FD1A06869
:10661000022803D22B681A54401CA060022816D10D
:106620000120A6600870062010E028680078552830
:106630000BD128684078AC2818BFBC2805D1286841
:106640000122411C062002F025FC032020700020BE
:1066500070BD70B503F0070200256F4C6F4B012A27
:1066600002D0022A24D021E0052018709D6002F09B
:10667000E6FB41F6E8710144B0F5283F10D8CA782E
:10668000086862F31F60674A904208BF002007D184
:106690000A18236812791A54401C1428F8D305E00C
:1066A000002021680D54401C1428FAD3002070BD2E
:1066B0001A78052A13D19A68142A28BF104607D2DF
:1066C000D4F800C01CF802C080F800C0501C9860CC
:1066D000142804D101209D60087003201870012047
:1066E00070BD70B503F0070200254B4C4B4B012ADF
:1066F00002D0022A3FD03CE0052018709D6002F0D5
:106700009EFB41F6E8710144B0F5283F2BD8CA78CA
:10671000086862F31F60434A904224D12268087CD3
:1067200010702268487C50702268887C90702068C5
:10673000CA7CC27020680A7A02712268487A507155
:106740002268887A90712268C87AD0712268087DA0
:1067500010722268487D50722268887D9072C87DD0
:106760002168C87205E0002021680D54401C0C28E7
:10677000FAD3002070BD1A78052A13D19A680C2A22
:1067800028BF104607D2D4F800C01CF802C080F819
:1067900000C0501C98600C2804D101209D60087036
:1067A00003201870012070BD70B503F007020025AA
:1067B000194C1A4E012A02D0022A3FD03CE004F0C4
:1067C00008FB40B3D0E906212368C0681A70D4F8EA
:1067D00000C0130A8CF80130D4F800C0130C120E5C
:1067E0008CF802302368DA702268117123680A0A73
:1067F0005A7123680A0C090E9A712268D1712168B6
:1068000008722268010A51722268010C9172010E0D
:106810002068C1720DE007E0CC3B010004050110C7
:10682000F805011034CD12AB21680D54401C0C2822
:10683000FAD305203070B560002070BD3278052A8B
:1068400010D1B2680C2A28BF104604D223689B5C82
:106850000370501CB0600C2804D10120B560087092
:1068600003203070012070BD70B503F007020024D2
:10687000FA4DFB4B012A02D0022A3ED03BE0052014
:10688000187000269C6002F0DAFA00F50051B0F5AD
:10689000283F98BF11F0030F27D1F24A08689042B1
:1068A00004BF0022104620D151F82030401C1A4469
:1068B0000728F9D302B1C6B128680A7C02702A6899
:1068C000487C50702A68887C90702A68C87CD07098
:1068D0002A68087D10712A68487D50712A68887D71
:1068E0009071C87D2968C87105E0002029680C54A2
:1068F000401C0828FAD3002070BD1A78052A13D14D
:106900009A68082A28BF104607D2D5F800C01CF89C
:1069100002C080F800C0501C9860082804D10120F3
:106920009C60087003201870012070BD2DE9F041B3
:1069300003F0070C0027CA4E4FF00508BCF1010F09
:106940000DD013F0070F0FD03246BCF1020F1278B2
:1069500010D0BCF1040F08BF062A26D058E086F8F4
:1069600000807770B76053E07270BF48B062062055
:1069700030704DE0052A15D1B268042A28BF1046B0
:1069800009D2C2F10303D6F828C0DB002CFA03F3C6
:106990000370501CB060042804D10120B760087057
:1069A000032030700120BDE8F081707801250024BB
:1069B00010F0010F11D002F042FAB0F5283F23D8B1
:1069C0006A030021B1EB900F07D252F8043B491C37
:1069D0001C44B1EB900FF8D3B5B1707810F0020FF2
:1069E0000ED004F0F6F978B182680021B1EB920F75
:1069F00006D250F8043B491C1C44B1EB920FF8D36B
:106A0000002D18BFB46200D1B762777086F800809D
:106A10000020BDE8F081F0B503F0070C00268F4D93
:106A20008F4C83B0BCF1010F0ED013F0070F1DD0B7
:106A3000224603271278BCF1020F26D0BCF1040FC6
:106A400008BF062A36D03CE002AA01A9684602F037
:106A500073FD052020702968019808702968009846
:106A60004870296802988870A6602AE0A068032808
:106A700003D229680A54401CA060022821D30621B1
:106A80002170032808BFA6601BE0052A0FD1A26869
:106A9000032A28BF104604D22B689B5C0370501C4D
:106AA000A060032803D10120A6600870277003B0FE
:106AB0000120F0BD286882780178407802F031FD2D
:106AC000277003B00020F0BD08B503F007000128CF
:106AD0000AD104F051F938B101208DF800000246C6
:106AE00069460D2002F0D6F9002008BD08B503F074
:106AF000070001280AD104F03FF938B100208DF8D1
:106B00000000012269460D2002F0C4F9002008BDF2
:106B100008B503F00700012809D104F02DF930B1C0
:106B200003208DF800000122694602F0B3F900202D
:106B300008BD0020704708B503F0070001280AD1FE
:106B400004F01AF938B10B208DF8000001226946D3
:106B5000032002F09FF9002008BD1FB513F0070FB6
:106B60000ED104F009F958B19DF80800F0280AD0B8
:106B700004F002F920B1012202A9092002F08AF9E9
:106B800004B0002010BDFEF7C1FBF9E700207047FC
:106B900070B503F00700314C314D012808D013F0D7
:106BA000070F12D0042804BF2878062816D01FE04B
:106BB0000020A860216808702168487021688870EA
:106BC0002168C8700520287012E0A86804280FD238
:106BD00021680A54401CA860062008E004F0CCF8A4
:106BE00030B104221046216802F054F903202870C5
:106BF000002070BD10B503F00700012804D103F098
:106C000043F9174900200871002010BD70B50546F2
:106C100003F007000C4601280AD013F0070F02D03A
:106C2000022807D004E0012200211B2002F032F9E3
:106C3000002070BD03F012FB28700120207070BD91
:106C400010B503F0070C064CBCF1010F0ED013F089
:106C5000070F11D0BCF1020F20D01DE0CC3B01008A
:106C60000405011054464953EFBEADDE0020A0607C
:106C700006F0AFF8A0610FE0A068002804BF100282
:106C8000A06106D0012804D1A0691043A06106F0DC
:106C90009FF8A068401CA060002010BDA26812B13F
:106CA000012A04D007E0218B090A017003E0237E4A
:106CB000037001200870501CA060012010BD10B5A9
:106CC00003F0070CFE4CBCF1010F06D013F0070FC8
:106CD00009D0BCF1020F18D015E00020A06006F02A
:106CE0007BF8A0610FE0A068002804BF1002A0613B
:106CF00006D0012804D1A0691043A06106F06FF806
:106D0000A068401CA060002010BDA26812B1012A3A
:106D100004D007E0218B090A017003E0237E037091
:106D200001200870501CA060012010BD70B503F058
:106D3000070CE34D0E460446BCF1010F06D013F0DC
:106D4000070F07D0BCF1020F18D015E00020A86093
:106D5000E86011E0A868002804BF1002A86108D00C
:106D6000012806D1A869104381B2A861E8880AF019
:106D70007FFCA868401CA860002070BDE86802285D
:106D80000ED2E8880AF079FCEB6882B2002B04BFCF
:106D9000100A207004D0012B02D122700120307023
:106DA000E868401CE860012070BD10B403F0070CD7
:106DB000C34CBCF1010F08BF00200BD013F0070F2C
:106DC00003D0BCF1020F09D005E0A068002808BF7D
:106DD000E280401CA06010BC00207047A2681AB975
:106DE000A379037001200870501CA06010BC012022
:106DF00070472DE9F047064603F00700B04F89467B
:106E0000012808BF002039D0DFF8B882AE4D13F05A
:106E1000070F02D0022835D031E0B868002808BF3B
:106E20007A7029D0012804BF1002B86124D002284A
:106E300022D1B8691043B8617E7884B203F09CFF18
:106E4000D0B1062E18D2DFE806F00306090C1014A4
:106E5000A8F80E4010E0A8F80C400DE028688486E1
:106E60000AE02868A0F80C4106E02868A0F8504025
:106E700002E02868A0F85240B868401CB8600020C2
:106E8000BDE8F087F86802282CD297F801A000240A
:106E900003F072FFD8B1BAF1060F18D2DFE80AF09A
:106EA0000306090C1014B8F80E4010E0B8F80C40B6
:106EB0000DE02868848E0AE02868B0F80C4106E0EE
:106EC0002868B0F8504002E02868B0F85240F868EE
:106ED000002804BF200A307004D0012802D1347089
:106EE00089F80000F868401CF8600120BDE8F087D0
:106EF0002DE9F0411C4617460E46054603F03CFFBF
:106F000068B114F0070F04D004F00700022809D07C
:106F100005E0002F14BF012000200AF0B3FB002081
:106F2000BDE8F081674890F86C00C0082870012027
:106F30003070BDE8F0812DE9F0411C4615460F4642
:106F4000064613F0070F08D103F016FF28B1022DF3
:106F50003CBF28460AF09BFB03E004F00700022830
:106F600002D00020BDE8F0810AF096FB30700120CD
:106F70003870BDE8F08170B503F007020026534C6D
:106F80004F4D012A02D0022A15D012E006F0FBFB79
:106F900021680870FDF7DCFE2168487003F0BCFA38
:106FA00021688870FDF7DAFE2168C8700520287016
:106FB000AE60002070BD2A78052A10D1AA68042A84
:106FC00028BF104604D223689B5C0370501CA86045
:106FD000042804D10120AE6008700320287001202D
:106FE00070BD70B503F00702384C0025344E012AFD
:106FF00002D0022A54D051E0FEF766F9002836D0BC
:107000004169FF292CBFFF21C9B222681170816933
:10701000FF2934BFC9B2FF2122685170C169FF291D
:1070200034BFC9B2FF21226891702268017CD170FF
:10703000226890F820101171018C2268090A5171A0
:10704000016A2268090C9171016A2268090ED171E6
:10705000016BFF2934BFC9B2FF2122681172406B56
:10706000FF2834BFC0B2FF202168487215E02068B5
:107070000570206845702068857021685020C870B0
:107080002168FF2008712168487121688871216892
:10709000C8712068057220684572B560002070BD17
:1070A000B2680A2A28BF104604D223689B5C03708A
:1070B000501CB0600A2802D10120B560087007E0BA
:1070C00004050110D0AC0110F8050110CC3B010003
:1070D000012070BD03F00702FE4B4FF0000C012AA7
:1070E00008BFC3F808C001D0022A01D000207047B1
:1070F0009A68022A3DBF80F800C0501C9860104674
:10710000022803D10120C3F808C00870012070478D
:107110002DE9F047064603F00700EE4F8A464FF090
:107120000008012808BFC7F8088001D0022802D053
:107130000020BDE8F087B868A0BB0024254601F018
:107140007EFE014600F5005018384FF400524FF013
:107150004009B1F5283F20D890F803C003686CF3CC
:107160001F63DFF874C3634517D1091FB4EB910F98
:1071700006D252F8043B641C5D40B4EB910FF8D387
:10718000C17D406961F31F60A84206D103F0BAFDDA
:10719000012804BF8020307001D086F80090B868C4
:1071A000401CB860012803D1C7F808808AF80000A5
:1071B0000120BDE8F0872DE9F04103F00702002629
:1071C000C64CC44D012A02D0022A56D052E0FCF728
:1071D00001F90520287003F0CFFD002849D0C04FE9
:1071E000386803F0B7FE002843D00AF05AFA804608
:1071F0000AF05CFA39680A7E12F0040F11D0C98ACD
:107200002268090A117039682268897D51703968CD
:107210002268898A090A917039682268097DD170CB
:1072200010E0898A2268090A117039682268097D8C
:10723000517039682268C98A090A917039682268D0
:10724000897DD17022684FEA18211171216881F877
:1072500005802268010A91712168C8713868226826
:10726000817C11722268017C5172008B2168000AB6
:107270008872AE600020BDE8F0812A78052A10D11E
:10728000AA680B2A28BF104604D223689B5C0370AF
:10729000501CA8600B2804D10120AE6008700320A8
:1072A00028700120BDE8F0812DE9F04703F00702C6
:1072B00000268A4D874B012A02D0022A5DD059E070
:1072C0000520187000249E6001F0B9FD00F5005300
:1072D000B0F5283F98BF13F0030F45D1814A1968D4
:1072E000914204BF0022114608D153F821C0491C25
:1072F00062440729F9D3002A08BF01249F7C93F830
:10730000138084B341F6E8710144B0F5283F07D8F3
:10731000CA78086862F31F606F4A904208BF012470
:1073200091F8129091F813A0002C08BF002014D0FF
:1073300003F04FFD2968806981F80090296881F881
:1073400001A02A68010C000E91702968C870286895
:107350000771286880F805800CE029680E54401CED
:107360000628FAD306E0FFE7002029680E54401CE7
:107370000628FAD30020BDE8F0871A78052A13D131
:107380009A68072A28BF104607D2D5F800C01CF813
:1073900002C080F800C0501C9860072804D101206A
:1073A0009E600870032018700120BDE8F08710B5BA
:1073B00003F0070C474CBCF1010F06D013F0070F88
:1073C0000AD0BCF1020F1AD017E00020A060E060E4
:1073D0000AF071F9A06110E0A068002804BF100253
:1073E000A06107D0012805D1A0691043A06180B237
:1073F0000AF066F9A068401CA060002010BDE26899
:10740000022A0BD212B1012A04D007E0218B090A0B
:10741000017003E0237E037001200870501CE060BF
:10742000012010BD70B503F007010026294D044668
:10743000012908BFEE6201D0022901D0002070BDF1
:10744000E86A002804BF28480AF03FF9E96A0829D9
:1074500028BF267002D22448405C2070481CE86295
:10746000012070BD2DE9F04103F007010026194D00
:107470000746012908BFEE6201D0022902D0002090
:10748000BDE8F08195F82C0000F00704287920432E
:1074900004D115480AF019F901202871052C28BFDC
:1074A0002E711148005D3870E86A401CE8620120C6
:1074B000BDE8F08170B5044603F007000D460228D0
:1074C0001CBF002070BD0AF005F920700120287053
:1074D00070BD00000405011034CD12ABCC3B01009F
:1074E000F8050110544649533405011070B503F0F6
:1074F00007020025F94C012A02D0022A12D00FE01F
:1075000005202070002211461046A56002F014F8F4
:107510004FF6FF7101EA4000206102F020F860623E
:10752000002070BD2278052A17D1D4F810C0A268B7
:10753000624528BF104607D212F0010F1CBF6378C6
:1075400003700CD0501CA060604506D10120A560DE
:1075500008700320207002F010F8012070BD666AE8
:1075600022F00103F35A1E0A06706370EAE770B551
:1075700003F007020025D94C012A02D0022A11D0BB
:107580000EE0D74805220068B0F91210B0F91000DB
:10759000227008444000A560206102F0E3F96062B7
:1075A000002070BD2278052A17D1D4F810C0A26837
:1075B000624528BF104607D212F0010F1CBF637846
:1075C00003700CD0501CA060604506D10120A5605E
:1075D00008700320207002F0D3F9012070BD666AA4
:1075E00022F00103F35A1E0A06706370EAE70020D6
:1075F000704770B50D46044613F0070F04D003F032
:107600000700022805D002E01046FDF799FB002094
:1076100070BDFDF79AFB20700120287070BD70B519
:1076200003F007020325AD4C012A02D0022A11D033
:107630000EE0FDF78AFB03F026FEE06100281ABF8A
:1076400005202070257003F016FE20620020A06047
:10765000002070BD2278052A0BD1E369A2689B5CEB
:107660000370501CA060226A904202D3012008706F
:107670002570012070BD7FB51C460E46054613F0EF
:10768000070F08D103F078FB28B1012202A92A20B4
:1076900001F000FC03E004F00700022802D004B06F
:1076A000002070BD02F013F828700120307004B083
:1076B00070BD2DE9F04103F007020027874E884690
:1076C0000546012A02D0022A0BD007E005203070BF
:1076D0000A20B760306101F042FF70620020BDE80F
:1076E000F0813078052819D1B2683069824228BF0C
:1076F000104608D212F0010F1CBF7078287010D00D
:10770000B068401CB0603169884207D10120B76081
:1077100088F800000320307001F02FFF0120BDE841
:10772000F081002401F0D3FF012804D1B068716A10
:1077300020F001000C5A200A28707470E0E77FB531
:107740001C460E46054613F0070F08D103F014FB44
:1077500028B1012202A9242001F09CFB03E004F0DF
:107760000700022802D004B0002070BD06F0FCF82B
:1077700028700120307004B070BD7FB51C460E46E5
:10778000054613F0070F08D103F0F6FA28B10122DD
:1077900002A90C2001F07EFB03E004F007000228A0
:1077A00002D004B0002070BD05F0EDFF287001206C
:1077B000307004B070BD7FB51C460E46054613F010
:1077C000070F08D103F0D8FA28B1012202A90F202F
:1077D00001F060FB03E004F00700022802D004B0CF
:1077E000002070BD03F043F900F00F0040F01000DE
:1077F00028700120307004B070BD2DE9F04103F015
:10780000070C364D0E460746BCF1010F07D0354C2C
:1078100013F0070F07D0BCF1020F1BD017E00020B8
:10782000A860E86013E0A86804283CBF21680A54F7
:10783000032809D1206821680068C97800BA20F0BF
:10784000FF000843FDF766F8A868401CA860002008
:10785000BDE8F081E86870B9FDF761F8216820F0B3
:107860007E42100E08702168100C48702168100AC2
:1078700088702068C270EA68042A06D22068032A49
:10788000805C387004BF01203070501CE86001201B
:10789000BDE8F0817FB51C460D46064613F0070F84
:1078A00008D103F069FA28B1012202A9102001F0E1
:1078B000F1FA03E004F00700022802D004B000202F
:1078C00070BD03F016F900F00F0403F0D0F864F374
:1078D0001F1030700120287004B070BD0405011025
:1078E000F8050110CC3B010010B503F00702F74C7E
:1078F000012A02D0022A0DD00AE003F046FD002141
:10790000E06100281ABF4FF4056020622162A16087
:10791000002010BD236AA2689A4228BF104607D2F1
:10792000D4F81CC01CF802C080F800C0501CA06035
:10793000984204BF01200870012010BD10B413F05C
:10794000070F4FF0402C04D003F00702022A13D097
:107950000FE0012A04BFDCF8140040F0010006D05B
:10796000002A04BFDCF8140020F0010001D1CCF89B
:10797000140010BC00207047DCF81430002213F013
:10798000010F18BF0122D24BD3F83CC0D14B1B686A
:10799000B3F8A430C3F30334012303FA04F41CEA5C
:1079A000040F18BF42F0020202700B7010BC0120DD
:1079B000704770B514460E46054613F0070F04D005
:1079C00003F00700022813D010E0002C14BF0120A0
:1079D000002002F04BFA4CB14FF04020016B21F433
:1079E000405141F4BE0141F020410163002070BDCF
:1079F00002F043FA002814BF012200222A7001205D
:107A0000307070BD2DE9F04103F0070CAF4C0F460C
:107A10008046BCF1010F12D0AD4E13F0070F4FF0AE
:107A2000030510D02046BCF1020F027822D0BCF131
:107A3000040F02BFA0680128062A2FD032E00520DB
:107A40002070002014E0A06810B1012804D00DE0DF
:107A500062700620207009E0607800EA020131635C
:107A600020EA02017163FBF723F82570A068401C2F
:107A7000A06017E0A068012808BF062A03D160783B
:107A8000FBF71BF82570F06B88F8000001203870B8
:107A9000A068401CA0600120BDE8F0816078FBF781
:107AA0000CF825700020BDE8F08170B5044603F0A5
:107AB00007000D4602281CBF002070BDFDF735FAF7
:107AC000002814BF0122002222700120287070BDFE
:107AD00070B50D46044613F0070F04D003F00700FD
:107AE000022805D002E0104605F07EFD002070BDA2
:107AF00005F07DFD20700120287070BD70B50D4629
:107B0000044613F0070F04D003F00700022805D045
:107B100002E01046F9F798F8002070BDF9F797F8E1
:107B200020700120287070BD70B503F00702DFF8E7
:107B30009CC10C460546012A08BF05200DD013F054
:107B4000070F08BF062008D0022A09D0042A04BF64
:107B50009CF80000062809D00EE08CF800000BE02D
:107B6000FDF7E9F928700120207070BD03208CF822
:107B700000000120FDF7E2F9002070BD70B503F0B0
:107B80000702524D0E460446012A04BF0020A86099
:107B900001D0022A01D0002070BD09F0A0FDAA6822
:107BA000002A04BF000A207004D0012A02D12070EC
:107BB00001203070501CA860012070BD70B50446D3
:107BC00003F007000D46022807D013F0070F04BF8B
:107BD0001046FDF7AFF8002070BDFDF7AEF820703D
:107BE0000120287070BD70B5044603F00700374DC2
:107BF0000E46012804BF0020A86014D013F0070F20
:107C000002D0022811D00EE0A868334904283CBFF6
:107C10000B681A54401CA860042804D10422096887
:107C2000132001F037F9002070BD06F0ACFBAA6804
:107C3000002A04BF000E20700FD0012A08BF000CDC
:107C400006D0022A08BF000A02D0032A02D004E0AC
:107C5000207002E0207001203070501CA8600120CC
:107C600070BD70B503F0070C184D0E460446BCF10C
:107C7000010F04BF0020A86015D013F0070F03D038
:107C8000BCF1020F11D00EE0A868134902283CBFD6
:107C90000B681A54401CA860022804D1022209680B
:107CA000142001F0F7F8002070BD06F03FFBAA6831
:107CB000002A04BF000A207004D0012A02D12070DB
:107CC00001203070501CA860012070BD0405011017
:107CD00000100040F8050110CC3B010070B50446CF
:107CE00003F00700FE4D0E46012804BF0020A860E7
:107CF00014D013F0070F02D0022811D00EE0A868AC
:107D0000F84904283CBF0B681A54401CA86004289A
:107D100004D104220968152001F0BCF8002070BDD0
:107D200006F05AFBAA68002A04BF000E20700FD08C
:107D3000012A08BF000C06D0022A08BF000A02D0A0
:107D4000032A02D004E0207002E02070012030708D
:107D5000501CA860012070BD70B5044603F00700F8
:107D6000DF4D0E46012804BF0020A86037D013F075
:107D7000070F02D0022834D031E0A868D94C00287F
:107D800004BF21680A7021680978012901D039B13E
:107D90001BE0002818BF04283CBF21680A5414E0E7
:107DA00006F033FB21680009487006F024FBC0F39D
:107DB000032606F02AFB216846EA0010887006F0C8
:107DC0001AFB2168C8700320A860A868401CA8603E
:107DD000042804D104221620216801F05BF8002059
:107DE00070BD06F01EFBAA68002A04BF000E2070BA
:107DF0000FD0012A08BF000C06D0022A08BF000AD3
:107E000002D0032A02D004E0207002E0207001209A
:107E10003070501CA860012070BD10B503F007023F
:107E2000AF4C012A02D0022A27D024E003F0ADFA99
:107E30000023002804BFE36123621BD000F150013E
:107E4000E1614168B1F5887F90F820100CD390F87B
:107E5000212001EB020C01FB02C190F8222090F8D6
:107E600023001044084404E090F822000A1801FBA3
:107E700000202062A360002010BD236AA2689A42FD
:107E800028BF104607D2D4F81CC01CF802C080F8E6
:107E900000C0501CA060984204BF0120087001205F
:107EA00010BD03F00702012A02D0022A05D002E029
:107EB0008B490020886000207047012202700A7000
:107EC0001046704710B513F0070F04D003F00702F7
:107ED000022A05D002E0104601F05CFB002010BD34
:107EE000814A127802700120087010BD10B513F09D
:107EF000070F04D003F00702022A05D002E0104663
:107F000001F04BFD002010BD784A1278027001206C
:107F1000087010BD002070471FB513F0070F07D180
:107F200002F02AFF20B1012202A90B2000F0B2FFCB
:107F300004B0002010BD70B503F00700684C154672
:107F4000012804BF0020A06024D013F0070F21D126
:107F500002F012FFF0B1A068624E03283CBF316806
:107F60000D54401CA060032814D1F9F7F5FC3068CB
:107F7000B0F8010045BAF9F74BFC040018BFF9F757
:107F800085FE306829460078F9F7F3F8002C18BF11
:107F9000F9F77FFE002070BD70B503F00700504C6C
:107FA0001646012804BF0020A06029D013F0070F57
:107FB00026D102F0E1FE18B3A0684A4D02283CBF6A
:107FC00029680E54401CA060022819D1F9F7C4FC9E
:107FD000F9F71EFC040018BFF9F758FE286800786E
:107FE00080B129684978F9F73BF928684178007829
:107FF00040F01000F9F734F9002C18BFF9F749FEEA
:10800000002070BD286841780020F3E77FB51C464A
:108010000E46054613F0070F08D102F0ADFE28B159
:10802000012202A91A2000F035FF03E004F0070046
:10803000022802D004B0002070BD05F07FFB0028AC
:1080400014BF012200222A700120307004B070BDDC
:108050007FB51C460E46054613F0070F08D102F007
:108060008BFE28B1012202A91C2000F013FF03E0BF
:1080700004F00700022802D004B0002070BD05F013
:108080004AFB28700120307004B070BD2DE9F0412A
:1080900003F0070C124C0E460746BCF1010F07D047
:1080A000104D13F0070F07D0BCF1020F22D015E0DE
:1080B0000020A060E06011E0A06803283CBF2968B0
:1080C0000A54401CA060032808D12868B0F80100B9
:1080D00040BA01B228680078FEF79DF8002007E05A
:1080E00004050110CC3B0100490501104E050110AB
:1080F000BDE8F081E268022A12D242B9286800780D
:10810000FEF792F82A68010A517029688870286879
:10811000E2681044012A4078387004BF01203070B2
:10812000E068401CE0600120D9E770B503F007006B
:10813000FA4C1546012804BF0020A06017D013F0A8
:10814000070F14D102F018FE88B1A068F44B032881
:108150003CBF19680D54401CA060032807D1186863
:10816000B0F8010041BA18680078FAF713F8002057
:1081700070BD10B503F00702E84C012A02D0022AB4
:1081800007D004E00020A060FBF715F8A0610020F4
:1081900010BDA268042A07D2C2F10303D4F818C0A4
:1081A000DB002CFA03F30370501CA060042804BF0A
:1081B00001200870012010BD10B503F00700012850
:1081C00007D102F0D9FD20B100221146202000F095
:1081D00061FE002010BD2DE9F04103F00705CF4EF0
:1081E000174688460446012D04BF0020B0601BD00E
:1081F00013F0070F16D102F0BFFD98B1B068C84B5D
:1082000003283CBF19680F54401CB06003280BD1F1
:10821000186890F9022090F9011090F90000FCF71D
:108220002AFA01E0022D02D00020BDE8F081B068FA
:1082300030B1012809D002280CD003280FD015E056
:108240001420FCF748F9207010E01520FCF743F9E2
:1082500020700BE01620FCF73EF9207006E0172096
:10826000FCF739F92070012088F80000B068401C44
:10827000B0600120BDE8F08170B50D46044613F0F2
:10828000070F04D003F00700022805D002E0A3493D
:1082900000208860002070BD0120FCF71CF92070D0
:1082A0000120287070BD70B503F0070C00269C4CAF
:1082B0009A4DBCF1010F06D013F0070F0CD0BCF1A2
:1082C000020F1FD01CE005F026FBAE60216808708D
:1082D0002168000A487013E0A868022803D22168C8
:1082E0000A54401CA86002280AD1AE6020680078B9
:1082F00010F0010F04D002221D20216800F0CAFDF9
:10830000002070BDAA68022A28BF104604D2236844
:108310009B5C0370501CA860022804D10120AE6051
:10832000087003202870012070BD7FB51C460E46E2
:10833000054613F0070F08D102F01EFD28B10122F7
:1083400002A9272000F0A6FD03E004F007000228A0
:1083500002D004B0002070BD09F0C6F928700120D9
:10836000307004B070BD7FB51C460E46054613F054
:10837000070F08D102F000FD28B1012202A9222036
:1083800000F088FD03E004F00700022802D004B0EA
:10839000002070BD09F0ADF928700120307004B0E4
:1083A00070BD7FB51C460E46054613F0070F08D179
:1083B00002F0E2FC28B1012202A9262000F06AFDA9
:1083C00003E004F00700022802D004B0002070BDD2
:1083D00009F094F928700120307004B070BD7FB5A9
:1083E0001C460E46054613F0070F0ED102F0C4FCE2
:1083F00058B19DF80800002818BF09F084F901223F
:1084000002A9212000F046FD03E004F00700022845
:1084100002D004B0002070BD09F07AF92870012064
:10842000307004B070BD2DE9FF413C4E1C460F4634
:10843000054613F0070F1CD102F09EFCC8B19DF851
:108440000800002818BF012802D0022807D014E035
:10845000F070012202A9082000F01CFD0DE0F07070
:1084600004208DF80800012202A9082000F012FD66
:1084700003E004F00700022803D004B00020BDE8A8
:10848000F081F07828700120387004B0BDE8F081E8
:108490007FB51C460D46064613F0070F08D102F0C3
:1084A0006BFC28B1012202A9082000F0F3FC03E0D4
:1084B00004F00700022802D004B0002070BDFCF7D1
:1084C00047FC801E05280ED2DFE800F003070905EF
:1084D0000B00002008E0012006E0022004E0032059
:1084E00002E0042000E0FF2030700120287004B07A
:1084F00070BD2DE9F0411C4617460E46054613F0A7
:10850000070F0FD102F038FC60B1384605F066F86D
:1085100000221146012000F0BDFC07E00405011017
:10852000CC3B010004F00700022802D00020BDE887
:10853000F08105F056F8287001203070BDE8F08118
:1085400010B5104613F0070F08BF05F00AF9002018
:1085500010BD10B5104613F0070F08BF05F008F95D
:10856000002010BD70B5044603F007000D46022838
:108570001CBF002070BD05F003F920700120287099
:1085800070BD03F0070230B4FA4B4FF0000C012A23
:1085900005D0022A04BF1A78022A0BD01EE002205E
:1085A0001870F548C3F808C06FF07F410068081ADA
:1085B000986113E09A68042A28BF104606D29D6984
:1085C000D40025FA04F40470501C9860042805D1E6
:1085D0000120C3F808C008700320187030BC0120C7
:1085E000704713F0070F04BFE44802700020704783
:1085F00010B503F00700DF49012804BF00208860A0
:1086000013D013F0070F10D18868DD4B04283CBF4E
:10861000D3F800C00CF80020401C8860042804D166
:1086200004221220196800F035FC002010BD2DE94D
:10863000F0478C4603F007010024CE4F164601296F
:1086400004BFBC60FC6062D013F0070FCD4BDFF8B5
:10865000388307D0022932D0042904BF387806288D
:108660004DD055E0BD68002D08BFFE6124D0012D1E
:1086700006D0D7F81090AC1E4C4515D27CB908E056
:10868000701C3861F9690844B0F5807F88BF3C618F
:1086900012E04FF480721946BC4808F094FFB849C4
:1086A000F869096820440E54601C484504D1B74855
:1086B000C0F8FC8006203870681CB86028E0FF21F4
:1086C00001703B69C3B1FA69F9680A44B2F5807F69
:1086D00010D2AF4D2D68454518BF047004D102F586
:1086E000283292F8002A0270481C984204BF0120E8
:1086F0008CF80000481CF8600120BDE8F0871D469A
:108700001846FAF765F8A1492846FAF703F93C70CC
:108710000020BDE8F0870020704770B503F0070027
:10872000944C1546012804BF0020A06014D013F01B
:10873000070F11D102F020FB70B1A0689049022808
:108740003CBF0A681554401CA060022804D10222D4
:108750000968052000F09EFB002070BD2DE9F04166
:10876000054603F00700864C824E0F4601280AD0CA
:1087700013F0070F14D002281BD0042804BF307850
:10878000062834D03FE00020B060216808702168DE
:108790004870216888702168C8700520307032E008
:1087A000B06804282FD221680A54401CB06006200B
:1087B00028E0B06860B904F005FF216808702268FD
:1087C000010A51702268010C000E91702168C87076
:1087D000B06804283ABF2168095CFF21297024BFD2
:1087E00001213970401CB0600120BDE8F08102F029
:1087F000C3FA40B12068C178006861F31F6004F0DB
:10880000DCFE032030700020BDE8F08100207047BE
:108810007FB51C460E46054613F0070F08D102F03F
:10882000ABFA28B1012202A9112000F033FB03E0CA
:1088300004F00700022802D004B0002070BD08F048
:108840006CFF28700120307004B070BD00207047AC
:108850001FB513F0070F04D1012202A91E2000F05A
:1088600019FB04B0002010BD03F0070041490128A6
:1088700006D013F0070F04BF0878012806D014E0D3
:10888000012008700020886048610DE08868042895
:1088900005D24B69401C42EA03224A6188600428E1
:1088A00003D1032008704869C8610020704703F0B5
:1088B0000700DFF8C0C0012807D013F0070F04BF7E
:1088C0009CF80000022809D01EE002208CF800006D
:1088D0000020CCF80800CCF8180015E0DCF80800FF
:1088E000022808D2DCF81810401C42EA0121CCF81A
:1088F0001810CCF80800022806D1DCF81800CCF8D3
:10890000200003208CF800000020704770B403F0B2
:1089100007020025174C012A02D0022A06D002E0E5
:1089200002202070A56070BC002070472278022AC7
:108930001CD1D4F820C0A268624528BF10460ED2D0
:1089400012F0030F04D1E36953F8046BC4E9066322
:10895000237E0370A069000AA061501CA0606045DE
:1089600004D10120A56008700320207070BC012094
:108970007047000004050110880401102404011050
:10898000CC3B010000AA0200554E564D902201102A
:10899000FCAA020070B503F007000025FE4C0E464D
:1089A000012806D013F0070F04BF2078022805D055
:1089B0002BE002202070A560A56126E0216AA06856
:1089C000884219D2A169090A41EA0262401CA261E7
:1089D00010F0030FA0600FD1E069B0F5303F28BF61
:1089E000026006D2B0F5005F03D30422EB49F9F729
:1089F000EEFFE069001DE061216AA068884204D1B1
:108A00000120A560307003202070002070BD70B57B
:108A100003F0070C0025E04CBCF1010F08BFA56076
:108A200039D013F0070F03D0BCF1020F35D032E07C
:108A3000052A08BFDA482DD005DC16D2DFE802F09F
:108A4000171A1D202200D748202A006808BFB4301A
:108A500020D006DC102A1DD0112A08BFD24819D018
:108A600003E0302A11D0312A12D0656113E04FF4AF
:108A700000500FE04FF42F300CE04FF41C3009E0B1
:108A8000CA4807E04FF42C3004E001F0D5FA01E0C9
:108A900006F0EEFE6061002070BDA268042A07D2D5
:108AA000C2F10303D4F814C0DB002CFA03F3037003
:108AB000501CA060042824BF01200870012070BD54
:108AC00070B403F0070CB44DBCF1010F07D0B84CE3
:108AD00013F0070F07D0BCF1020F21D01DE00020DA
:108AE000A860E86019E0A86805283CBF21680A541E
:108AF000042810D123682268D4F800C0D3F80130CC
:108B0000696912781BBA9CF804C023F0FF0343EA9A
:108B10000C0341F82230401CA86070BC0020704754
:108B2000EB6873B1042B07D22268032B1A445278E6
:108B3000027004BF01200870581CE86070BC01205E
:108B400070472268D5F814C012785CF82220266895
:108B50004FEA126C86F801C026684FEA124C86F87C
:108B600002C026684FEA122C86F803C0D4F800C071
:108B70008CF80420D8E710B503F00700012804D1D1
:108B8000002211460E2000F085F9002010BD2DE9CD
:108B9000F04103F00704804E174688460546012C35
:108BA00004BF0020B06017D013F0070F12D102F0FD
:108BB000E3F878B1B0687E4902283CBF0A681754D0
:108BC000401CB060022807D102220968072000F08B
:108BD00061F901E0022C02D00020BDE8F081B2680A
:108BE00012B1012A04D009E0FCF7B2F8287005E0C0
:108BF000FCF7B4F82870012088F80000B068401C29
:108C0000B0600120BDE8F08170B503F007000025D9
:108C1000614C012808D013F0070F0BD0042804BFC3
:108C20002078062825D02DE06561A5616570A560D6
:108C3000257027E0A068022807D2616942EA012175
:108C4000616161781144617010E0042807D2A16964
:108C500042EA0121A16161781144617006E00528B2
:108C600004D261788A4204BF06212170401CA060B2
:108C700008E0D4E9050101F03DFA002804BF012015
:108C8000A0702570002070BD10B5434C13F0070F85
:108C900007D003F00700042804BF207806281FD05F
:108CA00028E0A068022807D2616942EA01216161D7
:108CB00061781144617010E0B0F5817F08D23C49C1
:108CC0000968014401F8022C61781144617004E0E4
:108CD00001BF61788A4206212170401CA06009E032
:108CE0003449606901F028FA002804BF0120A0700F
:108CF00000202070002010BD03F0070CBCF1010F14
:108D000000D0C1E72449002048614870886008709D
:108D1000704730B403F007050024DFF87CC0012D54
:108D200007D013F0070F0DD0022D4FD0042D67D0C0
:108D300082E0CCF81440CCF81840CCF808408CF80D
:108D4000004079E0DCF8080002280BD2DCF81410AF
:108D500042EA0121CCF814109CF8011011448CF85F
:108D600001102CE004282AD2DCF81810032842EA6B
:108D70000121CCF818109CF801301A448CF801201D
:108D80001DD106228CF80020DCF81420114308BF06
:108D90004FF4307110E00000040501101C050110B3
:108DA00000AA0200F8050110D0AC011000AF0200CB
:108DB000CC3B01009022011008BFCCF818102849C4
:108DC000401CCCF82810CCF8080035E0DCF808206E
:108DD000042A28BF10460AD2C2F10303DCF8285047
:108DE000DB0025FA03F30370501CCCF808000428BC
:108DF00003D10120CCF80840087030BC0120704736
:108E00009CF80000062815D1DCF8140000220102AD
:108E1000DCF8180003021046B2EB930F06D251F8AB
:108E2000045B401C2A44B0EB930FF8D3CCF8282005
:108E30008CF80040CCF8084030BC002070474FF45C
:108E40002F300168880A424211EB822218BF401C71
:108E5000404201EB8000C01C20F00300704700007E
:108E6000EFBEADDEF84800220270427082700271DF
:108E70004271C270DFF8D4C3114601EB41030020F8
:108E80000CEB43031A54401C0628FBD3491C202931
:108E9000F3D3704708F046BC2DE9F04115460E4665
:108EA0000746FAF79DF800F008040820FAF793F84F
:108EB0002A463146384608F035FC05462046FAF782
:108EC00085F82846BDE8F081DF4880787047DE48A5
:108ED00040787047DC49002048707047DA49082024
:108EE0008871704770B50026F8F753FE044610F0FD
:108EF0000F052DD02846F8F74FFE012D17D0FBF7B0
:108F00002DFF44EA0064002322460321072003F0DA
:108F100069FF14F0060F1BD00126FBF719FF04466A
:108F200004F070FB022C18BF052C09D010E0FBF7F1
:108F30000FFFC5498A79904218BF8871DFD1E8E7F1
:108F4000022805D0022C4FF0020003D001F024F9D2
:108F5000304670BD04F0F7FBFAE72DE9F84F002723
:108F6000FAF7AFFCFBF7F4FE022804D101F03DFD57
:108F7000002818BF0127FFF7B5FF002818BF0127F9
:108F8000DFF8C49299F80200002800F08882D9F82E
:108F900008006D464FF0FF34002640B1D9F8082094
:108FA00000230121084603F01DFFC9F80860FAF705
:108FB00017F800F0080A0820FAF70DF899F80300EE
:108FC000DFF888B200B399F8050000EB4001401CBF
:108FD000C0B20BEB410189F80500202828BF89F8B1
:108FE000056099F80300401E89F803004C7891F859
:108FF00000800020002C05DD0A1892782A54401CBD
:109000008442F9DC0E704E705046F9F7DFFF002CF9
:10901000C0F2358208F0FF0000242B2880F0EC819C
:10902000DFE800F0CF38F21F2A3B1648F14FCF8C13
:1090300092D0F097B1B7EFEEEDECEBCFCFCFF8E9F0
:10904000E8E7E6CFE5E4E3CFE2CFE1E0CFCFDF0032
:109050009DF80000AC280CBF01200220FBF73CFF6C
:1090600018E09DF800100120FBF787FE012089F829
:109070000100044600F0C0B99DF80310009861F3A8
:109080001F6002F0F5F801210320FBF776FE0120B6
:1090900089F80100012400F0AFB9BDF8000040BA22
:1090A00004F093FA02210320FBF767FE012089F800
:1090B0000100EFE79DF801109DF80000FBF75DFE51
:1090C000E8E74FF0010A89F801A099F8000088BB91
:1090D000F8F754FD70B39DF8005089F800A0FBF735
:1090E00037FE012808BF002515F0040F18BFFDF753
:1090F000EFF815F0020F07D0FF210F20FCF7A1FCBD
:10910000FBF70FF945F0010515F0010F10D0FBF743
:109110001FFE022802D104F075FA48B1FBF718FED1
:10912000052802D101F043F810B10020FBF7E8F860
:1091300089F8006089F8016000F05EB99DF80000D0
:10914000401E01F089FAA5E79DF8000004F01EFB1F
:10915000A0E79DF8000010F00F0F0BD0012001F0E8
:10916000B3FC9DF80000102100F00F0001F083FC1B
:1091700000F042B9002001F0A7FC9DF8000000219A
:1091800000F00F00F2E79DF8000001F0A3FC00F0F2
:1091900033B99DF8000018B1012809D000F02CB9AE
:1091A000002008F0C4FA002006F064FB002006E06E
:1091B000012008F0BCFA032006F05CFB012006F059
:1091C0007CFB19E19DF80000F8B1FBF7C1FD022816
:1091D00018BF012404F0BFFA01460220FBF7CDFDC1
:1091E0000AE105E1FDE0F7E0D8E0DCE0C9E07FE07E
:1091F00038E032E02CE01CE00CE0A8E099E092E0DE
:1092000079E06AE040E051E0C4E000210620FBF78D
:10921000B4FD3FE79DF80000002818BF012004F0CE
:1092200083FA9DF80000002818BF012000F0AAFF73
:10923000E2E0002000F0A6FF00210520FBF79DFDE5
:10924000012001F006F8D7E03C0501109023011041
:109250009DF8000004F054FACEE0BDF8000004F0E0
:10926000EFFA17E79DF8000020B101283FD002284F
:1092700005D0C1E04FF42F30F9F7AAFABCE001F0B5
:10928000A1FD00210420C2E7F9F7AAFE00F00804BE
:109290000820F9F7A0FE99F80300002808BF89F814
:1092A00002602046F9F792FE0121AFE79DF8000029
:1092B000012804BF02210520A9D0022804BF0021F3
:1092C0000320A4D0032804BF002104209FD0042839
:1092D0001CBF0221084698D099E79DF80300009A28
:1092E000002360F31F626221072003F07BFD83E00F
:1092F000FBF7F6F9CEE69DF800009DF8011000019D
:1093000040EA111005F021F89DF801109DF80200C7
:1093100001F00F0140EA012005F01DF89DF803005F
:1093200005F025F82AE0BDF8000040BA05F001F884
:1093300062E09DF8000005F032F89DF8010005F0AC
:1093400038F8BDF8020040BA05F03DF854E09DF849
:10935000000005F04DF89DF801009DF80210000195
:1093600040EA111005F054F89DF802109DF8030032
:1093700001F00F0140EA012005F040F805F07EF809
:109380003AE09DF8000008F0BEF99DF800000028C2
:109390007FF480AE0020FAF7ECFE7BE69DF800003B
:1093A00004F0DFFA76E608F0A4F99DF8004004F036
:1093B000B2FA012C0AD0022C08BF40F0805005D030
:1093C000042C14BF082C40F0005001D104F017FA0F
:1093D000204608F0B1F95DE69DF8000008F0B1F90B
:1093E0000AE09DF8000008F0B1F904F041F903E04B
:1093F0009DF8000000F05CF90CB101273FE0D9F8BE
:1094000008006D464FF0FF3440B1D9F80820002322
:109410000121084603F0E6FCC9F80860F9F7E0FD11
:1094200000F0080A0820F9F7D6FD99F8030000B308
:1094300099F8050000EB4001401CC0B20BEB410164
:1094400089F80500202828BF89F8056099F80300ED
:10945000401E89F803004C7891F800800020002C11
:1094600005DD0A1892782A54401C8442F9DC0E70FB
:109470004E705046F9F7AAFD002CBFF6CBADF9F7B8
:10948000AFFD00F008040820F9F7A5FD99F80310D6
:10949000002908BF89F802602046F9F797FD002FE0
:1094A00014BF01200020BDE8F88F00000246002014
:1094B000022928BF704752B1012A18BF704701EB3B
:1094C000810000EBC100FE4901EBC0007047C1EB19
:1094D000C100FC4900EB400001EB8010704770B503
:1094E000F9F77EFD00F008060820F9F774FDF64C48
:1094F00000256078FF2806D24FF42861F14808F073
:1095000067F8A570E570A079FF2805D2D021EC4856
:1095100008F05EF8E57125723046BDE87040F9F755
:1095200055BD00FB01F3B3F5287F88BF7047E64BBC
:109530009A61C3E904017047DFF88CC30028DCF8A6
:10954000103018BF0360E0480029406918BF086068
:10955000002A1CBFDCF81810116058437047DA4825
:10956000012101710078D74980F00100C0EBC000F3
:1095700000EB400001EB80107047D3488278002157
:1095800032B1C27822B9027882F001020270817091
:1095900001717047CC491E284A78487008BF0020E6
:1095A00003D01F2808BF012000D108701046704763
:1095B000C5480078C34980F00100C0EBC00000EB53
:1095C000400001EB80107047F0B4BF4E96F800C029
:1095D000BC4CCCEBCC0C35690CEB4C0C04EB8C1C70
:1095E00003FB05F40CEB440C8D4234BF2C460C46B7
:1095F0007669F31A934238BF1A460026002A9CBFA8
:10960000F0BC70470023002C06D930F813702CF8FA
:1096100013705B1C9C42F8D8761C0CEB450C00EBDD
:1096200041009642EED3F0BC70472DE9F041A64FC1
:1096300014468C4601467A7806981D468A4218BF21
:10964000BDE8F0810121F970012802D0022825D05F
:109650002AE038789B49C0EBC0003E6900EB40002F
:1096600001EB8011A64234BF324622467869A842F7
:1096700038BF05460023002D16D90020002A06D940
:109680001CF8007021F81070401C8242F8D85B1C56
:1096900001EB4601A444AB42EFD305E000232A4688
:1096A00021466046FFF790FFBDE8F04100F079BB2E
:1096B000854A012811469072497808BF242004D0B9
:1096C000002806BF2429FF207047507070477E484D
:1096D000807A70472DE9F04F7B4B8AB01B78DFF81A
:1096E000E4C1C3EBC30303EB43030CEB8315930803
:1096F0008C08A2EB920C05945208ACF1010C00937B
:10970000CDE901C24A08CDE90642A1EB9102521E01
:1097100008920992CDE9033C00239E460DF1140AFC
:10972000E94625F813E059F82320A2F1010C02F1D3
:109730000108E04524BF5AF823707E1C13D37A1E1B
:1097400096420CD30CFB012435F913B030F91440C8
:109750005C45C8BF25F81340521C9642F2D20CF16A
:10976000010CE045EBD25B1C052BDAD30AB0BDE857
:10977000F08F002808BF70475349544B4A7854492A
:109780001B78002A097818BF022A05D0042A18BFBE
:10979000092A01D0012217E74E4A1278012A84BF14
:1097A0004D4A1378012200F016BB2DE9F04F464CCC
:1097B00083B00121E17049496278464D0F784349F1
:1097C000454E122A91F800A02CD00CDC042A1AD0A5
:1097D00004DC002A18BF022A0DD114E0092A12D095
:1097E000112A1FD007E0132A1CD0212A18BF222AD1
:1097F0007AD0242A79D0002878D0002352463946DE
:10980000FFF7E2FEA9E02978012903D9344996F847
:1098100000A00F78002869D000235246394600F096
:10982000DAFA9AE0F8F798F8F7F7F2FF00900028D4
:1098300018BFF8F72BFA2878012888BF96F800A0FF
:10984000F8F7A4F910F0040F18BF0AF1010A25482F
:1098500001906078A0F1110920781A49C0EBC0008E
:1098600000EB400001EB80152069B84238BF074685
:109870006069504538BF8246F8F745FA83460020B4
:10988000F8F703FD0026BAF1000F4CDD0024002F8D
:10989000C4BF019800EB86183EDD1BF904002028A8
:1098A00024BF002025F8140033D200EBD0714910FA
:1098B000C00758F82110C00E21FA00F081B216E05E
:1098C000D02E01105024011048050110C8040110C9
:1098D000CE040110C9040110CB040110C70401100B
:1098E000CA040110004000302AE031E035E04FF0BA
:1098F000FF30B9F1000F1CD0B9F1010F08BFC8B299
:1099000005D0B9F1020F04BF0846F8F7C4FC25F8EA
:109910001400641CBC42C0DBFE48761C564500693E
:1099200005EB4005B2DB0098002818BFF8F7B1F945
:1099300013E011F4005FC1F3042018BF4042E6E7D2
:1099400058B100230AF102023946FFF73DFE04E058
:1099500018B152463946FFF7BDFE03B0BDE8F04FDF
:1099600000F01FBAEB4801214172407980F00100FC
:1099700000EB800101EBC000E74901EBC00070473C
:10998000E448C279002132B1027A22B9427982F0E8
:1099900001024271C17141727047DE491E288A7905
:1099A000887108BF002003D01F2808BF012000D104
:1099B000487110467047D748407980F0010000EBAD
:1099C000800101EBC000D44901EBC00070472DE9D4
:1099D000F04FD24985B0012291F80080D04991F82A
:1099E0000090CC490A728979CB4C11291CBF1229ED
:1099F000132936D0F8B1C749497901EB810202EB4E
:109A0000C10104EBC102002119EB080C18BFC54CC1
:109A100011D02368B9F1000F5B8A03BF30F81150F1
:109A20000B4422F8135030F8113018BF22F81130CF
:109A3000491C8C45EDD8F9F7D3FA00F00805082049
:109A4000F9F7C9FAB34C607A002818BF01217CD01D
:109A5000E1712846F9F7BAFA0020207205B0BDE896
:109A6000F08FF7F779FFF7F7D3FE0190002818BFC2
:109A7000F8F70CF9A7488179A1F11105C1690091A6
:109A8000407900EB800101EBC00004EBC006F7F762
:109A9000FDF8A54FA5494FF0110A002804BF8B46D9
:109AA000012004D0BB4650460F464FF0010AF8F79C
:109AB000ECFBF8F726F900240390B9F1000F29D93F
:109AC00000988001029003980057202824BF0020AE
:109AD00026F814001BD200EBD0720299521001EB51
:109AE0008201C00751F80B10C00E21FA00F081B2BC
:109AF0004FF0FF30002D48D0012D08BFC8B204D070
:109B0000022D04BF0846F8F7C6FB26F81400641CB3
:109B10004C45D8D306EB49065046F8F7B6FBF8F7A4
:109B2000F2F800248246B8F1000F28D90098A34625
:109B30004FEA80191AF90400202828BF26F814B02B
:109B40001AD200EBD071491000E02CE009EB810142
:109B5000C007C959C00E21FA00F081B24FF0FF30A2
:109B6000D5B1012D08BFC8B204D0022D04BF0846EC
:109B7000F8F791FB26F81400641C4445DAD30198E9
:109B8000002818BFF8F785F855E711F4005FC1F316
:109B9000042018BF4042B8E711F4005FC1F304206D
:109BA00018BF4042E6E7607980F001006071002153
:109BB0004EE770B50D4657490122CA705C4A497894
:109BC00016785C4A212914781EBF2229232970BDEA
:109BD000002818BF002D11D0002322463146FFF780
:109BE000F3FC631C012221462846FFF7EDFC05EB40
:109BF0004400A31C01223146FFF7E6FCBDE870409B
:109C000000F0CFB870B5434D0446687890B9E0686D
:109C100068B149490978012994BF464947490B78F9
:109C200047490122097800F0D6F8687810B9A06891
:109C3000FFF7BBFD6878112804BF0020FFF7B5FDD2
:109C40006878122804BF0020FFF7AFFD687813285A
:109C500004BF0020FFF7A9FD206920B1A9790029E0
:109C600008BFFFF7B4FEA879112804BF0020FFF752
:109C7000AEFEA879122804BF0020FFF7A8FEA8793D
:109C8000132818BF70BD0020BDE870409FE62DE985
:109C9000F74F804626480D46002690F800A025483C
:109CA0001C49344690F80090BAFBF5F000FB09F728
:109CB0000120C870C87A0978DFF888B0884211D0CE
:109CC000144AC0EBC00000EB40000BEB8011107891
:109CD0004FF4A862C0EBC00000EB40000BEB80101B
:109CE00007F080FC0298002888BFDFF828B048D928
:109CF0009BF80CC00022BCFBF9F009FB10C101FB72
:109D00000AF100FB0510002D2DD938F814309BF80E
:109D1000001019E048050110D02E0110CC040110EC
:109D2000CD040110F8050110C04800304048003053
:109D3000C7040110C8040110C9040110CB040110AC
:109D4000CE04011050240110C1EBC10101EB410E02
:109D50004449641C01EB8E1100EB020E521C21F8E9
:109D60001E309542D1D80CF10100C0B28BF80C0026
:109D7000B84224BF00208BF80C00761C0298864263
:109D8000B6D33949087B401EC0B2087387429CBFD6
:109D9000781E08730878C87203B0BDE8F04FAFF3BF
:109DA000008070B5F9F71CF900F008060820F9F7F3
:109DB00012F92D4C20790025002801BF207880F071
:109DC00001002070A5701CBF0120A0703046F9F77B
:109DD000FDF8E57070BD2DE9F047994616460D4631
:109DE0000446F7F795FF5FEA000C1DD01E4908787E
:109DF0001C4AC0EBC000D1F8108000EB400002EB21
:109E0000801009FB08F200EB4200454594BF2F4645
:109E100047464969A1EB0901B14238BF0E4600210E
:109E2000002E09D8BDE8F0874B4632462946204629
:109E3000BDE8F047FFF7C8BB0023002F08D91CF985
:109E4000032034F8122020F813205B1C9F42F6D820
:109E5000491C00EB480004EB4504B142ECD3BDE8DB
:109E6000F0870000502401104805011068490028BF
:109E700014BF002001200870704765480078002852
:109E80000CBF0120002070476148017879B14FF084
:109E900040214A6942F001024A618A6912F0010FC9
:109EA00005D00A6B5B4B22F440521A430A6300212F
:109EB00041608160C160016170475548017879B1A6
:109EC0004FF040214A6942F001024A618A6912F06A
:109ED000010F05D00A6B4F4B22F440521A430A631C
:109EE000002141608160C1600161704770B5044626
:109EF000F9F776F800F008050820F9F76CF8444AFD
:109F000045490023D06801EBC001401CD060B0F58A
:109F1000807F28BFD3602078087060784870A07870
:109F20008870E078C8702079087160794871A079EC
:109F30008871E079C8711069B0F5807F3CBF401C22
:109F4000106116D31D200870012048702078887099
:109F50006078C870A0780871E078487120798871BD
:109F60006079C8719068401C9060B0F5807F28BF10
:109F70009360506840F001005060107888B14FF055
:109F80004020416921F001014161016B11F4405F02
:109F900007D0016B21F4405141F4BE0141F0204152
:109FA00001632846F9F712F8012070BD00B5017869
:109FB000427883B0890141EA82018DF8001041881E
:109FC00009098DF80110818809098DF8021081783E
:109FD00001F00F02017962F31F118DF80310017A6D
:109FE0008DF80410417A8DF805108179C27901F05D
:109FF0003F0102F00C0241EA02118DF80610C0790F
:10A0000080018DF807006846FFF770FF03B000BDC0
:10A010006805011000205FA0A02F0110002818BFC4
:10A020002D482E49886370472C48806B2A49884206
:10A030000CBF01200020704728487047284B4FF084
:10A04000000C1D681B1F1C68244B19605A602549B1
:10A05000D963DD6215F0804F22D0210C5985210A89
:10A0600083F8291083F82840598D19B15A8D0121A0
:10A0700041EA024C93F8291039B193F829100222D1
:10A0800042EA014C18490968196393F8281039B15C
:10A0900093F82810032242EA014C144909685963D5
:10A0A0004FF04021C1F878C08269CA67B0E8341027
:10A0B0009A60DC601D61C3F814C090E815109861C7
:10A0C000DA611C62C3F824C0986B034A904204BF53
:10A0D00007480867FEE70000504D554400DF0110B7
:10A0E0002CED00E0544C414638ED00E034ED00E04A
:10A0F000AD2007B070B50E460446FAF729FE0428D5
:10A1000011D1A4F51C7050280DD2A019A0F2712015
:10A11000502808D225020024002E04D92846F8F73A
:10A1200057FB012801D0002070BD641C05F5807527
:10A13000B442F3D3012070BD70B50D460446FAF762
:10A1400007FE04280AD1A4F51C70502806D220026C
:10A150002946F8F7DFFB012808BF70BD002070BD5D
:10A1600010B5074CFEF7F9FE012808BF10BD2068A6
:10A1700000F0F0FE002818BFFAF742FEF2E70000F8
:10A18000F8050110CD4A0028516814BF41F00100C4
:10A1900021F0010050607047C84B59680A0E120741
:10A1A00021F07F4142EA0060084358607047C3488D
:10A1B0004068C0F303607047C0484068000F7047B4
:10A1C000BE4840697047BD49012048617047BB499E
:10A1D0000020486170472DE9F041AEB0002707F03C
:10A1E000BAFA0646A02102A807F0F2F90024254693
:10A1F0004FF00308305D10F0800F18D0601C8DF810
:10A20000A9008DF8AF508DF8A880ADF8AC508DF84E
:10A21000B050ADF8AA508DF8AE508DF8B1508DF811
:10A22000B450355501272AA902A8F6F759F9601C40
:10A23000C4B20A2CDED3012F06D1102302AA0621B4
:10A240000120009506F052F807F08AFA2EB0BDE81A
:10A25000F0819A49FF220A70886170479748007818
:10A2600070472DE9F04FDFF8588287B0D8F800002A
:10A27000B0F90E11B0F90C0107F0F5F9F6F7F8F99D
:10A280000120F9F776FF07F070FAD8F800008B4F3D
:10A29000D0F8F800C0F30344C0F30321C0F3033542
:10A2A0008C420DD10F2D0BD003F09AFA20B107F09C
:10A2B00020FA082818BF2C46B86AA04218BFBC6212
:10A2C0002046F9F720FFFAF743FD05284CD1DFF8C7
:10A2D000F4B14FF000094FF0402A7868C7F80890B1
:10A2E000C7F80C90C0F30365C7F81090D8F80000C9
:10A2F000A900D0F8F80020FA01F101F00F04C0F332
:10A300000321C0F303368C420DD10F2E0BD003F086
:10A3100067FA20B107F0EDF9082818BF3446B86A8B
:10A32000A04218BFBC622946052002F0E9FD002DBD
:10A330007ED0022D1FD0042D7BD078680A2D4FEAE5
:10A34000106120F07F404FEA017118BF41F00071A9
:10A3500008437860FEF701FE012805D007F000FAF7
:10A36000FAF7F6FC0528B8D0F9F702FF07B0BDE808
:10A37000F04F07F0FFB90D212046FAF744FE002800
:10A38000E8D007F0FCF907F0FFF9F9F780FE0400C8
:10A3900065D1F6F7D0FE4C48F7F783FA0120F7F7BE
:10A3A00075FAF8F73FFE4948F8F7F1FEF8F7D8FEDE
:10A3B000F8F701FFD8F800104000B1F80621B0FB13
:10A3C000F2F0401CC0F34F00788091F808117970CA
:10A3D00059B1F8F7F0FED8F800104000B1F80411B8
:10A3E000B0FBF1F0401CC0F34F00F8F755FE3848C1
:10A3F000CAF81800F7F7B0FAF7F715FC787838B113
:10A40000401E10F0FF00787004BF7888F8F744FE13
:10A410007868C0F3036529460520F5F75CFFFEF771
:10A420009CFD012809D07868C0F30360A84201E0D0
:10A430003BE03EE008BF002C18D0CAF818B0F8F78F
:10A4400063FEF8F798FE0020F8F7A1FEF8F7F3FD99
:10A45000F7F782FAF7F7DEF90020F7F722FA07F0AC
:10A4600093F907F096F9FAF71BFF73E76846F7F7D9
:10A4700098FD70B16846FFF7C5FB0198F9F7A0FA9F
:10A48000684607F08BF90446F7F7D3FDFAF7D9FCD5
:10A49000C5E7D8F80000406E10F0704F02D0FAF710
:10A4A000AFFCBCE7FAF7D4FCB9E7204607F07BF92C
:10A4B00050E7204603F03CFB4CE700007C05011010
:10A4C000F805011000005FA0C79C00103597001030
:10A4D00007005FA07047002808BF70478022014630
:10A4E000014807F070B87047A0370110704708287E
:10A4F0003CBFFE49087070470020FC4988604860F6
:10A50000FB48006890F88100082838BF0870704741
:10A510000020F64948607047F4480078704770B5ED
:10A52000F34D0024286890F86C0010F0020F0BD057
:10A53000FAF70EFC022807D1EC482968007801EBF5
:10A540008000B0F8840084B2204670BD70B5E84D3C
:10A550004FF48054286890F86C0010F0020F0DD072
:10A56000FAF7F6FB022809D1E0482968007801EBE8
:10A570008000D0F88400000CC0F31304204670BDA6
:10A58000DA488078002818BF012070472DE9F04193
:10A59000FAF7DEFB022803D103F034F8022803D0D7
:10A5A0004FF48050BDE8F0814FF480552E4603F003
:10A5B000EAF8CF4F0446DFF83483386890F86C101F
:10A5C00011F0010F0ED0B0F87600D8F80810404214
:10A5D000814207DC34B10020641EC8F80800204620
:10A5E00003F0D4F8396891F86C0010F0040F18BF2C
:10A5F000002C0AD0B1F87C00621E9040B1F87E2099
:10A60000824238BF1046C0F31306D1F8A40010F000
:10A61000020F1CBF98F80210002902D0000CC0F3F2
:10A620001305B54298BF354607F0C2F810F4817F94
:10A630000FD0FAF7C6FC01463868B0F85800C0F3EE
:10A64000033081421CBF4FF40050B5F5005F38BFA6
:10A6500005462846BDE8F0812DE9F04FDFF890A2CD
:10A6600087B0DAF8001091F86C2012F0020F0DD0CC
:10A670009E4A91F88090DFF87CB21778002809DBB9
:10A68000484503D2B84218BF064643D107B0002060
:10A69000BDE8F08F3E464FF0FF38F7F7BBF8F7F70D
:10A6A0005AFE0025B9F1000F34D9DAF80000002471
:10A6B00000EB8500B0F8840081B22046F6F759FD22
:10A6C000F7F7B1FA6846F7F76CFC002866D00298F5
:10A6D00078B1014688489BF8002000785043421E1C
:10A6E00007D331F9020B0028B8BF40420444521E80
:10A6F000F7D2F7F79EFCF7F78DF800232246922158
:10A70000072002F06FFBA04584BF2E46A0466D1CBB
:10A710004D45CAD3B74244D0082E3CBF73490E7092
:10A72000DAF80000B0F8821039B300EB870200EBD2
:10A730008600B2F88420B0F8840092B280B2801A09
:10A74000484340F30F34F9F78BF96C4B9BF800202A
:10A75000002193F800C002FB0CF2002A0DD930F85A
:10A760001120224420F811209BF8002093F800C00B
:10A77000491C02FB0CF28A42F1D84FF4800003F02E
:10A78000F9F8DAF80000002300EB86008021B0F829
:10A79000840082B2072002F025FB09E0FAF730FBC3
:10A7A00090E702F0F0FF03283CBF401C02F0EEFFF0
:10A7B000012007B0BDE8F08F4D484C490068B0F863
:10A7C0007600424288688242BCBF401E8860704763
:10A7D0002DE9F04F91B093460E4604464FF0000A23
:10A7E00002F0D1FFDFF80881404F0500D14610D1BB
:10A7F00006F0E3FFD8F80010B1F87810884208D3CB
:10A800000120C7F8089002F0C1FF11B00120BDE897
:10A81000F08F002E1FDDB8680028B8BFC7F8089079
:10A8200007DBD8F80010B1F874108842BCBF401C98
:10A83000B860D8F80000B968B0F87400884215DC38
:10A84000032D13D2681CC7F8089002F09FFF11B0C7
:10A850000120BDE8F08F09D1D8F80000B0F87600EB
:10A860004142B8688842C4BF401EB860B87850B151
:10A87000D8F8000090F8A40010F0040F1EBF0020CC
:10A8800011B0BDE8F08FD8F80000B0F972108C421A
:10A890000EDD796821447960B0F86E00884210DCE2
:10A8A0004FF0FF30C7F80490FFF7D6FE824608E06D
:10A8B0007868002805DD002CD4BF01212146401A0C
:10A8C0007860DFF83C9099F8000007283AD10D48ED
:10A8D000594600784200684606F084FEADF8004014
:10A8E000ADF80260ADF8045038890DE0D8050110CC
:10A8F000F8050110C7040110CB040110C8040110B1
:10A9000049050110CE040110ADF80600B888ADF875
:10A910000800D8F80000B0F87210ADF80A10B0F8CE
:10A920007410ADF80C10B0F86E10ADF80E10B0F851
:10A930007600ADF8100099F80000072804BF6846BB
:10A94000FEF717FF504611B0BDE8F08F3D4810B537
:10A950000068D0F8A40010F4807F06D0C0F3033064
:10A96000012101FA00F0F8F7A8F8374900204870F3
:10A97000887010BD70B5344D0024A878002814BF2D
:10A9800001260026687828B902F00CFF002808BFCD
:10A99000002100D001218E4225D00A1C18BF0122BF
:10A9A000AA7028480068D0F8A43013F0040F0ED025
:10A9B00021B1C3F30310082808D206E00021A960E2
:10A9C000696090F88100082800D22870012413F0F3
:10A9D000020F18BF0124002A18BF01220023822180
:10A9E000072002F0FFF9204670BD164900200968D3
:10A9F000D1F8A41011F4807F08BF7047DFF848C079
:10AA00009CF80120131C18BF012330B40F4CC1F374
:10AA10000332E46B012505FA02F2224011F4007FB3
:10AA200001D00AB102E00AB1002100E001218B420D
:10AA300004BF30BC7047081C18BF01208CF801000F
:10AA400030BC97E7F8050110D80501100010004050
:10AA5000AB48C079704710F5167FA8BF704701203A
:10AA6000A749C8717047A6490020C8717047A4481B
:10AA700090F90100704770B5A14E04460D4696F955
:10AA80000100A04218D0FAF763F902280FD1B4F1FF
:10AA9000FF3F0CD0357096F90100B0F1FF3F06D0B2
:10AAA00044EA052200236421072002F09BF9747018
:10AAB000002C04BF0020F071FAF74AF905281CBFEA
:10AAC000B4F1FF3FB47070BD8D49C87070478C48B9
:10AAD000C0787047024600F00F0011210228A8BF7D
:10AAE0007047874B1209002818715A7108BF00215E
:10AAF000C1E783484079704781480079704710B5B5
:10AB00000446F9F70FFF01467D4A2046012982BF1E
:10AB10000021917110BD9179142905D8491CC9B241
:10AB20009171142938BF10BD002010BD70B50C46BE
:10AB3000054606F047FE00214FF0140C0DB300222D
:10AB4000401E00281DDD35F91230002BB8BF5B42D6
:10AB50009BB2634511D90221B3EBCC0F88BF032010
:10AB600009D8B3EB8C0F88BF022004D8B3EB4C0F8D
:10AB70008CBF01200020207003E0521CD2B2824220
:10AB8000E1DB084670BD2DE9FF4F81B0924680465B
:10AB9000CCB200270E9D06F01AFE009006F01CFEB7
:10ABA000DFF85C910646BB4699F90100B0F1FF3F22
:10ABB00004BF99F80200012808D1FAF7C9F805285E
:10ABC00004D002240127CAF800B069E054EA050065
:10ABD00006D0002C64D096F8E804012860D14DE03E
:10ABE000307B80B196F8420000281CBF0224274623
:10ABF000F1D196F8E804012819BF96F8EA04012873
:10AC000002240327E7D05D46D8F8148006F0DAFD69
:10AC1000002414220146B8F1000F20D000204B1E62
:10AC2000002B1CDD38F910100029B8BF494289B249
:10AC3000914210D90224B1EBC20F88BF03250ED870
:10AC4000B1EB820F88BF022509D8B1EB420F8CBF50
:10AC500001255D4603E0401CC0B29842E2DB002CB7
:10AC600018BF45F0A007B6D1DAF800002C2817D29B
:10AC7000307B002818BF022412D0ACE7F9F752FE4F
:10AC8000012888BF89F806B00AD899F80600142868
:10AC900005D8401CC0B289F80600142800D300244F
:10ACA00099F80300012804BF002C02240098007DBD
:10ACB000012808BF002406F094FD012808D104985B
:10ACC000022441F28831884202D906F08FFD002427
:10ACD00099F80500012808D07CB139460120FFF71A
:10ACE000CAFE05B02046BDE8F08F99F8040010F0C8
:10ACF000FF0F14BF02240024EFD100210846EEE725
:10AD0000E40501107F4880494FF0000C426810684C
:10AD1000884204BF5068B0F5087F03D19068B0F551
:10AD2000485F01D90020704770B47849D5688D42DA
:10AD30001FD0002413462146B4EB900F07D253F8DE
:10AD4000046B491C7440B1EB900FF8D374B9116ACD
:10AD500079B10021B1EB900F06D252F8043B491CA7
:10AD60009C44B1EB900FF8D3654502D070BC002035
:10AD7000704770BC01207047624800787047614896
:10AD8000406800F5407070475E48406800F580708C
:10AD9000704710B55B4C4FF41C306060FFF7B2FF9A
:10ADA00070B1606800F5807000F0D4F840B1606860
:10ADB00000F5407000F0DDF810B10120207010BDEA
:10ADC000002010BD4F49002008704FF41C30F7F7E9
:10ADD000FFBC4C48017841B140684B4A0168914240
:10ADE00002BF4168B1F5087F704700207047454BAE
:10ADF0005B6803F580731844F7F7E9BD414B5B6866
:10AE000003F540731844F7F7E2BD3E484068006917
:10AE100070473C4949680A6982429CBF00207047DC
:10AE2000C0EBC00001EBC00000F580607047354A00
:10AE3000526802EB80035B6A1A44354B53F820C01A
:10AE4000403333F810000CEB0003401E5B1E23EA76
:10AE5000000000FB012070472A498860704729489C
:10AE6000806870472DE9F00F264B0022DFF8A080A4
:10AE7000D3E90145012708F140069146831893F96B
:10AE800028C0BCF1000F18DB07FA02F32B4214D0E4
:10AE9000D3B204EB830A58F823B036F81330DAF84B
:10AEA00024A09B445B1EABF1010BA2442BEA0303DD
:10AEB00003FB0CA341F8223001E041F82290521C20
:10AEC000102ADBD3BDE8F00F70470029B8BF7047E8
:10AED00030B494460B4A0F4C526802EB80035B6A15
:10AEE00013440B4A52F8202034F810001418401E66
:10AEF000641E24EA000001FB003030BC6146F7F715
:10AF000066BD0000EC05011054465053EFBEADDEA7
:10AF1000D03B0100103C010010B5FFF73AFFA8B18B
:10AF2000FFF72DFF0146D022174806F04CFBFFF734
:10AF30002BFF164C01464FF4E272206806F043FBEB
:10AF40002068406DBDE8104002F0A8BB0220F9F770
:10AF5000C3FFE2E758B10E4A0168914207D1406849
:10AF600020F00F00B0F5107F04BF012070470020D3
:10AF7000704730B1006820F00F00702804BF012036
:10AF80007047002070470000D0AC0110F805011098
:10AF900041505352AD4810B5806810F0020F15D0E3
:10AFA000F6F736FC90B1F6F7F6FB0402F9F7D0FE9F
:10AFB00044EA0044F9F7D2FE44EA00604EF2AF01E1
:10AFC00008434FF04021C867012010BD002010BD8C
:10AFD00010B572B60120F7F7FBFAF8F7A7F9F8F702
:10AFE000D1F94FF0FF30F7F7F6FF994880234FF47F
:10AFF0000052002152F821C040F821C0491CB1EB99
:10B00000930FF7D3F7F7F9FFF8F720FCF8F742FCB6
:10B010009048F8F75BFC0120F8F719FCF7F76AFB9A
:10B020001E20F8F709FCF8F7C9F9F7F751FDF8F712
:10B03000C5FBF8F713FAF7F7F1FFF7F7C1FDF6F7DD
:10B04000FCFBFFF769FFF7F770FFF7F73BFFFDF732
:10B0500009FFFBF7DFF9FEF730FF62B6F9F7C9FF2A
:10B060007D4C206890F8640000F00F00F7F7D4F9E9
:10B070002068018BC1F30722418A008AFEF751FA4A
:10B080002068806E000C01F0AAFE744806F0B3FB45
:10B090002068B0F90C0106F0B3FBF5F702F9FFF7F1
:10B0A00025FAF8F72FFCFAF734F9FFF713FA06F050
:10B0B000ACFB206890F8200010F0010F04BF0021C5
:10B0C000032003D002F047FB01460220F9F755FEAA
:10B0D0004FF040242069002300F07002194602203E
:10B0E00001F080FE206910F0200F17D0226F00239E
:10B0F0000521072001F076FE626F0023052107205D
:10B1000001F070FEA26F00230521072001F06AFE06
:10B11000E26F00230521072001F064FEFFF716FC13
:10B120000020206710BD02244D4DFDF716FF0128B9
:10B1300006D0F9F70DFE032802D101F00EFF58B337
:10B14000002D05DC02F007FB01460220F9F715FE91
:10B15000DFF814914FF00108424FDFF810A14FF0D3
:10B160004026A9F1030BF9F7F3FD0546F9F7F6FDC3
:10B170000146284601F0C4FEF9F7F0FD01462846D5
:10B18000F5F7A9F8FDF7AAFE072D5BD2DFE805F079
:10B190005A1D08272A192D006D1E002DC5DCD1E788
:10B1A000387850B9FBF74DF838B900231A462021FA
:10B1B000072001F017FE87F8008002F057FF0224F5
:10B1C000D1E7FFF74EF80524CDE7FAF7A1FEF9F72E
:10B1D000BFFD012804BF2046F9F7CCFDC3E702F00C
:10B1E000A4F9C0E7FEF7BCFFBDE7C6F81890F7F773
:10B1F00019FFF7F7B5FFF7F7DEFF4000AAFB0010D5
:10B200004009401C4008F7F747FFFDF7A6FE01285C
:10B210000CD1F9F79DFD062808D0F7F775FFF7F771
:10B22000AAFFF7F708FFC6F818B09CE7F9F793FDF7
:10B230000546F9F706FE15B1F9F70AFEE5E7F9F755
:10B24000DFFDE2E70220F9F747FE8CE700800040CF
:10B250000070011045CF0000F8050110D0AC0110BE
:10B26000FF700200FC05011003005FA0CDCCCCCC28
:10B27000FE4908607047FE4808210068428A008A3B
:10B2800002FB00107047401E022884BF0020704758
:10B290000822F74909684B8A098A03FB01214843C0
:10B2A00000F5003000F5224070472DE9F043ADF283
:10B2B0000C4D05460124F9F748FD8446401E02283E
:10B2C00082BF00200DF20C4DBDE8F08395F821906F
:10B2D00095F8208005F150066046FFF7D4FFE54A57
:10B2E000002730B10168914204BF4068CDE90010E9
:10B2F00001D0CDE90027B5F92600B5F9241009FBE6
:10B3000008F5084400EBD07042100021002D88BFE2
:10B310006B4614D936F91100801A7F28C8BF7F20E8
:10B3200005DC10F1800FB8BF6FF07F0000DA002459
:10B3300003EB0108491C88F808008D42EAD88DF813
:10B3400004409DF80500FF283CBF401C8DF8050017
:10B35000ADF806206C466046FFF795FF68B1C4491A
:10B3600008230A68518A128A01FB02322146F7F744
:10B370002EFB01280CBF0127002738460DF20C4D8B
:10B38000BDE8F083B94948607047B84810B44068D8
:10B39000002808BF4FF42C30B74A016891421CD1F5
:10B3A0004168B1F5007F18D3836800228446B3F565
:10B3B000056F88BF4FF405630021B1EB930F24BFE5
:10B3C00010BC70475CF82140491C2244B1EB930F3C
:10B3D000F8D3002A04BF10BC7047002010BC70478F
:10B3E00070B505460020E860D5F808C001212C465C
:10B3F0000346BCF5056F88BF4FF4056C0022B2EB25
:10B400009C0F06D254F82200521C0344B2EB9C0F4E
:10B41000F8D35842E8609548007810F0800F0AD1C0
:10B420002046FFF742FF4FF42C304FF405622946C7
:10B43000F7F7CDFA014601290CBF0120002070BDAD
:10B44000FF2270B50025044605614FF400615030BD
:10B4500006F0DCF8A584E584E562A56265632563F2
:10B46000E563A56365642564E5640120A56470BD9A
:10B470002DE9F0414FF42C3104467F4E0868B0426C
:10B4800018D14868B0F5007F14D38A6800230D46B0
:10B49000B2F5056F94BF94464FF4056C0020B0EBF5
:10B4A0009C0F26D255F82070401C3B44B0EB9C0FFB
:10B4B000F8D3F3B1FF224FF40561204606F0A6F859
:10B4C0004FF40870C4E900604FF40560A0600020EC
:10B4D000E06084F8200084F8210084F8220084F8D9
:10B4E000230020616061A061E0612046FFF7A8FFB2
:10B4F00007E0B2F5056F88BF4FF40562204606F0FD
:10B5000062F80120BDE8F08170B402684FF4087160
:10B510005160016801F1500291F821C091F820308A
:10B520000CFB03F102EB41010022BCF1000F08D932
:10B5300000EB4204521CB4F8EA4021F8024B944557
:10B54000F6D80022002B08D900EB4204521CB4F8B4
:10B550002A4121F8024B9342F6D80022BCF1000F99
:10B5600008D900EB4204521CB4F8644021F8024BA5
:10B570009445F6D80022002B08D900EB4204521C57
:10B58000B4F8A44021F8024B9342F6D8B0F8E62074
:10B5900021F8022BB0F8E82021F8022BB0F8E420C3
:10B5A00021F8022B00240022BCF1000F88BF00EB21
:10B5B000841508D905EB4206521CB6F86A6121F8D9
:10B5C000026B9445F6D80022002B88BF00EB84154F
:10B5D00008D905EB4206521CB6F86A6221F8026BE4
:10B5E0009342F6D8641C042CDDD370BC70472DE95F
:10B5F000F74F88B000250A992C462E460968049119
:10B6000001F150030999002984BF1949D1F800803C
:10B610001CD90022002888BFB8F9CE700DD933F9A3
:10B62000021B0029B4BFC1F1000C8C46BC45BCBF55
:10B630000D44641C521C8242F1D30999761C8E423F
:10B64000E7D3002CC8BF95FBF4FA08DC4908414356
:10B6500001EB5002049901EB4201B1F950A0002125
:10B660000291019104995031009107E00006011008
:10B67000F80501104654525953454C460021039198
:10B68000099900296DD9009E4FF00109FE490696DF
:10B690004FF0000B09685F46D846B1F9C0E0D1F819
:10B6A000B410CDF814B0C1F307410791002829D98F
:10B6B000B6F900204FF0000C069993446346002829
:10B6C0000DD9B1F90040A51A48BF151B7545B8BF83
:10B6D0000CF1010C01EB49015B1C8342F1D307998A
:10B6E0008C4503D305997F1C1144059108F101088D
:10B6F00006EB49068045DBD3002FC4BF059991FBBB
:10B70000F7F101DC9BFBF0F1039B0A9A09B202EB13
:10B710004302A2F86410DC4A1268B2F9BA30AAEB0C
:10B72000030399420ADDB2F9B82052448A4205DD8A
:10B73000019A114401910299491C02910099099AB8
:10B7400001EB400100910399491C039191429AD366
:10B750000299002905DDDDE9011291FBF2F1019169
:10B7600002E05146CDF804A00A9AA2F8E6100021A2
:10B770000291039104995031009100210491002815
:10B7800068D9C149009F069709684FF0000B099ED0
:10B79000B1F9BCE0D1F8B410D846090ED946CDF8BD
:10B7A00014B00791002E2BD9B7F900204FF0000CF0
:10B7B000069993446346002E0DD9B1F90040A51AAD
:10B7C00048BF151B7545B8BF0CF1010C01EB4001DA
:10B7D0005B1CB342F1D307998C4504D3059908F15A
:10B7E00001081144059109F1010907EB4007B14532
:10B7F000DAD3B8F1000FC4BF059991FBF8F101DC71
:10B800009BFBF6F1049B0A9A09B202EB4302A2F8F1
:10B81000A4109D4A1268B2F9BA30AAEB0303994208
:10B820000ADDB2F9B82052448A4205DD039A114478
:10B8300003910299491C02910099891C0091049975
:10B84000491C049181429CD302980028C4BF0399EB
:10B8500091FBF0FA0A98A0F8E8A001980A995044E0
:10B8600000B200EBD0704010A1F8E4000BB0BDE8CE
:10B87000F08F2DE9F04F146889B015460E46074643
:10B88000A1F12008202928BF4FF0FF3A05D24FF040
:10B89000010000FA06F0A0F1010A38BF4FF0000BDA
:10B8A00005D34FF0010000FA08F0A0F1010B202FA2
:10B8B0003DBF0120B840401E4FF0FF3038BF00228E
:10B8C00007D3A7F120024FF0010101FA02F1A1F123
:10B8D0000102C6F12009202E34BF20FA09F100FA36
:10B8E00008F1B2401143B040CDE90001206920F4D5
:10B8F000FE6020616548007810F0010F7ED02A4676
:10B900003146384601F04EF90020A8616861002FE9
:10B9100084BFDFF874E101221BD905EB4001B1F9C6
:10B92000A4100029B8BF494209B2DEF80030B3F9CB
:10B93000CC308B420ADD410905EB810100F01F0C80
:10B940004B6902FA0CFC43EA0C034B61401CB84201
:10B95000E3D30020012F18BFA7F1010E3BD005EB68
:10B960004001B1F9A630B1F9A420991A48BFD11A03
:10B9700009B2DFF814C1DCF800C0BCF9C4C08C45C2
:10B9800026DAB5F9E810B2EB010C48BFA1EB020CC6
:10B990000FFA8CFC5A1A48BFCA1A11B28C450BDB3D
:10B9A000420905EB820100F01F0C01224B6902FAEB
:10B9B0000CF21A434A610BE0411C4B0905EB830270
:10B9C00001F01F0C0121536901FA0CF11943516177
:10B9D000401C7045C3D36969E869B14008432063DE
:10B9E000A969286AB140014361636869202E34BFA8
:10B9F00020FA09F000FA08F0084300E000E0606374
:10BA000022480068079010F0040F00F0BD8100206C
:10BA10002863E862002E88BFDFF86CE01BD9DEF8EF
:10BA2000002005EB4001B1F96A11B2F9D8308B4220
:10BA300003DCB2F9DA208A420ADA420905EB820114
:10BA400000F01F0C0122CB6A02FA0CF21A43CA6200
:10BA5000401CB042E3D30020A8626862002F88BF78
:10BA6000DFF824E021D9DEF8002005EB4001B1F930
:10BA70006A12B2F9D8308B4203DCB2F9DA208A427A
:10BA800010DA420904E00000F80501100006011078
:10BA900005EB820100F01F0C01224B6A02FA0CF246
:10BAA0001A434A62401CB842DDD300202864E86390
:10BAB000002E88BFDFF8D8E71BD9DEF8002005EBA1
:10BAC0004001B1F9AA11B2F9DC308B4203DCB2F9C2
:10BAD000DE208A420ADA420905EB820100F01F0CDF
:10BAE0000122CB6B02FA0CF21A43CA63401CB0422B
:10BAF000E3D30020A8636863002F88BFDFF890E7D6
:10BB00001BD9DEF8002005EB4001B1F9AA12B2F909
:10BB1000DC308B4203DCB2F9DE208A420ADA4209C9
:10BB200005EB820100F01F0C01224B6B02FA0CF2B4
:10BB30001A434A63401CB842E3D300202865E864F6
:10BB4000A8646864002E88BFDFF844E71CD9DEF8DB
:10BB5000003005EB4001B1F9EA11B3F9E0208A4267
:10BB600003DCB3F9E2208A420BDA410905EB810CD0
:10BB700000F01F030121DCF84C2099401143CCF860
:10BB80004C10401CB042E2D30020002F88BFDFF8E9
:10BB900000E71BD9DEF8002005EB4001B1F9EA12FD
:10BBA000B2F9E0308B4203DCB2F9E2208A420ADAD1
:10BBB000420905EB820100F01F0C01224B6C02FAD6
:10BBC0000CF21A434A64401CB842E3D3696AE86A3B
:10BBD000B14040EA010EC4F838E0A96A286BB140D0
:10BBE0000843E063696A202E34BF21FA09F101FAA3
:10BBF00008F141EA0000E0630590696BE86B01FA27
:10BC000006F140EA01022264A96B286C01FA06F1F0
:10BC100040EA01006064696B34BF21FA09F101FA5E
:10BC200008F141EA000161646B6CE86C03FA06F309
:10BC300040EA0300A0640490AB6C286D03FA06F39D
:10BC400040EA0300E0646B6C34BF23FA09F303FAA3
:10BC500008F343EA0000E0640290059832EA0E051A
:10BC600021EA000C4EEA05022564069240EA0C0027
:10BC7000C4F844C006EB0701039008BFBCF1000FF5
:10BC800042D000231A461846002988BF01273BD915
:10BC90004FEA501804EB880800F01F09D8F84080DC
:10BCA00007FA09F918EA090F03D0864294BF521C1B
:10BCB0005B1C401C8142EBD8012B0FD105EA0A0026
:10BCC00040EA0E00A06305980CEA0B031843E063FA
:10BCD00025EA0A0020642CEA0B006064012A13D1D3
:10BCE000226C0098A36B10401843A063606C019B0A
:10BCF000D4F83CC0034043EA0C03E363009B9A433F
:10BD00002264019A90436064069A049830EA020221
:10BD1000A264069840EA020CDDE9020320EA03006F
:10BD2000E064039B43EA000508BF002821D00023FC
:10BD30001A461846002988BF012717D94FEA50181C
:10BD400004EB880800F01F09D8F8488007FA09F9C1
:10BD500018EA090F03D0864294BF521C5B1C401C9A
:10BD60008142EBD8002B18BF002A02D10020A0642A
:10BD7000E064079810F0010F06D0206B20EA0C0059
:10BD80002063606BA8436063206B0099084203D175
:10BD9000626B01990A4203D0216941F010012161CF
:10BDA00010EA0A0F04BF606B10EA0B0F03D0206982
:10BDB00040F020002061A06B0099084203D1E26BA3
:10BDC00001990A4203D0216941F04001216110EA42
:10BDD0000A0F04BFE06B10EA0B0F03D0206940F09C
:10BDE00080002061206C0099084203D1626C0199A7
:10BDF0000A4203D0216941F48071216110EA0A0FDF
:10BE000004BF606C10EA0B0F03D0206940F400708F
:10BE10002061A06C002804BFE06C002803D02069DA
:10BE200040F48060206109B00120BDE8F08F2DE969
:10BE3000F04FB9B016460D460446F5F7EBFCF4F7A3
:10BE400025FF01004FF011001DBF0290012003905B
:10BE5000012108BFCDE90210CDE93454F5F751FFB7
:10BE60000022002D88BF04A904D9835C8B54521C86
:10BE70009542FAD8F5F747FF0021002C88BF04AAA5
:10BE800007D9435C02EB010C491C8CF820308C4232
:10BE9000F7D8F5F77BFE3890FE48007810F0200FB9
:10BEA0005FD0F4F7F3FEFC49FC4A00280CBFCDE953
:10BEB0000021CDE9001206F1EA003690403000255D
:10BEC000EA460DF1D8090DF1D00B379002A85BF8C6
:10BED000257050F82500F6F7D8F90024002F84BF0C
:10BEE00004A800EB45181AD918F90400202828BF27
:10BEF00000200DD25AF8251000EBD072521051F8E4
:10BF00002210C007C00E21FA00F080B2F6F7C3F984
:10BF100059F8251021F81400641CBC42E4D36D1CB0
:10BF2000022DD3D3DE4805781D2D1AD100210A46F3
:10BF300014AB5BF822400020002C88BF59F822C0C7
:10BF400007D93CF8107023F81170401C491C84423A
:10BF5000F7D8521C022AECD31D2D04BF1846FDF75A
:10BF600036FDCC4D287810F00C0F00F0AA82F4F7C3
:10BF70008DFECC49CC4A00280CBFCDE91421CDE977
:10BF80001412CA48F5F7D0FC0120F5F7E3F82C901D
:10BF90000120F5F72DF92B900120F5F7B5FB239043
:10BFA0000298F5F74EF924900398F5F74AF917909F
:10BFB0000120F5F7C9F92A901120F5F7C5F9279066
:10BFC0000120F5F7EDF928901120F5F7E9F9259012
:10BFD00020A800901EAB1CAA1AA90298F5F7E7FA50
:10BFE00021A800901FAB1DAA1BA90398F5F7DFFA43
:10BFF0000298F5F758FB22900298F5F754FBA44CF1
:10C0000001902068B0F8E4100120F5F7B2F80021A3
:10C010000120F5F764FB206890F8E6100298F5F728
:10C020001FF9206890F8E6100398F5F719F9002138
:10C030000120F5F79FF900211120F5F79BF9002168
:10C040000120F5F7C3F900211120F5F7BFF92068A9
:10C05000B0F8E8100298F5F7D7FA2068B0F8E810C1
:10C060000398F5F7D1FA00210120F5F75FFB29903D
:10C070008848007810F0040F00F0268125462868D3
:10C08000B0F8EC10009190F8EB3090F8EA200B211A
:10C090000298F5F760FA2868B0F8EC10009190F873
:10C0A000EB3090F8EA200B210398F5F754FA0021C1
:10C0B0000120F5F73BFB2EACF5F7B5FDFCF74DFF86
:10C0C000012805D02046F5F76CFF002800F04681D6
:10C0D000F5F7A0FB3299002234AC002054F822304E
:10C0E000002B88BF06EB022C08D931F8027B0CEB41
:10C0F0004008401CA8F86A718342F6D8521C022AF4
:10C10000EBD30298F4F78EFB18900398F4F78AFBB0
:10C1100016900298F5F70BF926900398F5F707F9B2
:10C120005B4D19902868B0F8EE10009190F8EB3054
:10C1300090F8EA200B210298F5F70DFA2868B0F87C
:10C14000EE10009190F8EB3090F8EA200B21039864
:10C15000F5F701FA002500210120F5F7E7FA0021A3
:10C160000298F4F74AFB00210398F4F746FB0DF11F
:10C170000808012158F82500F4F73FFB34A80024F3
:10C1800050F8257014A8002F50F825A030D904A825
:10C1900000EB451906EB0528002119F804B0084604
:10C1A000F5F7D5FA012000FA0BF102A88B4650F8FA
:10C1B0002500F5F7AFF86FEA0B010920F5F7C7FA8C
:10C1C0000DF1B80BF5F72FFDFCF7C7FE012804D0E1
:10C1D0005846F5F7E6FE002859D0F5F71BFBBAF8EC
:10C1E000000008EB4401641CA1F8AA01BC42D3D3AF
:10C1F00000210846F5F7ABFA6D1C022DABD3189958
:10C200000298F4F7FAFA16990398F4F7F6FA2699D1
:10C210000298F5F77FF819990398F5F77BF81C4C0D
:10C220002068B0F8F010009190F8EB3090F8EA2018
:10C230000B210298F5F78FF92068B0F8F010009103
:10C2400090F8EB3090F8EA200B210398F5F783F98A
:10C2500001210846F5F76AFA2EACF5F7E4FCFCF785
:10C260007CFE012804D02046F5F79BFE00287BD0F9
:10C27000F5F7D0FA3299002234AC002054F822C0ED
:10C28000BCF1000F88BF06EB02231AD910E068E06A
:10C29000F805011000060110C04800304048003089
:10C2A0004E050110C00A00304008003001000E00A9
:10C2B00031F8025B03EB4007401CA7F8EA518445C4
:10C2C000E4D8521C022AD8D3FE48007810F0080F98
:10C2D0007ED0FD4D2868B0F8F210009190F8EB3058
:10C2E00090F8EA200B210298F5F735F92868B0F8A4
:10C2F000F210009190F8EB3090F8EA200B210398AF
:10C30000F5F729F900210A4634AF002057F821C07B
:10C31000BCF1000F88BF06EB012306D903EB4004F4
:10C32000401CA4F82A228445F8D8491C0229ECD3E1
:10C330002868002490F82401B4EB400F48DA2868FC
:10C3400090F82401A042D4BF012100210120F5F77B
:10C35000EDF92EAFF5F767FC09E005E0F8F750FDC1
:10C36000ACE6F8F74DFD2FE7F8F74AFD77E7FCF765
:10C37000F4FD012803D03846F5F713FE48B3F5F76E
:10C3800049FA32994FF000090DF1D00E00225EF803
:10C3900029701046002F05D931F91030401C1A447D
:10C3A0008742F9D8B2FBF7F2781E18BF06EB092ACC
:10C3B00038D031F9103001EB400C3CF9028CB3EB72
:10C3C000080348BF5B4231F91080B8EB020801E076
:10C3D00037E01CE031F910804CBFA2EB0808A8EB55
:10C3E00002083CF902BC3CF902CCBBEB020B4CBF8F
:10C3F000A2EB0C0CACEB020CE0450AEB400C09DDA7
:10C40000BCF92A824345C8BFACF82A3208E0F8F7E5
:10C41000F7FCACE7BCF928829845B8BFACF82832E5
:10C42000401EC6D109F1010901EB4701B9F1020F24
:10C43000ACD32868641C90F82401B4EB400FFFF6DD
:10C440007EAF01202C99F4F794FE01202B99F4F78C
:10C45000D8FE01202399F5F742F924990298F4F7C0
:10C46000FFFE17990398F4F7FBFE01202A99F4F7D1
:10C4700081FF11202799F4F77DFF01202899F4F717
:10C48000A5FF11202599F4F7A1FF209800901E9B8D
:10C490001C9A1A990298F5F75EF8219800901F9B54
:10C4A0001D9A1B990398F5F756F822990298F5F70B
:10C4B000ABF801990398F5F7A7F801202999F5F74A
:10C4C00035F93898F5F730FA39B0BDE8F08F2DE935
:10C4D000F04F7C4DADF5617D6C68F8F736FC0228B5
:10C4E0000FD10120FEF7CFFE00687849884208D0BE
:10C4F0000120F8F725FC2046FEF7D7FE0220F8F7CA
:10C500001FFCFF224FF45B71684605F07FF8009432
:10C51000288810F4804F1CBF2046FEF791FF6A4622
:10C52000009890F8203090F821C050300CFB03F1B7
:10C5300000EB41000021BCF1000F08D902EB4107DC
:10C5400030F8026B491CA7F8EA608C45F6D8002148
:10C55000002B08D902EB410730F8026B491CA7F801
:10C560002A618B42F6D80021BCF1000F08D902EBFA
:10C57000410730F8026B491CA7F864608C45F6D877
:10C580000021002B08D902EB410730F8026B491C4F
:10C59000A7F8A4608B42F6D830F8021BA2F8E61088
:10C5A00030F8021BA2F8E81030F8021BA2F8E410E1
:10C5B00000260021BCF1000F88BF02EB861708D9C6
:10C5C00007EB410930F8028B491CA9F86A818C45B8
:10C5D000F6D80021002B88BF02EB861708D907EB9D
:10C5E000410930F8028B491CA9F86A828B42F6D8BF
:10C5F000761C042EDDD361461846FEF7F8FF31485D
:10C600000127056815F4004F68D12F486E460027B2
:10C61000006890F8B40000F00F0800F0A4FC0128B6
:10C6200009D00F214046F8F7EEFC012812D0002077
:10C6300000F096FCA4E000210846F5F798F9F4F71D
:10C6400000FB50B12248D0F8B01241F48031C0F85C
:10C65000B01202E0012000F083FC1E4890F8009028
:10C660001D4890F800A0BAF1000F18BFB9F1000FF3
:10C670007ED00098002180F8209080F821A080F8DA
:10C68000221080F82310F5F73FFEF5F77FFA0746F2
:10C69000002015F0030F18BF4FF4817015F0200F24
:10C6A0001CBF40F20121084358B13840F5F73CF96E
:10C6B000FF210F20F9F7C5F9F5F7ACF83846F5F783
:10C6C00033F90CE000060110F805011046545259E8
:10C6D00000500040C7040110C804011050E015F0DC
:10C6E0002C0F04D0324651464846FFF7A0FB15F008
:10C6F000030F42D0DC960098DB9000F15006F5F76E
:10C7000002FB8346F5F786F80020F5F7BEFD00270B
:10C71000BAF1000F22D900254FEA871817E01BF95C
:10C720000500202812D200EBD071491008EB8101DE
:10C7300001F1405101F58041C0070968C00E21FA9E
:10C7400000F080B2F5F7A7FD26F8020B6D1C4D45F1
:10C7500038BF202DE3D37F1C5745DCD3FE4800783B
:10C760001D2803D1DB985030FDF71FF8514600E03B
:10C7700004E04846DC9AFEF73AFF0127F5F7C7F9CF
:10C7800094F82000DD9094F82100DE90002F1FBF68
:10C79000DD980028DE98002804BF0DF5617DBDE816
:10C7A000F08FEE480068DF9010F0020F00F0028179
:10C7B000009DDDE9DD2728696E4620F00F00286125
:10C7C00047F6FF706FEA0009DB90002005F1500882
:10C7D00004900390029082460190002F4DD90AFBED
:10C7E00002F04FF0010C38F9101000208B465B4628
:10C7F000DC90012A1BD90AFB02C038F910009842CC
:10C80000C8BF03468842B8BF0146B0EB0B0E48BF15
:10C81000ABEB000E0FFA8EFBDDF870E3F345C8BFFB
:10C82000CDF870B383460CF1010C9445E3D34B452E
:10C83000C8BF9946DB988142B8BFDB91581A48BF00
:10C84000C81A01B2C6480068B0F9C0308B4204DB98
:10C85000B0F9C210DC9888420BDD4FEA5A1006EBA3
:10C8600080000AF01F0C0121C36801FA0CF1194382
:10C87000C1600AF1010ABA45B1D34FF0000A002A9B
:10C880004BD938F91A00002183465B464FF0010C62
:10C89000DC91012F1BD90CFB02A138F91110994230
:10C8A000C8BF0B468142B8BF0846B1EB0B0E48BF6C
:10C8B000ABEB010E0FFA8EFBDDF870E3F345C8BF5A
:10C8C000CDF870B38B460CF1010CBC45E3D34B455E
:10C8D000C8BF9946DB998842B8BFDB90191A48BF98
:10C8E000C11A09B29E480068B0F9BC308B4204DB23
:10C8F000B0F9BE10DC9888420BDD4FEA5A1006EB07
:10C9000080000AF01F0C0121436801FA0CF1194361
:10C9100041600AF1010A9245B3D3F068002804BFD0
:10C920003069002803D0286940F008002861706849
:10C93000002804BFB068002803D0286940F0040034
:10C9400028617168F068B9400843A862B16830692D
:10C95000B9400143E9627068202F39BFC7F1200256
:10C96000D040A7F1200290400843E862DB98A884F9
:10C97000A5F82690B6F9E410B9EB010048BFA1EB89
:10C98000090077490968B1F9B820904203DD2869A8
:10C9900040F002002861B6F9E420DB98101A44BF89
:10C9A000DB98801AB1F9BA10884203DD286940F09B
:10C9B00001002861DF98694D10F0050F04D0DDE912
:10C9C000DD016A46FEF755FFD5F800A01AF0080F02
:10C9D0007CD0009ADDE9DD9311694FF0000B21F462
:10C9E000C05111616846CDF860B05946CDF85CB0D1
:10C9F000002B84BFDFF868E101261AD9DEF8007049
:10CA000000EB410CBCF92AC2B7F9267167450DDA73
:10CA10004FEA511C00EB8C0C01F01F08DCF85C7035
:10CA200006FA08F847EA0807CCF85C70491C9942F6
:10CA3000E4D3C0F858B00021C0F854B0B9F1000FE9
:10CA400084BF474E01271AD9D6F8008000EB410C6D
:10CA5000BCF92AC3B8F92681E0450DDA4FEA51182E
:10CA600000EB880C01F01F0BDCF8548007FA0BFB7D
:10CA700048EA0B08CCF85480491C4945E4D3916B33
:10CA8000D0F85CC041EA0C01D0F854C00CFA03FCA9
:10CA900041EA0C019163D16BD0F860C041EA0C010E
:10CAA000D0F858C00CFA03FC41EA0C0CC2F83CC0A8
:10CAB000416D202B39BFC3F12003D940203B994061
:10CAC00041EA0C01D163416D002900E011E004BF8F
:10CAD000816D002903D0116941F400611161C16DBC
:10CAE000002904BF006E002803D0106940F4805074
:10CAF00010611AF0400F0FD16069401C606120691D
:10CB0000002814BFE069A06900F1010014BFE061D2
:10CB1000A0616846FEF7F8FC00200346E060A068CC
:10CB20002146B0F5056F88BF4FF405600022B2EBD7
:10CB3000900F06D251F82260521C3344B2EB900F92
:10CB4000F8D35942E160287810F0800F11D12046C7
:10CB5000FEF7ABFB06E000004905011000060110DE
:10CB6000F80501104FF42C304FF405622146F5F71B
:10CB70002EFF41208DF86C03207C8DF86D03607CC6
:10CB80008DF86E03A07C8DF86F03E07C8DF8700348
:10CB900000230522DBA9072000F054F90DF5617D83
:10CBA000BDE8F08F2DE9F74F84B04FF00008C2F8D0
:10CBB0002080C2F81C80059B844E01274146002B33
:10CBC0001ED902EB4103B3F96430002BB8BF5B42BE
:10CBD0001BB2D6F800C0BCF9CCC09C450CDD4B099B
:10CBE00002EB830301F01F04D3F81CC007FA04F41E
:10CBF0004CEA040CC3F81CC0059B491C9942E0D3C5
:10CC00000021012B1CBF059BA3F1010940D002EBC1
:10CC10004103B3F96640B3F964C0B4EB0C0348BFF9
:10CC2000ACEB04031BB23568B5F9C6509D422CDA53
:10CC3000B2F9E630BCEB030548BFA3EB0C052DB2FF
:10CC4000B4EB030C48BFA3EB040C0FFA8CF39D422A
:10CC50000DDB4B0902EB830301F01F04D3F81CC06A
:10CC600007FA04F44CEA040CC3F81CC00DE04B1C9A
:10CC70004FEA531C02EB8C0C03F01F03DCF81C4042
:10CC800007FA03F32343CCF81C30491C4945BED3B3
:10CC9000316891F8CA30002B7DD091F8CB10146820
:10CCA0008B4288BF19460023DDF814C0BCF1000F89
:10CCB00084BF491C00916ED94FF0010EDDF800C011
:10CCC0004FF000090121CA46BCF1010F52D9DFF82B
:10CCD000FCC003FB0005DCF800C0CDF80CC0BCF9BB
:10CCE000CEC002950EFB0005019503FB001504EB79
:10CCF0004505B5F95080B8F1000FB4BFC8F1000583
:10CD00004546AC4536DB0EFB001504EB4505B5F991
:10CD10005070002FB4BF7D423D46AC452ADB029DDA
:10CD20006D1A04EB4505B5F94E60002EB4BF75428F
:10CD30003546AC451EDB019D6D1A04EB4505B5F982
:10CD40004E50002DB4BFC5F1000BAB46E34511DCDE
:10CD5000A7EB0808039FB7F9C8704745B8BF09F1AA
:10CD60000109AD1BBD42C8BF0AF1010A491C009D63
:10CD7000A942BAD3BAEB090148BFA9EB0A01DFF80F
:10CD80004CC0DCF800C09CF8CAC061450FDB5909F3
:10CD900002EB810100E015E003F01F064FF0010CEB
:10CDA000CD690CFA06FC45EA0C0CC1F81CC00599CB
:10CDB0005B1C8B4206D2002B18BFA3F1010E7FF43F
:10CDC0007DAF79E707B00120BDE8F08FF8050110CD
:10CDD00070474FF0FF3070475D48406870475C49CE
:10CDE0004860704710B582B007280BD14FEA111C7C
:10CDF000012404FA0CFC564C64681CEA040F04BFBE
:10CE000002B010BD9B0100F00F0043EA800040F02B
:10CE100001008DF800008DF801108DF80220100A35
:10CE20008DF80300100C8DF80400100E8DF805002D
:10CE300000208DF806008DF80700684604F0BEFB60
:10CE400002B010BD10B582B007280DD191F800C016
:10CE500001244FEA1C1C04FA0CFC3D4C64681CEADB
:10CE6000040F04BF02B010BD9B0100F00F0043EAA5
:10CE7000800040F001008DF80000072A88BF0722DB
:10CE800000206B46002A09D911F800C01C18401C6C
:10CE900084F801C09042F7D3072805D200211A1860
:10CEA000401C51700728FAD3184604F087FB02B0E3
:10CEB00010BD10B59B0100F00F0082B043EA800066
:10CEC00040F002008DF80000072A88BF07220020EA
:10CED0006B46002A09D911F800C01C18401C84F8C0
:10CEE00001C09042F7D3072805D200211A18401C30
:10CEF00051700728FAD3184604F060FB02B010BD49
:10CF000070B5134E40EA012502283488224618BF26
:10CF1000052803D1002918BF022900D12C46A242BE
:10CF200009D051B17088002344EA004290210720C3
:10CF3000FFF758FF3480758070BDF6F73CF944EA7E
:10CF40000042002390210720FFF74CFFF2E700008A
:10CF500008060110FE4908707047FD4800787047C8
:10CF6000FB4948707047FA48407870472DE9F04F08
:10CF7000F848F74CADF6640D00686178836D0229BE
:10CF8000C3F303201CD0626812F4007F1EBFC3F3FA
:10CF900003310F29084612F0800F1EBFC3F303119F
:10CFA0000F29084602F0070141F40031F8F72BF889
:10CFB000012814BF00200220607040F0B0820DE014
:10CFC00000210846F4F7D3FCF3F73BFE30B1E2480A
:10CFD000D0F8B01241F48031C0F8B012F4F7D6FDA9
:10CFE000CDF85008207910F0100F18BFF5F76BF945
:10CFF000207910F0080F03D1FF210F20F8F721FD51
:10D00000D6480078CDF84808D5480078CDF84C08C7
:10D01000D4480778D4480078CDF82C08DDF84C08BF
:10D0200000281CBFDDF84808002813D004F0A7FB37
:10D0300004F0AAFB0020F7F7E4F80020F7F752F914
:10D04000C348007910F0100F0CD00120F7F758F901
:10D0500001200BE0DDF82C08002818BF002FE5D1D7
:10D0600000F05DBA0020F7F74BF90020F7F748F918
:10D07000F3F7E7FD10F0010F04BF0120F4F75BF8B0
:10D08000F4F798FD1E20FCF785FA00210846FCF70E
:10D090000DFA834601210020FCF708FADDF84C2840
:10D0A000DDF848188246002001FB02F9B9F1000FB3
:10D0B00084BF47F6FF72D14306D92BF810102AF827
:10D0C0001020401C8145F8D81E20FCF766FC00218A
:10D0D0000120FCF7EBF9054601210846FCF7E6F9CB
:10D0E0000446DDF82C1800207E181CBF47F6FF729E
:10D0F000D14306D025F8101024F81020401C864299
:10D10000F8D893484FF000084088002840F2468144
:10D11000DDF82C18701C491ECDF85C18DDF82C18B1
:10D1200040083944491ECDF85418CDF85808FBF78B
:10D1300014FF012800F032810DF50360F4F731FF90
:10D14000002800F02481DDF83408F6F739FCDDF81A
:10D15000380800284FD004F05DFB07467C48007972
:10D1600010F0100F0AD03846DDF8381804F057FBDD
:10D170000190B84208BFDDF8387810E000200023A5
:10D180000090019002901A461946DDF8380804F024
:10D190004BFB01906E48007910F0200F0BD1F6F791
:10D1A0005FFCDDF84C28009201463846DDF848382F
:10D1B000019A04F03EFB6648808810F4804F1EBF41
:10D1C00001980028F6F787FC002F1CBF0020B9F15A
:10D1D000000F10D937F910103BF910208A42B8BF60
:10D1E0002BF810103AF910208A42C8BF2AF8101004
:10D1F000401C8145EED8DDF8500810F0010F1CBF2F
:10D20000DDF8400800287DD004F00AFA07465048AF
:10D21000007910F0400F07D000231A461946DDF8B8
:10D22000400804F00BFB0DE0F6F7E3FB022200924E
:10D2300001463846DDF85838DDF8402804F0F9FAA0
:10D24000DDF840084249898811F4005F1CBF0028BE
:10D25000F6F7D9FB002F55D03D48426812F4806F95
:10D2600033D0DDF82C180020012911D007EB400144
:10D2700037F910C0B1F90230B3EB0C0148BFACEB89
:10D28000030127F81010DDF85C18401C8842EDD32C
:10D290004FF0000C27F810C0DDF85418401C8842ED
:10D2A00011D207EB400137F91030B1F902E0BEEBC3
:10D2B000030148BFA3EB0E0127F81010DDF8541846
:10D2C000401C8142EDD827F810C00020002E10D954
:10D2D00037F9101035F910308B42B8BF25F810100F
:10D2E00034F910308B42C8BF24F81010401C86421D
:10D2F000EED812F4806F45D01C4A08F10100A2FB61
:10D30000003100E03EE08908494201EB8101C14261
:10D3100038D1A2FB08108008A2FB0021090949426C
:10D3200001EB810100EB810000EB800101EBC0010A
:10D3300003A800EBC1010020002E84BF47F6FF7C4C
:10D340006FEA0C021ED935F8103034F810700FE077
:10D3500010060110F805011000500040C70401102C
:10D36000C8040110CC040110CD040110CDCCCCCCEC
:10D37000DB1B21F8103025F8102024F810C0401CC9
:10D380008642E0D8F4F755FE08F1010801E0F7F70E
:10D3900037FD8F4840888045FFF4C9AEF4F73AFA6C
:10D3A00004F0F2F904F0F5F9894F7888804576D3D6
:10D3B000DDF8500810F0020F28D000224FF6FF735E
:10D3C0001046B9F1000F0ED93BF910103AF910C010
:10D3D000A1EB0C019142C8BF0A469942B8BF0B4667
:10D3E000401C8145F0D842208DF80000100A8DF8CD
:10D3F00001008DF80220180A8DF803008DF8043022
:10D400000023052269460720FFF71CFDDDF85008C0
:10D4100010F0010F7DD0B88810F4806F51D06D48A6
:10D42000A0FB08108308142B88BF14234FF00008BA
:10D4300047464146002E84BF0DF10C0BA3F1020EAE
:10D4400053D94FF0000CDFF8909147F6FF7A62460F
:10D45000002B11D902EB820000EBC2000BEBC000E5
:10D4600030F9110084444845C8BF81465045B8BFD3
:10D470008246521C9A42EDD3002B04BF002025F8AF
:10D4800011000DD09CFBF3F025F81100022B07D9F9
:10D49000ACEB0900A0EB0A0090FBFEF001E038E0E5
:10D4A000002024F8110035F91100B842C8BF074622
:10D4B00034F911004045C8BF8046491C8E42C0D88F
:10D4C00013E000274FF6FF783846002E0DD935F9C6
:10D4D000101034F91020891AB942C8BF0F464145CF
:10D4E000B8BF8846401C8642F1D843208DF8000022
:10D4F000380A8DF801008DF802704FEA18208DF877
:10D5000003008DF804800023052269460720FFF7F9
:10D5100099FCFF20FCF73EF8FF20FCF73EFAF4F7F9
:10D52000F6FA0DF6640DBDE8F08F10B5ADF5056D9A
:10D530004FF0FF30FDF790FC254C00206070F4F7B1
:10D54000DAFBFF224FF40561684604F05FF8684695
:10D55000FDF78EFF6846FDF715FFFBF7FEFC01287F
:10D5600003D1F7F7F5FB03281BD1207810F0010F4A
:10D5700007D0FEF7ACFF207820F001002070FBF709
:10D58000A9FC207810F0020F07D0FFF7EFFC2078FD
:10D5900020F002002070FBF79DFCF7F7D9FB032871
:10D5A00008D00020FDF7EEFE0120F4F7A4FB0DF5F6
:10D5B000056D10BDF7F724FCCFE705494860002052
:10D5C000487070470248406870470149488070477A
:10D5D00010060110CDCCCCCC0080FFFFFD490870B7
:10D5E0007047FC4800787047FA49C8717047F9489D
:10D5F000C0797047F748C069B0F5B47F2CBF0120EF
:10D6000000207047F34840787047F249002280B10B
:10D61000012818BF7047487802280CD0042818BF8A
:10D62000C86906D0B0F5B47F84BF4FF4B470C86148
:10D630007047CA617047C869401CC861F2E7E64894
:10D6400000787047E348C07910F0010F18BF7047A9
:10D6500010B50020E0490870F7F754FCBDE8104011
:10D660000020F6F739BEDC488088C0F30020704700
:10D67000D94910B589880020C1F3002151B104F0C7
:10D6800033F864280FBF4FF0C040012101FA00F0C9
:10D6900040F08040BDE8104004F0D5B8CE4A10B547
:10D6A00081B25160CB4AC0F30743C0F303605361BA
:10D6B000507090700020C1F30021906151B104F0CE
:10D6C00013F864280FBF4FF0C040012101FA00F0A9
:10D6D00040F08040BDE8104004F0B5B8BD48407946
:10D6E0007047BD4A0028516814BF41F0020021F084
:10D6F000020050607047B8480079C0F3400070479E
:10D70000B54A10F0010F506814BF40F0020020F03D
:10D71000020050607047B04900200979C1F3400110
:10D72000002918BF012070470028AB4A516814BF78
:10D7300041F0010021F0010050607047A6480079D7
:10D7400000F001007047A3494A788A70487070471A
:10D75000A04880787047A1480068406DC0F303601E
:10D760007047012181409B484269114041617047E7
:10D77000012181409748426922EA010141617047D5
:10D78000944840697047934880697047914910B543
:10D790008C6988610246002381210720FFF722FB64
:10D7A000204610BD8C488088C0F38020704789488F
:10D7B0008079704788480079C0F3800070478648B8
:10D7C0000079C0F3C000704783488088C0F34020D0
:10D7D000704781480079C0F3C0107047FCF7D0BE95
:10D7E0007D488088C0F3403070477B488088C0F314
:10D7F000C020704778488088C0F300307047764A70
:10D8000010F0805F516814BF41F4806121F48061A1
:10D8100010F0005F14BF41F4005021F4005050603C
:10D82000FDF7A8B86C484168002011F4806F18BF5C
:10D830004FF0805011F4005F18BF40F00050704767
:10D8400070B56549044610F0040F4D68284614BFB2
:10D8500040F4807020F4807014F0080F14BF40F47E
:10D86000007020F4007014F0100F14BF40F400603A
:10D8700020F4006014F0400F14BF40F4805020F4F6
:10D88000805014F0200F14BF40F0800020F0800082
:10D8900048600021C0F3002050B103F025FF642848
:10D8A0000FBF4FF0C041012101FA00F040F080416C
:10D8B000084603F0C8FFC4F38000C5F30021884286
:10D8C00019D003F075FF06460120F6F752FC16F05A
:10D8D000020F04D0022001F0CDFF002009E016F471
:10D8E000807018BF012001F0C5FF3D4890F86C0022
:10D8F000C00803F0C7FEC4F3C000C5F3402188424E
:10D9000008BF70BD0120F6F734FC04F00800BDE844
:10D91000704001F05FBF30484168002011F0040FF3
:10D9200018BF012011F0080F18BF40F0020011F4D9
:10D93000807F18BF40F0040011F4007F18BF40F052
:10D94000080011F4006F18BF40F0100011F4805F60
:10D9500018BF40F0400011F0800F18BF40F02000C9
:10D9600070471C49087370471A48007B7047194874
:10D97000806A704717490A6A10430862704770B599
:10D98000144E306A40F0007400203062124845683E
:10D9900015F0040F18BF44F0010415F0080F18BF6C
:10D9A00044F0020415F4807F18BF44F0040415F419
:10D9B000007F18BF44F00804FCF7E2FD002818BF00
:10D9C00044F0805415F4006F18BF44F0100415F0B3
:10D9D000800F07E01806011064AF0110F805011070
:10D9E000D0AC011018BF44F0200415F4805F18BFBC
:10D9F00044F0400415F4005F18BF44F00054B169CE
:10DA000044EA0140002918BF40F0806070BDFE4923
:10DA100048627047FC4890F8240000F0010070470D
:10DA2000F94890F82400C0F340007047F64890F899
:10DA30002400C0F380007047002818BF0120F2497D
:10DA40008872704770B5002486B02646F7F780F9D3
:10DA5000EE49052808680CBF90F8F80090F85800C7
:10DA600000F00F052846FDF7D4F9002818BF406ADA
:10DA700010F0010F14BF0220042040F400312846AA
:10DA8000F7F7C1FA002804BF06B070BD0120F3F714
:10DA900052FBF4F7C8F8FBF760FA01283BD0684660
:10DAA000F4F77FFA002832D06846FCF7ABF801980B
:10DAB000F5F786FF0298B8B10146D54803F0C8FED5
:10DAC000D34A904209D0D34AD34B014612781B78EF
:10DAD00052005A43CE4803F085FDD04800784928CB
:10DAE00004BFCB48FBF761FE049848B1CC48CD4950
:10DAF0000078097808444200CB48049903F072FD8D
:10DB0000C14901208872F4F794FA012603E0F7F77F
:10DB100077F9002CBFD0F3F77DFEF7F7C1FB06B015
:10DB2000304670BDB848807A002818BF0120704781
:10DB30002DE9F04F4FF0000A87B005460F24D1467B
:10DB4000F7F706F90746F7F709F9DFF8BCB20690D0
:10DB5000052F07D1FCF734FB002804BF00208BF809
:10DB60000A0002D09BF80A0058B9F7F73FFA0646B8
:10DB70004FF48050F7F737FAFFF764FF3046F7F7B6
:10DB800032FA052F0CBFDFF8A482DFF8A482214609
:10DB90002846F7F738FA002804BF07B0BDE8F08F31
:10DBA00003F0EDFD03F0F0FDF6F771FA04007CD10F
:10DBB0000125F3F746F806460020F3F7BCFA28469D
:10DBC000F4F711F890484563F5F7F8FAA5F1010B61
:10DBD000FBF7C3F901280AD0F7F7BAF8B84206D123
:10DBE000F7F7BCF80699884208BF002C12D0F3F76B
:10DBF00011FE90488088C0F3402000281CBF0120FF
:10DC000001F0E8FD804F16F0010F7D7834D0012C33
:10DC100027D031E06846F4F7C4F9F8B116F0010FE7
:10DC200003D00120F5F712FD82466846FBF7EAFFB4
:10DC30000198F5F7C5FE6846C0470446F4F7F9F9C0
:10DC4000002CC5D115B901985845C1D1F3F7E0FDB5
:10DC5000002804BF2846F3F7C6FFB9E7F7F7C5F871
:10DC6000B6E70120F5F7F2FC504505D2AAEB00011A
:10DC70000120F5F7FBFC8146F5F7C5FA16F0010F18
:10DC800029D0012C27D1B9F1000F24D0F3F79CF94A
:10DC90000446F2F7F2FF00EB800004EB400048443A
:10DCA000002144F20902904200E014E084BFA0F594
:10DCB00080400938002D08BF43F6390103D0022DFA
:10DCC00008BF41F6F901884205D2091A0120F5F78B
:10DCD000FCFC0120787203F05CFDF7F7E1FA07B075
:10DCE000BDE8F08F2DE9F14F88B04FF000094948A9
:10DCF000CDF80C90CDF80890CDF81890CDF8149090
:10DD0000CDF8109004784448DFF810B1C846067882
:10DD10009BF800004F4604FB06FA462804BF08980B
:10DD2000FBF743FD0898089900EB4A0003F090FDCB
:10DD300001909BF800004B2804BF0198FBF735FDCC
:10DD40000898234600EB8A05009631492846019A37
:10DD500003F06FFD9BF80000492804BF2C48FBF737
:10DD600024FD2E4800784C2804BF2846FBF71DFDF3
:10DD700005EB4A039B464FF0000C002E22D90020F1
:10DD8000611E13D005EB410E35F811203EF802EC70
:10DD9000A2EB0E0212B2002AB8BF524212B223F80E
:10DDA00011208242C8BF1046491EEBD1188005EBF6
:10DDB000440503EB44034045C8BF80460CF1010C09
:10DDC000B445DCD31048B0F90E0000908045A4BFE4
:10DDD0004FF00109CDF80C900BEB4A034FF0000C0B
:10DDE000002E3ED90021601E02282BD90BEB4002E9
:10DDF0003BF8105032F802EC32F8042C75442A44F7
:10DE000012B223F8102017E018060110F8050110CF
:10DE100080700110C7040110C804011049050110E9
:10DE2000CD040110CC04011080760110AD950010D6
:10DE3000AF99001064AF01108A42C8BF1146401E5E
:10DE40000228D3D800201980588098800BEB440B0F
:10DE500003EB4403B942C8BF0F460CF1010CB445B3
:10DE6000C0D3F64BB3F910209742A4BF4FF001097D
:10DE7000CDF80890B9F1000F14BFD86B186C00F101
:10DE8000010014BFD8631864ED480078FF2842D021
:10DE900008990AEB8A00022521F81090DDF820C0CD
:10DEA00003990CEB40004180029981800599C18063
:10DEB00006990181D96B4FEAE17C01EB1C5C6FF3A1
:10DEC0000B0CA1EB0C014181196CCB1701EB135327
:10DED0006FF30B03C91A8181A0F80E8007820499A1
:10DEE000418200998182C28206EB86000899B9F1CD
:10DEF000000F00F10103224600950CBF4E204D207B
:10DF0000FBF793FB06EB8600431C22460095472057
:10DF10000899FBF78AFB09B04846BDE8F08FC9486D
:10DF200070472DE9F84F8346C448C9490025B0F928
:10DF30000E80C6480978C44C00782E46AA46471879
:10DF4000F3F724FE0090C348A4F16809007849283B
:10DF500004BF4846FBF73BFD0020002F09D93BF8E2
:10DF6000101039F81020891A24F81010401C87422C
:10DF7000F5D8DFF8E09299F800004C2804BF20465D
:10DF8000FBF725FD009810F4007FA7F1010012D0E7
:10DF900000281CBFA949B1F9103026D034F910105F
:10DFA0000029B4BF4A420A469A42BCBF0D44761CBF
:10DFB000401EF3D119E000281CBFA049B1F9103070
:10DFC00013D004EB400234F8101032F8022C891AF6
:10DFD00009B224F810100029B4BF4A420A469A42F6
:10DFE000BCBF0D44761C401EEBD1002EC8BF95FB74
:10DFF000F6F52EB2268099F800004F2804BF20467F
:10E00000FBF7E5FC0025781E0ED034F81010891BB4
:10E0100009B224F810100029B8BF494209B28D4254
:10E02000B8BF0D46401EF0D1258003F0C1FB10F4AF
:10E03000817F18BF4FF00508454506DD99F80000BF
:10E040004FF0010A4D2807D103E099F800004E284F
:10E0500002D12046FBF7BBFC99F80000472804BF1B
:10E060002046FBF7B4FC5046BDE8F88F2DE9F04F91
:10E0700087B0FCF741FA784C2068B0F93610B0F957
:10E08000340003F0F0FA0120F6F773F8DFF8ACA1E2
:10E090009AF8140010F0100F06D0042000F009F9CF
:10E0A0000F2818BFF6F72FF8FF208AF80800002184
:10E0B000481EFCF7E0FC03F0D0FBF6F749FE02280F
:10E0C00008BF4FF0000B73D19AF801606248CAF89C
:10E0D0002CB0CAF830B00068B100806D20FA01F1B0
:10E0E00001F00F04C0F30325C0F30319C0F3033894
:10E0F000C0F30357AC4220D10F2F05D003F058FBDB
:10E1000010F4817F18BF3C46AC420CD1B8F10F0F20
:10E1100009D052488088C0F3403020B103F0E9FABA
:10E12000082818BF4446AC4207D1B9F10F0F04D0FC
:10E13000F6F7FBFE002818BF4C4631460220FEF7DA
:10E14000DFFE052E58D2DFE806F0920303039600A7
:10E150000F219AF801602046F6F755FF00284BD0B2
:10E1600003F00DFB03F010FBF5F791FF05003DD127
:10E170009AF8000000281CBF0001F2F739FF0024C4
:10E18000F3F704FD0690F2F75CFD10F0010F10D0DC
:10E19000F2F7CBFF02280CD39AF8090048B1069891
:10E1A00040F40030F3F7C0FB0124F3F73CFD02E03C
:10E1B00071E0F3F7FFFC8AF809B08AF803B0F5F7CD
:10E1C000EEFFF6F756FCDFF898804FF0E027DFF817
:10E1D0009490FAF7C2FE012808D0F6F7B9FD02289C
:10E1E00002BF9AF80100B042002D06D003F0CCFA2D
:10E1F00003F0CFFAF7F754F840E06846F3F7D1FEA2
:10E20000D8B12CB1641E0698F3F78EFBF3F7D2FC5D
:10E210006846FBF7F7FC0198F5F7D2FB684603F078
:10E2200021FB054698F8000020B1B869C9F8000044
:10E23000C7F810B0F3F7FDFECBE715E018060110A4
:10E240004905011080760110E8760110CD04011017
:10E25000CC0401104E050110F805011064AF011047
:10E260002404011088040110F6F7CAFDB1E7204626
:10E2700003F099FA02E02046FFF75AFCFAF76DFE28
:10E28000012803D1F6F764FD022804D1F6F760FDFA
:10E2900002283FF419AF03F063FAF5F769FF07B0FE
:10E2A000BDE8F04FFCF728B94A0001461C4803F0CE
:10E2B00099B92DE9F0411B4980000968896D21FA5F
:10E2C00000F000F00F04C1F30325C1F30317C1F3FD
:10E2D0000336C1F30358AC421FD1B8F10F0F05D07C
:10E2E00003F066FA10F4817F18BF4446AC420BD1AC
:10E2F0000F2E09D00C488088C0F3403020B103F0C5
:10E30000F8F9082818BF3446AC4206D10F2F04D0C4
:10E31000F6F70BFE002818BF3C462046BDE8F0810A
:10E3200080760110F805011064AF0110FE48408AA4
:10E330007047FD49B0F5C87F488284BF4FF4C8706C
:10E3400048827047F848808A7047F749888270474A
:10E35000F548C08A7047F44AF449D0820968098BAD
:10E36000814238BFD1827047EF4840787047EE490C
:10E370000228487004D8888ACA8A824228BF704717
:10E38000002048707047E848818AC28A09054078B1
:10E3900041EA022108437047E348C0897047E249D7
:10E3A000C828C88184BFC820C8817047DE48008A59
:10E3B0007047DD49C828088284BFC820088270479A
:10E3C000D94880897047D84AD84990810968098B13
:10E3D000814238BF91817047D348817B028A090608
:10E3E000808941EA024108437047CF4880787047EE
:10E3F000CD4988707047CC48008B7047CA49C828FF
:10E40000088384BFC82008837047C748408B704783
:10E41000C549B0F5C87F488384BF4FF4C8704883AE
:10E420007047C1488178428B0906008B41EA02316E
:10E4300008437047BC490A78104308707047BA48CF
:10E4400000787047B84900200870704710B504463E
:10E4500003F00DFAB44AB6492CB9137891F800C00C
:10E4600013EA0C0F06D1401E844205D1107849787A
:10E47000084201D0012010BD002010BD2DE9F05F41
:10E48000DFF8A4B200252E469BF80140BBF814A08B
:10E49000BBF8169003F096F90746A44820210068BF
:10E4A000008BB0FBF7F8A34803F0E6F99BF80200F5
:10E4B000012808BFBDE8F09FF6F74AFC05281EBFFB
:10E4C000002C0024002F98BFBDE8F09F7B1E9748CA
:10E4D000026808FB04F081B29C420FBF108B601CE5
:10E4E00008FB00F080B28A4524BF50452546894587
:10E4F00024BF48452646601CC4B2BC42E9D3B5429D
:10E5000028BFBDE8F09F8B4ADBF82010012099B1AD
:10E51000002D08BFBDE8F09F791B491EBB1BC9B287
:10E520005B1E8B42C8BFBDE8F09F5054491EC9B264
:10E530008B42FADDBDE8F09FB54288BFBDE8F09F91
:10E540005055691CCDB2B542FAD9BDE8F09F2DE90E
:10E55000F003754875494FF0070CA0F80EC0096824
:10E56000002340F22634B1F8C620028240F29A22FB
:10E570008281B1F8C42042824370848240F2855483
:10E58000C4828370A0F818C0428391F86C1011F017
:10E59000040F09D011F0010218BF0122C26111F06D
:10E5A000020118BF01210162D0F81C8001216048DE
:10E5B0000426402302220827802420254FF0100C37
:10E5C000B8F1000F0BD0017086700171837180F873
:10E5D00008C04270C7704271C47145720AE002708F
:10E5E00087700271847105724170C6704171C37188
:10E5F00080F809C0BDE8F00340E72DE9F04703F0DB
:10E60000EBF804464A4E90F8E804DFF81C81002736
:10E61000A6F14A05C0B9B078F178727A0843317A28
:10E62000114340EA010903F0D2F803F0CBF80100EE
:10E63000384607D02A5C22EA09022A54401CC0B29C
:10E640008142F7D8A8F8037094F8EA04A0B93079A9
:10E65000717940EA010903F0BAF803F0B3F8002138
:10E66000002807D96A5C22EA09026A54491CC9B227
:10E670008842F7D8A8F8057094F8EC04002818BF71
:10E68000BDE8F087B079F17940EA010403F09FF822
:10E6900003F098F80021002898BFBDE8F0876A5C75
:10E6A000A2436A54491CC9B28842F8D8BDE8F08731
:10E6B00070B514460D46064603F084F803F087F85B
:10E6C00003F0DFF80023012E02D0022E0CD016E05A
:10E6D000042C08BF012312D0052C08BF04230ED040
:10E6E000082C08BF41230AE0042C08BF022306D0EF
:10E6F000052C08BF082302D0082C08BF8223C5EBD5
:10E70000051101EB451100EB8101087B8A7B8242F8
:10E710002CBF094A70BD12F800C04CEA030C02F885
:10E7200000C0401CC0B209E0F4060110240701102B
:10E73000E2800110C28001109880011091F80EC093
:10E740008445E8D270BD2DE9FF4F91B0044603F037
:10E7500043F8DDE9126005940090149C03F037F84B
:10E7600003F03AF8FF4990F8E8240968012A0CBF41
:10E77000B1F90E1091F8CC104625049103F077F80A
:10E78000079003F01FF84FF0000901900098C84669
:10E790004A464946CC464B46A0426BD8DFF8C8A350
:10E7A000019F9AF806E07F1E06979AF804709AF87F
:10E7B00002A0CDF80CA0DDF814A01AF800A0BAF160
:10E7C000000F2ED036F910B0DDF810A0D34528DBAD
:10E7D000DFF898A31AF800A0CDF808A01AEA070FEE
:10E7E00014D138B1DFF884A382441AF801AC1AEAD4
:10E7F000070F0BD1DDF818A0504509DADFF86CA33C
:10E8000082449AF801A01AEA070F01D0521CD2B232
:10E81000DDE902AB1AEA0B0F1CBF09F1010909F08F
:10E82000FF0936F910A0AA4504DB002B08BF844677
:10E830005B1CDBB2AA4501DBA04217D1062B14D327
:10E840006344E2460293534588BFC84B0DD913F881
:10E850000AB04BEA0E0B03F80AB00AF1010ADDF820
:10E8600008B00AF0FF0AD345F1D80023401CC0B21B
:10E87000A042A0D900984FF0000AD446A0426BD81D
:10E88000079B5B1E0093019B5B1E0793B64BDF79D2
:10E89000069793F805B0DB780393DDE9007307FB77
:10E8A00003039FB2059BDB5D33B336F917E0049B8E
:10E8B0009E4521DBAD4B13F800E01EEA0B0F0FD194
:10E8C00028B1034413F8013C13EA0B0F08D1079B4E
:10E8D000984207DAA54B03445B7813EA0B0F01D08B
:10E8E000491CC9B27346DDF80CE013EA0E0F1CBFD9
:10E8F00008F1010303F0FF0836F91730AB4207DBDC
:10E90000BCF1000F08BF82460CF1010C0CF0FF0CAB
:10E91000AB4201DBA0421BD1BCF1060F16D3D4449D
:10E920005346CDF808C09C4588BFDFF840E20DD9BA
:10E930001EF80370DDF818C047EA0C0C0EF803C08F
:10E940005B1CDDF808C0DBB29C45F1D84FF0000C31
:10E95000401CC0B2A042A0D9854F87F8009087F82C
:10E96000018007F1020888F8002088F80110DDE92D
:10E970001254149E02F02BFF029002F02DFF019022
:10E98000387898F8001098F801200844C1B27878D7
:10E990004FF0010A1044C2B2019890F8E80401282F
:10E9A00047D1002918BF002A43D0029880F8E8A474
:10E9B0000020009002F00BFF02F059FF074602F022
:10E9C00001FF6A4A2821B442B2F84C20ADF8002079
:10E9D0002FD87B1EA7F102089DF800C09DF801709A
:10E9E000DFF8889135F914B002198B45BCBF35F9B1
:10E9F00012208A4205DA19F8042022EA0C0209F8EA
:10EA0000042003FB004292B208FB004B35F91220B0
:10EA10001FFA8BFB8A42BCBF35F91B208A4204DAFD
:10EA200019F80420BA4309F80420621CD4B2B44295
:10EA3000D8D9019890F8EA04012830D14D4E3078A9
:10EA400071780144CCB288B94748057902F0BFFE1D
:10EA500002F0B8FE0021002888BF444A06D9535C62
:10EA6000AB435354491CC9B28842F8D8707888B96E
:10EA70003D48457902F0ABFE02F0A4FE00210028DB
:10EA800088BF3A4A06D9535CAB435354491CC9B2B8
:10EA90008842F8D8002C1CBF029880F8EAA4002015
:10EAA000DDE91394DDF84880009001900290039016
:10EAB0000490059006900790089009900A900B909A
:10EAC0000C900D900E900F9002F081FE90F8E814DB
:10EAD00001291FBF90F8EA14012990F8EC040128DD
:10EAE0001CBF15B0BDE8F08F6E4608AD02F06AFE9F
:10EAF000074602F0BCFE864628214FF0020C48462D
:10EB0000A14598BF7B1E15D80CFB070238F91220CF
:10EB10008A420BDB06F800A000281CBF321802F85E
:10EB200001AC9842BCBF321882F801A0401CC0B2B0
:10EB3000A042E9D9AEF10300C2B24846A14598BF50
:10EB40007B1E26D802FB070C1FFA8CFC38F91CC070
:10EB50008C451ADB05F800A0002818BF05EB000C57
:10EB60000AE0000024070110E280011098800110E3
:10EB7000F7060110F906011018BF0CF801AC984215
:10EB8000BCBF05EB000C8CF801A0401CC0B2A04239
:10EB9000D8D9DFF858B46F4608AE9BF801A002F050
:10EBA0001BFE02F064FE109002F00CFE05469BF87E
:10EBB0000200012803D0F6F7CBF8052801D14FF069
:10EBC000000AA14584BF15B0BDE8F08FDFF820C46E
:10EBD00010980CF14A03A0F1010B9A7893F804E025
:10EBE00009EB050042EA0E021CF809E012EA0E0FDA
:10EBF00010D01A78524504D1FE4A12F80920012A91
:10EC000008D0002228F8192017F80910002908BF99
:10EC100028F810200BFB0590DA7893F805E080B215
:10EC200042EA0E02411B1CF809E089B212EA0E0FFB
:10EC300010D05A78524504D1EE4A12F80920012A20
:10EC400008D0002228F8102016F80900002808BF74
:10EC500028F8112009F1010000F0FF09A145BCD9F5
:10EC600015B0BDE8F08F2DE9F14FE0488AB090F87B
:10EC70000190818A0491B0F8168002F0A8FD044644
:10EC800002F0AAFD02F0FDFD0290DB4800260068BC
:10EC900090F8CE0080000590A0790190207A009035
:10ECA00094F84170002F88BF4FF0010A5FD9C6EB7E
:10ECB000061000EB4611029800EB8105CE48B5F82E
:10ECC00064100268B2F818B001FB0BF0118A90FBD7
:10ECD000F1F081B2ADF81C10B5F86600B2F81AC0B8
:10ECE000538A00FB0CF090FBF3F080B2ADF80C00FF
:10ECF00092F86C2012F0040F14BF2AEA020302F00B
:10ED000001031BB1ACEB0000401E80B212F0020FF9
:10ED100003D0ABEB0101491E89B212F0040F19BFF9
:10ED2000ADF81C00ADF80C10ADF81C10ADF80C00DF
:10ED3000BDF81C00A5F8A200BDF80C00A5F8A400C1
:10ED4000AA48807801280ED0F6F702F8052818BFE7
:10ED5000B9F1000F07D0BDF80C000499884224BF18
:10ED6000804585F899A0701CC6B2BE429FD3DFF8DB
:10ED70007C9299F80180B9F80E60B9F81050B9F892
:10ED80000C70B9F818A002F022FD029002F079FD93
:10ED9000099002F07BFD029890F841B09648006817
:10EDA000438B99F80200012804BF554656460020BF
:10EDB0008146BBF1000F61D9A3F1C8010891991BED
:10EDC0000691591B4FF0010E0491C0EB001101EBAD
:10EDD0004012099901EB8201B1F8A220B1F8A4C058
:10EDE00081F89690C82A13D8B8F1010F04BF91F8A2
:10EDF00099A0BAF1010F04D0BC4506D8964201D2C1
:10EE000038E03ABB81F896E01AE0AA42FAD931E03C
:10EE1000DDF820A052452DDBB8F1020F04BF91F8B8
:10EE200099A0BAF1010F06D0BC4514D8DDF818C07E
:10EE3000944502DD1EE09A421CD3022281F89620FE
:10EE4000D1F8B020022A0BD0032A04BF91F86F201A
:10EE5000012A05D00EE0DDF810C09445EDDD09E093
:10EE6000029A82F8E9E40622C1F8902091F89620EF
:10EE700081F89720401CC0B25845A6D394F8E80406
:10EE8000002865D0594D2889401C80B22881B0F5F2
:10EE9000167F84BF4FF4167028816889401C80B2A9
:10EEA00068810599884229D302F08CFC03004FF059
:10EEB000000118BF4E4A1FD0505C10F0100F1CBF4D
:10EEC00020F010005054C0B210F0200F1CBF20F0F2
:10EED00020005054C0B210F0040F1CBF40F01000CE
:10EEE0005054C0B210F0080F1CBF40F02000505426
:10EEF000481CC1B29942DFD3A5F80A903B4D68780F
:10EF0000059002F064FC074602F0BBFC049002F09E
:10EF1000BDFC029038480068D0F8C810069190F8FF
:10EF2000CE100891AA786E8A698B97F841A0408B21
:10EF3000012A08BF0E46801B4FF0000B87B25D46CA
:10EF4000BAF1000F88BF4FF001087DD800F068B912
:10EF50000A980690019805900098049002F037FCFA
:10EF6000064602F08EFC054602F090FC2248002185
:10EF700096F8416000680A460B46B0F81AC090F84F
:10EF8000CDB0002E2DD9DFF874A0ACF125084FF0DC
:10EF9000010E0227C3EB031000EB431005EB8000CA
:10EFA00080F8979090F8A8C01CF0010F15D0B0F829
:10EFB000A2C0BCF1250F06D880F897E09AF80000AF
:10EFC000012808D13DE0C44507DB80F897709AF826
:10EFD0000000022835D0501CC2B2581CC3B2B34244
:10EFE000D8D3074B187808440CE00000F406011051
:10EFF00098800110C280011024070110E2800110E6
:10F00000F9060110597810F0FF001144C9B24FF011
:10F01000000518BF00290BD00844834508D8DDE956
:10F0200005100125049A00F06FFBFE48A0F80A9035
:10F03000FC4884F8E854A0F80890A0F80A905DE72E
:10F0400002E0481CC1B2C8E7C5EB051000EB451152
:10F05000049800EB810090F85510D0F890C0C1EBF7
:10F06000011202EB41120299B0F8A43001EB8201C7
:10F07000B0F8A220BCF1060F6AD0D0F8B0C0BCF145
:10F08000020F18BFBCF1030F08D090F8A82012F0AF
:10F09000010F5DD0026D022A7ED0BCE080F897900F
:10F0A000B24282BF97424FF0020CC0F890C00AD81B
:10F0B000D0F850C0BCF1020F02BFD1F890C0BCF133
:10F0C000020FC0F890C0D0F8B0C0BCF1030F04BF6D
:10F0D000D0F850C0BCF1020F07D1D1F890C0BCF1FC
:10F0E000010F08BFC0F8908032D0D0F890C0BCF1BA
:10F0F000020F18BFBCF1010F2AD0B24298BF80F8AE
:10F10000978006D997429CBF4FF0020C80F897C0B9
:10F110001ED890F897E0DDF814C0E64504BF90F8DB
:10F1200099C0BCF1010F5DD0D0F8B0C0BCF1020FA6
:10F130000FD0D0F850C0BCF1020F6CD191F898C03C
:10F14000BCF1000F05D0D1F890C0BCF1030F12D074
:10F1500061E0A0F89A20A0F89C30B0F86410A0F804
:10F160009E10B0F86610A0F8A0100321C0F890100F
:10F1700080F898804FE0B1F89AC0B1F89CE0A2EB1B
:10F180000C02A3EB0E03524303FB0322069B9A429D
:10F1900028DCA0F89AC000E02DE0B1F89C20A0F88F
:10F1A0009C20B1F89E20A0F89E20B1F8A020A0F8E5
:10F1B000A02091F89810491CC9B280F89810089ABC
:10F1C00091423CBF0321C0F8901024D30421C0F821
:10F1D00090100A4690F897002946FFF769FA4FF019
:10F1E000010B18E0C0F89080D0F8A81041F400712D
:10F1F000C0F8A8100FE0B1F89A20A0F89A20B1F852
:10F200009C20A0F89C20B1F89E20A0F89E20B1F888
:10F21000A010A0F8A010681CC5B25545FFF414AFAB
:10F2200094F8EA044FF000084BEA000084F8EA047E
:10F230000A980690019805900098C3464FF0020A7C
:10F24000049002F0C4FA009002F01BFB074602F0A3
:10F250001DFB009890F841507348006890F8CE006C
:10F26000460802F004FB0190009890F8E804012899
:10F270007ED16C480089B04208D8DDE90510049AB7
:10F2800000F042FA6748A0F80A9038E00026002D06
:10F290003AD90198801E0290C6EB061000EB46108A
:10F2A00007EB8000D0F8A81011F0010F23D011F463
:10F2B000007F20D1417801290ED803785B4AD35CC6
:10F2C0004A3292F808C013EA0C0F05D010780522D4
:10F2D0003146FFF7EDF90EE0029A91420BDB01781F
:10F2E0005248415C4A30427A114204D040780522AB
:10F2F0003146FFF7DDF9701CC6B2AE42CCD30098A0
:10F3000090F8E804012851D10020002D84BF019914
:10F31000A1EB0A0318D9C0EB001101EB401107EB78
:10F320008101D1F8B020022A18BF032A08D14978F8
:10F33000514505D39942BCBF08F1010101F0FF0816
:10F34000401CC0B2A842E6D3B8F1000F1CBF002693
:10F35000002D2BD90198DFF8D8A0A0F10108C6EB49
:10F36000061000EB461007EB800090F8A81000E0B4
:10F370001CE011F0010F15D04178002908BF9AF860
:10F38000003004D0414508BF9AF801300AD14BB192
:10F390000421C0F890100A4631461846FFF788F954
:10F3A0004FF0010B701CC6B2AE42D8D394F8EA04F9
:10F3B0004FF0000A4BEA000084F8EA04DFF864B07A
:10F3C00002F005FA054602F05CFA009095F84180DB
:10F3D00002F04DFA00218BF800100D46B8F1000F35
:10F3E0007AD9DFF84890461F09F14A07C5EB0510A6
:10F3F00000EB4511009800EB810BDBF8900004282E
:10F4000018BF06287CD0DBF8B000022818BF0328FC
:10F4100076D100219BF801000A46042811D89BF8F8
:10F42000003007E0F4060110240701109880011055
:10F43000E280011019F8033097F806C013EA0C0FA8
:10F440000AD1B04221DB9BF8003097F807C019F8C9
:10F45000033013EA0C0F18D09BF8003097F804C063
:10F46000012219F8033013EA0C0F03D0042801D845
:10F47000387807E097F805C013EA0C0F05D08642EC
:10F4800003DC78788BF8970029E09BF89730002B05
:10F4900008BF002A34D09BF80E209BF80CC09BF8C4
:10F4A0000DE0A2EB0C0202F0FF0C9BF80F20A2EB88
:10F4B0000E02BBF846E0D2B2BEF12D0F04D2ACEB87
:10F4C0000202921D0C2A00D901213BB931B1042856
:10F4D000CED9B042D5DA02E017E011E081B10920BF
:10F4E000CBF890009BF8970008222946FFF7E0F838
:10F4F000B4499BF897004FF0010A0A78104308704E
:10F50000681CC5B24545FFF471AF94F8EA044AEAB5
:10F51000000084F8EA044FF0000ACDF800A0CDF80E
:10F5200004A0CDF808A002F052F9044602F054F904
:10F53000814602F0A6F9804602F0A8F9074684F851
:10F54000EBA494F84100002200282CD901250326C1
:10F550004FF0020C4FF00A0B0DF1FF30C2EB02111D
:10F5600001EB421108EB810191F85530C3EB031E0A
:10F570000EEB4313D1F8B0E007EB8303BEF1020FAB
:10F5800018BFBEF1030F15D091F8A83013F0010F8A
:10F590001CBF91F8541001F800B0511CCAB294F885
:10F5A00041109142DAD80025EB468748405D01289A
:10F5B00038D099E091F898E0BEF1000F13D0D1F85F
:10F5C0009030042B18BF092B06D0BEF1050F84BF65
:10F5D00091F854301D5403D891F8543003F800C00A
:10F5E00081F86F60D9E7D1F890E0BEF1010F18BF44
:10F5F000BEF1020FD1D1D1F850E0BEF1020F0CD113
:10F6000093F898E0BEF1000F07D0B3F89EE0A1F8A0
:10F6100064E0B3F8A030A1F8663091F8541001F816
:10F6200000C0BAE71BF8051021B10A2908BF0BF882
:10F63000050059E094F841C0BCF10A0F3CBF94F8B2
:10F6400042000A2850D299F841300020002B88BF90
:10F650006A1C49D9C0EB001101EB401108EB81068F
:10F6600007EB810191F854E0964539D1D1F890E04B
:10F67000BEF1090F1FBFD6F89060062E91F8A810B2
:10F6800011F0010F2CD0CCEB0C1101EB4C1108EB5D
:10F690008106C0EB001101EB401007EB8001BC229A
:10F6A000304601F090FF94F84100401C84F841007E
:10F6B00094F84200401C84F8420094F8EB04401C8B
:10F6C00084F8EB04B6F89E00A6F86400B6F8A00033
:10F6D000A6F8660086F898A00720C6F8900003E018
:10F6E000401CC0B28342B5D8681CC5B20A2DFFF4D5
:10F6F0005CAF36480099016201994162BDF808107B
:10F7000001850BB0BDE8F08F2DE9F05F15460F467F
:10F71000064602F05CF8044602F0B3F802F0A7F8DF
:10F72000804602F04FF88346294894F8E8140068B0
:10F73000012906BF90F8CC00420890F8CC203C4646
:10F74000DFF888C0AF420CF14A0A9CBF9AF8020069
:10F750009AF8089013D836F9141091420BDD1CF872
:10F7600004100F2C41EA00030CF8043024BF43EAD4
:10F7700009010CF80410611CCCB2AC42EBD9A8F121
:10F78000010000FB0BF081B2AF423ABF9AF80330A0
:10F790009AF80940BDE8F09FC81936F91000904268
:10F7A00009DD1CF8070018430CF807000F2F24BFD1
:10F7B00020430CF80700781CC7B2AF42ECD3BDE879
:10F7C000F09F0000F4060110B8800110988001102D
:10F7D00024070110002818BF0120FD490860704768
:10F7E000FB480068704730B44FEA216C4FF47A74DC
:10F7F0000CFB04FCC0F80CC041F3072C0CFB04FC10
:10F80000C0F804C04FFA81FC0CFB04FC40F808CBA4
:10F8100041F30741614340F8081B92E83210A0E829
:10F8200032101169C0E9001330BC704770B5EB4C61
:10F83000E84BE94A2068816CE948FFF7D4FF20686B
:10F84000E74DE84B416DE84A05F12800FFF7CBFF93
:10F85000206890F8401011F0100F08BF70BDE34B06
:10F86000D0F8841005F15000BDE87040E04ABAE7D6
:10F87000DB487047D949DFF868C3096860B10128DF
:10F880000FD0022813D0032818BF7047D14BD24A9B
:10F89000D1F890106046A6E7CE4BCF4A896C6046FF
:10F8A000A1E7D44BD44AD1F8881060469BE7D14BEE
:10F8B000D14AD1F88C10604695E7C849DFF83CC3BF
:10F8C000096840B1012818BF7047C64BC64AD1F835
:10F8D0009410604687E7C34BC34A496D604682E790
:10F8E000BF4AC06A92689042A5BFC86A9042012090
:10F8F000002070472DE9F04FDFF8E08204468DB01C
:10F90000D8F800304FF0010793F8400010F0080FCE
:10F910001CBFD4E90250D4F810C02FD050F8142CDA
:10F92000BC3812F0010F27D0016D022924D190F8C4
:10F930005510C1EB011606EB41110CEB8101B1F83A
:10F94000A86016F4006F17D091F8B46007FA06F6B5
:10F9500016F0060F10D0D1F88C10032918BF042917
:10F9600006D012F4007F03D190F84A10022903D97F
:10F9700042F40061C0F8A810A842CFD8D4E903052A
:10F98000D4F800C0A66810F8141CBC3811F0010FA0
:10F990002AD090F855200021C2EB021909EB42123F
:10F9A000D0F8509005EB8202B9F1020F08D09CF814
:10F9B0004120012A04BF9CF8E624002A12D012E05C
:10F9C00092F8B41007FA01F111F0060F18BF0221E6
:10F9D00009D192F8381007FA01F111F00C0F08BFA5
:10F9E000012100D003218163B042CCD893F84400B8
:10F9F00010F0010F04D0824A2C21204601F04BFF69
:10FA0000D4E902C0764A50F8143CBC3813F0010F18
:10FA100020D0C16A13F4006F18BFC0F8AC7015D1C4
:10FA2000D3688B42B8BF01210EDB53688B42B8BF4D
:10FA3000032109DB13688B42B8BF042104DB936800
:10FA40008B42B4BF05210221C0F8AC1090F8AC1075
:10FA500080F84F106045D6D8D8F8000090F84000E4
:10FA600010F0100F7CD0D4E90295664E4FF0040AD6
:10FA700015F8140CBC3D10F0010F13D0726A294622
:10FA800068469047316A049BEC4606F110025046E6
:10FA90001944401E5CF8203052F820B003FB0B11D3
:10FAA000F7D169634D45E3D8D8F8000090F880009D
:10FAB00010F0010F04D0544A3421204601F0EBFE2F
:10FAC00001F0EEFE00286AD041480068012866D1A6
:10FAD0002068434DA36890F841002669C0EB0011EF
:10FAE00001EB4010D5F80CC003EB800151F8142C49
:10FAF000BC3912F0010F11D0086D02281CBF42F46E
:10FB00008050C1F8A80062D010F4805F1CBFCA6AA0
:10FB10006245C4BF20F48050C1F8A8009942E5D8DE
:10FB20002D4905F1500201F16006D4E9023096E852
:10FB300060128DE86012D1F870C04D6F896FCDE909
:10FB400004C50691EC4650F8141CBC3811F0010FA6
:10FB500018BF11F4805F20D0416BD568A94200E046
:10FB60001DE0C8BF01210EDC5568A942C8BF0321B2
:10FB700009DC1568A942C8BF042104DC95688D42E0
:10FB8000B4BF052102215CF82150D0F8AC605CF8CC
:10FB90002660B54238BFC0F8AC109842D3D80E48A2
:10FBA000D8F80020D4E9001CD0E9145692F840207F
:10FBB000D0E9169012F0010F08AB4FF0FF321EBFD4
:10FBC00091F848A0BAF1010F91F814A01EE070E07E
:10FBD0004807011035DF0010F03F01002407011035
:10FBE0007C97011075DF00100440010097DF0010C2
:10FBF0002C40010059DF001018400100A4970110AB
:10FC000091180100CC9701106538010014BFBAF1BA
:10FC1000010F04205ED0CDE90A90CDE908569CF88A
:10FC20004300042822BF91F8410004280A92994613
:10FC30002569D4E90264F4F76AFED8F800804FF031
:10FC4000020A54F8142CBC3C12F0010F2CD094F88A
:10FC50005510D4F8ACC0C1EB011303EB411105EB17
:10FC60008103A16B12F4805F0AD0D4F850B0BBF1CD
:10FC7000010F36D0B3F8A82012F4005F18BF00219E
:10FC800098F8442012F0020F04D0012902BF9A6BA9
:10FC9000002A002159F8211007FA0CF2114214BF72
:10FCA000C4F8AC70C4F8ACA0B442CAD80DB0BDE87A
:10FCB000F08F91F85500C0EB001909EB401006EBEE
:10FCC0008000B0F8A800000B60F30C321046C1F8B9
:10FCD000A82019E703EB8001401E41F8042CF9D15C
:10FCE000A5E700281CBF42F40051C4F8A810012168
:10FCF000C6E710B5044601F06AFD206001F0C1FDC1
:10FD00000146A060206890F84100C0EB001202EBB1
:10FD1000401001EB8000E06001F05EFD606001F0EA
:10FD2000B5FD206110BD002908BF7047F0B5A7B030
:10FD3000044601F04CFD219001F0A3FD2199239090
:10FD400091F84110C1EB011202EB411100EB81006F
:10FD5000249001F041FD229001F098FD259021A80A
:10FD6000FFF7C8FD214621A800F07AF8FE48007888
:10FD700030281CBF27B0F0BD8421684601F028FC64
:10FD8000DDE92110DDE9234791F841106E46002995
:10FD90005BD090F84100354630B9F4F7DFFF4FF4FF
:10FDA0007A714843ADF80000F04994F8A80010F0CB
:10FDB000010F3AD0B5F9000094F854200244206DA8
:10FDC000012818BF002000EBC00303EB001002EB7A
:10FDD000800025F8020BB4F8A80094F84F20C0F377
:10FDE000403000EBC00303EB001002EB800025F86D
:10FDF000020BB4F8AC0025F8020BE06A81FB00208E
:10FE00004211A2EBE07025F8060B206B81FB00206D
:10FE10004211A2EBE07025F8040C606B81FB00201E
:10FE20004211A2EBE07025F8020CBC34BC42BCD3FA
:10FE3000CF49A81B81FB00104110B1EBE07004D04A
:10FE40004FF618412980421C00E00022002A04BF1E
:10FE500027B0F0BD06216846F9F719FF27B0F0BDBD
:10FE60002DE9F04F8BB00F46064601F0A1FC10F4CF
:10FE7000807F4CD034683769B56894F841600021C0
:10FE8000C6EB061000EB461005EB80004FF00208B1
:10FE90004FF0010950F814CCBC381CF0010F1ABF08
:10FEA000D0F8AC20022A491C27D090F85520C2EB8C
:10FEB000021303EB4212036D07EB8202022B0CBF0D
:10FEC000D2F8B430002309FA03F313F0060F07D079
:10FED000B0F90230B2F90220B3EB620F0DDA09E09B
:10FEE00090F84C2090F84D30B2EB430F02D21CF446
:10FEF000806F02D0491CC0F8AC80A842CAD8701AE2
:10FF000084F8420084F845100BB0BDE8F08F10F083
:10FF1000020F49D0D6F800C0B46800219CF84150C7
:10FF20003769C5EB051000EB451004EB80004FF07E
:10FF30000208012610F8142CBC3812F0010F1ABF69
:10FF4000D0F8AC20022A491C24D090F85520C2EBEE
:10FF5000021303EB4212036D07EB8202022B0CBF6C
:10FF6000D2F8B430002306FA03F313F0060F07D0DB
:10FF7000B0F90230B2F90220B3EB620F0ADA06E000
:10FF800090F84C2090F84D30B2EB430F02D3491C4F
:10FF9000C0F8AC80A042CDD8681A8CF842008CF82A
:10FFA00045100BB0BDE8F08F3568D6F808A0306971
:10FFB0000790B5F902004FF0000B4010099095F83A
:10FFC000418001F0FFFB814601F051FC0890694837
:10FFD0000068069090F8400010F0020F55D0B1680C
:10FFE000304605913168D0E9034604916249426880
:10FFF00091E80A508DE80A5092F84310042907D37B
:020000021000EC
:10000000049991F84110042924BF4FF00041029156
:10001000069991F8501011F0010F03D0574A302182
:1000200001F039FC5348036854F8142CBC3C12F01E
:10003000010F27D012F4805F24D194F85500EC46CC
:10004000C0EB001101EB4010196D06EB800E12F4AD
:10005000006F17D1B4F84600C1F3072290420ED3C7
:10006000226BA06B11F0020F05D0012802BFDEF851
:100070003810002900205CF82000904202DD0220A8
:10008000C4F8AC0005988442CED801F00EFC20B133
:10009000287B022808BF4FF0010B0021C8EB081095
:1000A00000EB48100AEB80004FF0020C012450F8DE
:1000B000143CBC3813F0010F1ABFD0F8AC20022A50
:1000C000491C3FD090F85520C2EB021606EB4216B1
:1000D000079A02EB8602066D022E0CBFD2F8B02002
:1000E00000222E7B1EB112B913F4807F27D1B8F104
:1000F000010F27D904FA02F212F0030F18BFBBF167
:10010000000F1FD0B0F90230099A93421ADD4278ED
:100110004AB10678A2F1010E0EFB096637F91660A6
:10012000B6EBE30F0BDD089E521CB2420AD20678F2
:1001300002FB096237F91220B2EBE30F02DC491C23
:10014000C0F8ACC05045B2D8B8EB010085F8420009
:1001500085F8451004BF0BB0BDE8F08F297B99B935
:10016000297D01290CE00000490501101F85EB5194
:10017000ABAAAA2A24070110A497011025E10010B8
:100180001CBF0BB0BDE8F08F95F80F14814208BF7B
:1001900085F8114495F8D314814208BF85F8D544F9
:1001A000FFE62DE9F0410F4606460A2501F00AFB5D
:1001B000044601F05CFB5FEA000C06EB4C014FF0DB
:1001C000000314BF0020BDE8F0810022002C0ED9EE
:1001D00036F91380A84503DB31F91280454503DD6C
:1001E00003FB042827F81800521CA242F0D35B1C22
:1001F0006345EAD3BDE8F08170B5044601F041FBE8
:10020000002506464FF0FF3C284663462946002C51
:1002100015DDC1EB011202EB411206EB8202526ABC
:10022000AA4204DD2846634615B28C4603E090429C
:10023000BCBF10B20B46491C09B2A142E9DB002148
:10024000002CD8BF70BD614518BF99420BD0C1EBDF
:10025000011000EB411006EB8000D0F8A82022F03E
:100260000102C0F8A820481C01B2A142EBDB70BD1E
:100270000846022998BF7047BEE70000002808D052
:10028000002906D0002B04D08B4202D8194601F079
:10029000BDB970472023002219461248EEE71148E5
:1002A000704720207047F0F7EAB9F0F7F3B9F0F79C
:1002B000F4B9F0F711BAF0F710BA30B414460028C8
:1002C0000CD000290AD0002C08D0002B06D08B427D
:1002D00004D8214630BC1A4601F084B930BC7047BE
:1002E000F0F7C6B9000001100020704730B41D4679
:1002F000029B144658B101280DD0022811D00328C2
:1003000013D1C8B22A46214630BC00F035BA30BC01
:10031000C8B200F025B9C8B2AAB2214630BC00F07C
:100320005EB930BC084600F0F0B930BC70477CB50F
:1003300014460D460646FFF7B2FF002200929DF8D4
:100340000010019241F040018DF800104470A007A8
:100350000ED4600704D59DF8000040F0040005E0CD
:10036000200705D59DF8000040F010008DF8000032
:100370009DF8000040F002008DF8000030098DF873
:10038000020028098DF8030006F00F0060F31F1526
:100390008DF804506846FFF78AFF7CBD70B50546AE
:1003A000FFF77DFF0446FFF77AFF024669484FF6E4
:1003B000FF73022D4575018803EA4106A4F8F06138
:1003C00006D0032D13D003260023042D20D031E0C6
:1003D00024F81130018804EB41014B80018804EBC3
:1003E00041018B80018804EB4101CB809BE04EF6FC
:1003F000EE6224F81120018804EB41014A80018853
:1004000004EB41018A80018804EB4101CA808AE043
:100410005278550701D501220AE0950701D502223D
:1004200006E0950901D0067505E0120702D5042201
:10043000027500E00375427C032A00D9467424F853
:100440001130018804EB41014B80018804EB41012C
:100450008B80018804EB4101CB800188837C34F8D8
:100460001120C3F3100342EAC33224F81120C17CE7
:1004700003888903C1F3803142EA813124F81310E3
:10048000438902889B00C3F38B0341EA830124F86C
:100490001210037D028803F00303194324F812109D
:1004A0000188458804EB41026FF47023518803EA08
:1004B0000515294351800288C57B04EB420205F0F3
:1004C0000F05294351800188858804EB410203EA26
:1004D00005159188294391800288857B04EB4202AF
:1004E00005F00F0529439180017D0329018804EB64
:1004F0004101CA881DD0058903EA05131A43CA8041
:100500000188037C04EB41029B00D188C3F3810383
:1005100041EA8301D1800288437C04EB420203F06C
:1005200003031943D1800188B1F5F77F03D9FA217C
:1005300002E0C588E0E7091D018070BD06A0704794
:10054000042070471320704705207047704770479C
:10055000704700002298011041373330000000003E
:1005600070B5B44D00260446642801D0652C1CD11A
:10057000287818B1012801D0022805D1AE4884217D
:1005800001807220FFF7E4FF642C01D0652C0CD1B0
:10059000287818B1012801D0022806D1A748468141
:1005A000067346730220FFF7F9FEA5482C700680FB
:1005B000204600F063F9204600F058F9204600F08C
:1005C00059F9204600F04EF9204600F047F9204640
:1005D00000F058F92046BDE8704000F021BC2DE93C
:1005E000F04789460446014690462120FFF7B0FFB8
:1005F000FFF755FEB0F94800B0F5704F01DB012060
:1006000004E0FFF74CFEB0F94800401C01B2242082
:10061000FFF79EFF8A4D5020B5F90010FFF798FFB5
:10062000844E3078652817D1062C15D1B5F90020F5
:10063000501C11D0521C11B229802320FFF788FFD3
:10064000B5F90000C62807DBE01F28800121222021
:10065000FFF77EFFFFF727FE784D00276889B0F58A
:10066000616F03D16F810320FFF798FE3078642813
:1006700002D0652816D10BE0287B401CC0B228733D
:10068000282803D16889401C68812F73BDE8F08752
:10069000687B401CC0B268733C2803D16889401C49
:1006A00068816F73082CF1D2DFE804F0050B111795
:1006B0001D042329EAE741464846BDE8F04700F01B
:1006C000DEB841464846BDE8F04700F0D0B84146A4
:1006D0004846BDE8F04700F0CEB841464846BDE880
:1006E000F04700F0C0B841464846BDE8F04700F08A
:1006F000B6B841464846BDE8F04700F0B5BA4146B5
:100700004846BDE8F04700F08CBB70B50546FFF7E2
:10071000C6FD0478FFF7C3FD4A4A0078C4F34001E0
:10072000494B1170C4F380021A70484BC0F380101B
:1007300011431870C4F3C003454C0143237004D126
:10074000481E3F490880FFF7AEFD284600F098F8A4
:10075000284600F08DF8284600F08EF8284600F074
:1007600083F8284600F07CF8284600F0DBFA28469B
:10077000BDE8704000F056BB2DE9F0411E4617461B
:100780008846050029D12B493220002408702C48C6
:1007900030490480062008702B48047029480470F2
:1007A0002D48047024480480FFF774FDFFF777FD9F
:1007B00002462248FA214FF4F773018002210174A6
:1007C0004475FA2002EB400122F810404C80001DD5
:1007D0008C8080B2CC809842F4D933463A46414668
:1007E000284600F04EF833463A464146284600F087
:1007F00040F833463A464146284600F03EF8334634
:100800003A464146284600F030F833463A464146DB
:10081000284600F026F833463A464146284600F07E
:100820009AFA33463A4641462846BDE8F04100F080
:10083000FABA00005D070110660701102298011046
:100840005E070110600701106107011062070110C7
:10085000640701105C0701106307011070477047BF
:1008600070477047704770477047704770477047D0
:1008700070477047704770477047704770477047C0
:100880007047704710B5044601B25720FFF760FE6D
:10089000FFF705FDB0F8B000401C01B25820FFF78B
:1008A00057FE642C06D0652C09D100F065FBFF498A
:1008B00000200880BDE81040FD4800F0B5BA10BD2A
:1008C00010B5FFF7ECFCFA49448810310C8083889E
:1008D0004B80C2888A800089C8800A81488122446E
:1008E0008A811844C88110BD2DE9F04F0027DDE949
:1008F0000AA9DDF824B03E4642F2107E00EB061550
:1009000042F21074698842F210786143090B4FF487
:1009100087646143AC88B1FBFEF104FB08F4240B4F
:1009200040F6AC0804FB08F4B4FBFEF495F801C0F3
:1009300089B2A4B2BCF1010F0ED0994214D95C4522
:1009400012D9514502D3B1F5876F0DD94C4503D368
:1009500040F6AC08444507D9214302D1BCF1010F50
:1009600002D17F1CFFB21560761C0A2EC6DB4FF049
:10097000FF30002F07D0012F07D004D94FF000001F
:1009800010606FF00100BDE8F08F4FF00000FAE753
:10099000417899BB418842F210725143090B4FF4E0
:1009A0008762514342F21072808840F6AC03504394
:1009B000000B5843B0FBF2F0B1FBF2F1BC4A89B234
:1009C000103280B213898B4208D293898B4205D9A9
:1009D0005389834202D2D289824210D8B1F5C87FAE
:1009E00009D9B1F52A7F06D9B1F5E66F03D940F6EA
:1009F000AC00814203D84FF0FF307047FFE7002082
:100A0000FBE72DE9FF47AB4E002481460394307885
:100A10008846002873D0A848007800286FD1A448E1
:100A200010300189502901D25021018182894FF46F
:100A30007A718A4200D981814189C38982898DE88E
:100A40000E00038903AA41464846FFF74DFF9B4924
:100A50009C4D47F6FF77CC74994C10F1020F14D0DF
:100A6000B0F1FF3F01D0D8BB12E040F6AC024FF42A
:100A70002A714FF4E6608DE807004FF4C87303AAAB
:100A800041464846FFF730FF10B127802F8027E00E
:100A90000398407808B9FFF723FC039841780129AF
:100AA0001BD009B1022918D1418842F2107251437A
:100AB0000A0B4FF487614A4342F21071B2FBF1F224
:100AC0002A80828840F6AC034A43120B5A43B2FB99
:100AD000F1F17D4A2180018911807C4940780870BC
:100AE000307800280BD0FFF7DAFB807B4009012823
:100AF00005D16F4842464946103000F0A5FABDE8DE
:100B0000FF877FB5002540F6AC024FF47A7303955A
:100B10000095CDE90132502303AAFFF7E5FE044614
:100B200010F1020F04D0B0F1FF3F01D084BB03E00D
:100B30005F4800F079F92BE0FFF7B1FB03984078AC
:100B400008B9FFF7CDFB03984178012920D042F284
:100B50001072E9B9418813465943090B4FF4876372
:100B60005943808813465843000B40F6AC03B1FB51
:100B7000F2F15843B0FBF2F089B2CE3980B2B1F550
:100B8000277F05D840F60401884201D948484580AE
:100B90004F480078002822D04E48008800281ED1F7
:100BA000002C1CD14248039900F044F9002816D0CB
:100BB000012814D0022812D1FFF771FB4570FFF70E
:100BC0006EFB417841F002014170FFF768FB42780B
:100BD00000210846FFF7ABFB0420FFF7DFFB7FBDDA
:100BE0007FB5002640F6AC024FF47A730396009668
:100BF000CDE90132502303AAFFF776FE364C374D7C
:100C000010F1020F04D0B0F1FF3F01D070B902E043
:100C100026802E800AE0FFF742FB039841780129E5
:100C200004D042F2107241B1022906D00398002884
:100C300002D02B49407808807FBD418842F2107372
:100C40005943090B4FF487635943B1FBF2F12180FB
:100C5000808842F210714843000B40F6AC014843D3
:100C6000B0FBF2F02880E1E770B506461D4800248D
:100C70000D460278002A54D0012A52D0022A50D0C0
:100C8000652A4ED1304600F024FC29463046FFF755
:100C9000B8FE1049088800B1401E088001B27220D9
:100CA000FFF756FC294630461EE000005E070110A3
:100CB0003898011061070110640701102298011093
:100CC00074070110720701107807011076070110F0
:100CD0006007011066070110680701106A0701101C
:100CE0006C0701105D070110FFF70BFF2946304626
:100CF000FFF776FF2946304600F042F84048018869
:100D00002520FFF724FC3F4801882620FFF71FFC21
:100D10003D4801882720FFF71AFC2046BDE87040B7
:100D200036E670BD70B5394D287808B1FFF7C8FDBB
:100D3000374C38492078087010B1084600F079F82F
:100D400029782078014334480078BDE87040014399
:100D50000620FFF7AABA10B5002810D1FFF79FFAB6
:100D6000202181732949002008702A4908702A48E7
:100D700001210170BDE810400620FFF796BA10BDB2
:100D800070B50446002939D0244E002520787074AF
:100D900061783174207AF073A07AB073608800B300
:100DA000A288F2B142F210725043000B4FF48762F6
:100DB000504342F21072B0FBF2F07080A08840F60F
:100DC000AC035043000B5843B0FBF2F0B080608896
:100DD00038B1A08828B121B9707B30810120FFF79C
:100DE000DDFA307C012804D1707B30810120FFF7CF
:100DF000D5FA6D1CADB210340A2DC7D370BD0000FA
:100E00006E070110700701106C07011061070110D7
:100E10006007011038980110630701102298011033
:100E20007047704770477047002141808181417051
:100E3000704770472DE9F05F04464878DFF82C8151
:100E40000D4600276FF00B094FF0010A20B16188B1
:100E5000884601293CD134E0688800F08FFD49467E
:100E600000F09EFE424900F09DFD00F067FD86B255
:100E7000A88800F083FD494600F092FE3D4900F04D
:100E800091FD00F05BFDA6F1CE0180B2B1F5277FA8
:100E900066D840F60401884262D9618800295FD192
:100EA000298954295CD8A680E08026816081A4F835
:100EB00002A06770A781E7815046A8F80070BDE8DE
:100EC000F09F2A490228B1F9006002D001283CD0E5
:100ED00046E0688800F052FDCB46494600F060FECF
:100EE000234900F05FFD00F029FD8146A88800F04D
:100EF00045FD594600F054FE1E4900F053FD00F038
:100F00001DFDA4F808906081E0886189401A00B254
:100F1000A081B4F90E10884200DD0146E1816278BB
:100F2000012A04D0A0F24312B2F5077F0BD23C2E67
:100F300005DC4039884202DB2889542801D96770D2
:100F400001E084F801A04046B9E7607840B1032E83
:100F500006DD3C2E04DA6780A78167700220AEE7C9
:100F60006780A78167703846A9E700005E07011017
:100F70000000874400C00A450020FF4B024600EBFA
:100F80004001401C23F8112003EB410102284A8054
:100F90008A80F4DBF9484270428002707047F84959
:100FA00010B50A88F749038900240988934208D8B4
:100FB0008389934205D343898B4202D8C0898842F2
:100FC00001D24FF0FF34104600F037FA00B9002488
:100FD000204610BD30B5E94903460020497801EBB1
:100FE0004102E54901EB420419B2E54BB4F9022094
:100FF0001B88551A1BB29D420DDC0A449A420ADB3B
:10100000E04BB4F904201B88541A1BB29C4202DC4A
:101010001144994201DA4FF0FF3030BDD74A10B584
:101020005378012199435170D34B01EB410154880E
:1010300023F81140D24C03EB4101D24B24884C8061
:101040001B888B80107010BD2DE9F05F0746CC48DF
:101050000024DFF834B3028847F6FF70DFF824A3DA
:101060000E46824245D3BAF80020824241D3C3489B
:1010700000250078012801D002283AD106EB05119D
:10108000487890BB488842F210725043000B4FF4EE
:101090008762504342F21072898840F6AC0301FB2C
:1010A00002F14FEA1131B0FBF2F001FB03F1B1FBA9
:1010B000F2F10004000C89B202D03A89824210D2C7
:1010C00011B17A898A420CD2BA89824202D8B0F52B
:1010D000876F06D9FA898A4207D840F6AC02914256
:1010E00003D800F0AAF9401C2ED06D1CEDB20A2DD9
:1010F000C4D3A648008846287DD8A04EA449DFF86E
:1011000094923078012508B3012838D0DFF868823E
:10111000022859D0032855D1087801286CD002281C
:1011200050D10F214720FFF712FA7078454600EBA7
:10113000400008EB40079248B7F90220008801B24E
:10114000501A75D58B1A31E1142189E008780028EE
:1011500038D101214720FFF7FAF93846FFF71FFF82
:10116000002848DB02214720FFF7F1F9A9F80040E9
:1011700074803078401CC0B2FFF750FF20E0087840
:10118000012802D002280ED01AE003214720FFF7E1
:10119000DEF94F20FFF71EFF0028E2DB0421472085
:1011A000FFF7D5F969E005214720FFF7D0F94F2077
:1011B000FFF710FF0028D4DB06214720FFF7C7F90F
:1011C0008BF81350BDE8F09F08780028FAD107216A
:1011D0004720FFF7BCF97078424600EB40016848B1
:1011E00008EB41030088B3F902800FFA80FCB8EBEA
:1011F0000C0004D501E0B2E043E0ACEB080000B223
:101200004F2823DCBAF80000B3F904C003B2BCEBEA
:10121000030001D5A3EB0C0000B24F2816DC32F915
:101220001120B9F90010501A03D5A1EB020C01E00E
:10123000BBE084460FFA8CFCBCF1030F06DBC8460A
:10124000002800D5881A00B221280DDD082147208A
:10125000FFF77DF93846FFF7A2FE00287EDA092164
:101260004720FFF774F9E0E00A214720FFF76FF904
:10127000B8F800107180A8F800403078401C307039
:101280009EE7B9F900004F46401C68D00B2147206B
:10129000FFF75DF94F20FFF79DFE00285FDB0C2173
:1012A0004720FFF754F970883988084470803078F7
:1012B000FFF7B4FE7078C14600EB400125EA000C50
:1012C0000CEB4C0008EB410208EB4003B2F9027052
:1012D000B3F902C0B7EB0C0801D5ACEB07080FFA65
:1012E00088F74F2F43DAB2F90420B3F904304F46A0
:1012F000B2EB030C01D5A3EB020C0FFA8CF24F2AD0
:1013000035DA37F9111037F91020881A01D5531A38
:1013100000E003461BB2032B29DD002800D5501A3C
:1013200000B2212823DA0D214720FFF710F9102100
:101330004720FFF70CF90020FFF770FE70780422B9
:10134000854305EB450007EB400081884088FEF7A8
:10135000EEFF3C807C80BC80FC8001E055E064E0D6
:101360003C817C81BDE8F05F0420FFF717B80E21B7
:101370004720FFF7ECF80FE0589801107A070110AA
:1013800072070110740701102298011078070110EC
:10139000760701105E070110FFF7EEFD02203070A6
:1013A0007480FEF79DFF30783CE003461BB24F2B64
:1013B0000EDCBAF80030B7F904700FFA83FCB7EB13
:1013C0000C0301D5ACEB07031BB24F2B7FF7FAAE32
:1013D000002800D5881A01B25420FFF7B9F87078B8
:1013E00000EB400005EB4000B0F90410BAF8000033
:1013F00002B2881A00D5501A01B25520FFF7A8F89A
:101400004F215620FFF7A4F80FE011214720FFF7E6
:101410009EF83846FFF7C3FD002806DBA9F8004018
:1014200074800120BDE8F05FF8E50C488BF81340AC
:1014300044800470BDE8F05F9EE5A0F5C870B0F58B
:101440008C7F06D8B1F5E66F03D340F6AC0081423D
:1014500002D94FF0FF307047002070477A07011023
:101460002DE9F041424D43490024287830B301284A
:1014700022D16878B1F90020022826D001281BD19A
:101480006888E98803B20EB2991B00D5F11A09B237
:101490004A291CDCA9882B890EB21FB2F31B00D588
:1014A000BB1B1BB24A2B12DC142A10DC2C70082246
:1014B000FEF73DFF6C80AC80BDE8F08168780028C5
:1014C000FAD10C8001202870F6E7142AF4DD2C7084
:1014D000F0E77FB5284A1278002A47D0274A1278C9
:1014E000002A43D0002440F6AC024FF47D730394ED
:1014F0000094CDE90132442303AAFFF7F5F940B285
:101500001B4B10F1020F04D0B0F1FF3F01D058BBCC
:1015100004E047F6FF70D880188125E003984178F1
:1015200001291FD009B102291CD1418842F2107251
:101530005143090B4FF48762514342F21075B1FBDE
:10154000F5F189B2D980828840F6AC066A43120B65
:101550007243B2FBF5F292B21A81457815B91C704C
:1015600059809A8040785870FFF77AFF7FBD00005D
:101570007E0701105E07011061070110640701106A
:101580000446AFF300802046EEF77CFE7047000073
:1015900001491820ABBEFEE7260002001EF0040F32
:1015A0000CBFEFF30880EFF309800249024AF8F715
:1015B00045BD00006498011030C8011049F2452C67
:1015C000C1F2000C604748F21F7CC1F2000C60477A
:1015D00048F2D77CC1F2000C604748F6AD6CC1F20E
:1015E000000C604748F2956CC1F2000C604748F26D
:1015F0004D6CC1F2000C60474AF66B4CC1F2000C16
:10160000604749F27D7CC1F2000C604748F2837C60
:10161000C1F2000C604740F6451CC1F2000C604767
:1016200041F60F5CC1F2000C604741F6135CC1F259
:10163000000C604749F2091CC1F2000C604748F6F3
:10164000B17CC1F2000C604749F2170CC1F2000CEA
:10165000604740F2590CC1F2000C604740F2691C2F
:10166000C1F2000C604740F6870CC1F2000C6047E5
:1016700045F6413CC1F2000C604745F6493CC1F2D9
:10168000000C604744F2471CC1F2000C604742F274
:10169000830CC1F2000C604742F2750CC1F2000CE1
:1016A000604745F6F92CC1F2000C604745F6013C55
:1016B000C1F2000C604745F6034CC1F2000C6047D4
:1016C00045F6FD3CC1F2000C604749F2612CC1F2C5
:1016D000000C604749F2573CC1F2000C604746F6E7
:1016E000A51CC1F2000C604745F6E13CC1F2000CBC
:1016F000604745F6F73CC1F2000C604747F6BF7CF7
:10170000C1F2000C604745F6094CC1F2000C60477D
:1017100045F60F4CC1F2000C604747F6B74CC1F2DA
:10172000000C604749F2BD1CC1F2000C604747F64F
:10173000B14CC1F2000C604745F6ED3CC1F2000C23
:10174000604747F6C57CC1F2000C604745F6DB3CBC
:10175000C1F2000C604747F6F37CC1F2000C604711
:1017600047F6075CC1F2000C604747F6A77CC1F260
:10177000000C604747F6B17CC1F2000C604741F6AF
:101780001B7CC1F2000C604741F6077CC1F2000CE3
:10179000604741F6457CC1F2000C604749F2AD5C00
:1017A000C1F2000C604749F63B5CC1F2000C604797
:1017B00045F6093CC1F2000C604740F2AD1CC1F295
:1017C000000C604745F6B92CC1F2000C604745F6A5
:1017D000692CC1F2000C604745F68D2CC1F2000C5B
:1017E000604742F2630CC1F2000C604747F2671C8D
:1017F000C1F2000C604747F6BD4CC1F2000C6047D7
:1018000047F6A37CC1F2000C604741F6117CC1F29F
:10181000000C604740F6353CC1F2000C60474AF6C8
:10182000D13CC1F2000C604740F69F3CC1F2000C75
:1018300060474CF6517CC1F2000C604741F6175CE2
:10184000C1F2000C604745F6E73CC1F2000C60476E
:101850004AF6214CC1F2000C604746F6AB1CC1F2BF
:10186000000C604749F6AF1CC1F2000C604745F61A
:10187000C12CC1F2000C604748F2937CC1F2000C0D
:10188000604745F67D2CC1F2000C604745F6A52C5B
:10189000C1F2000C60474EF24B1CC1F2000C6047D5
:1018A00045F6C92CC1F2000C604745F62D4CC1F23B
:1018B000000C604790F8AC00012101FA00F010F034
:1018C0000A0018BF01207047DFF85CC0DCF8002078
:1018D000012A18BF7047002908BF704710B4C1EB38
:1018E000011202EB4111114A00EB8101126892F8DA
:1018F000833051F8142CBC3912F0010F0FD012F4C0
:10190000805F04BFD1F8B420012A08D1B1F90220C8
:101910009A4204DB0020CCF8000010BC70478142E2
:10192000E7D810BC704700004807011024070110D9
:10193000014800F003B900BF0000C07FC10DD1F124
:101940009E0206DB4FEA002343F0004323FA02F035
:101950007047004207D54FEA4001B1F1FE4F02D275
:101960004FF00000704710B500F09DF849922480B8
:10197000002070476FEA200070470000B0FA80F343
:1019800010FA03F2C3F19D030AD0D90501EB12202E
:10199000530638BF704700F1010008BF20F0010076
:1019A000704700004FF47F0C1CEAD0121EBF1CEAE7
:1019B000D11392EA0C0F93EA0C0F00F0478090EAE3
:1019C000010F48BF42F480724FF0004C4CEA0020F7
:1019D0004CEA012102EB0302A0FB0113A2F5000275
:1019E000002918BF43F001035B0028BF4FEA33030F
:1019F00042EB22425FEA132C4CEBC2502EBFBCEBF1
:101A0000436FB2F57C0F70474FEA036CBCF1004F97
:101A100008BF20F00100B2F57C0F38BF70470BD52E
:101A200082F0FF0212F5803FC8BF704700F1C0404E
:101A3000D8BF00F00040704700F5000C5FEA4C0C86
:101A400048BF7047B0F1C04000F073B890EA010F92
:101A50000CEAD11348BF42F48072624538BF634537
:101A600004D280EA010000F00040704710B500F099
:101A70001AF800BF8900013E00F007B800F009B86D
:101A80005FEA410C5FEA1C6C08D080EA010000F0BC
:101A900050B85FEA400C5FEA1C6CF6D14FF0004092
:101AA000A0F5800070470EF1020E2EF0030E5EF8D6
:101AB000044B244204D44FEA4102B2F17F4F11D8C3
:101AC0004FEA4003B3F17F4F0CD80ED14FEAD07CE0
:101AD000B2F17F4F0CEB4C0C0CF1020C08BF4CEB3D
:101AE000D17C04E04FF0080C01E04FEAD17C0CEB14
:101AF0004C0324FA03F404F00704B4F1040C06D2F6
:101B00000EEB840CBDE810404CF0010C6047DFE8A0
:101B10000CF0070802024FF00040A0F5800010BD55
:101B20000846420018BFD2F1807288BF00F0004022
:101B300010BDFF2141EAD050C00570470CF00F03E3
:101B4000092B08BF082000F051800A2B0BD0082B6E
:101B500018BF704708BF1CF0400F0AD04FF00000BC
:101B60004FF0000170471CF0400F18BF4FF00040CD
:101B700070471CF0100F08D020F0704300F07F4237
:101B800042EAD3014FEA4370704700F0604021F011
:101B90007F4242EA000201F07F4040EA72707047E3
:101BA0004FF0FF0212EAD0521CBF92F0FF038B42AB
:101BB000C2BFD14200EBC1507047002A0AD0002BAF
:101BC0000BD0002900F00040A4BF40F0FE4040F4DC
:101BD0000000704700F00040704743024FF00B0CCC
:101BE00018BF4CF0806C7FF4A3AE70471CF4801FCC
:101BF00011D01CF4E02F03D06FEACC3149007047BC
:101C00004FF04050EFF3008222F0704242EA0002AF
